:020000040800F2
:1000000000000120A93D00084726000849260008F5
:100010004B2600084D2600084F260008000000006F
:100020000000000000000000000000005126000851
:100030005326000800000000552600085726000837
:10004000F93D0008F93D000859260008F93D00086F
:10005000F93D0008F93D000865260008F93D000853
:10006000F93D0008F93D0008F93D0008F93D000898
:10007000F93D0008F93D0008F93D0008F93D000888
:10008000F93D00086D260008F93D0008F93D00081B
:1000900000000000F93D0008F93D0008F93D0008A6
:1000A000F93D0008F93D0008F93D0008F93D000858
:1000B000F93D0008F93D0008F93D0008F93D000848
:1000C000F93D0008F93D0008F93D0008F93D000838
:1000D000F93D000879260008F93D0008F93D0008BF
:1000E000F93D0008F93D000885260008F93D0008A3
:1000F000F93D00080000000000000000F93D000884
:10010000F93D0008F93D000891260008F93D000876
:10011000F93D0008F93D0008F93D0008F93D0008E7
:10012000F93D0008F93D0008F93D0008F93D0008D7
:08013000F93D0008F93D00084B
:1001380010B5054C237833B9044B13B10448AFF319
:1001480000800123237010BD4C0100200000000036
:10015800380C010808B5034B1BB103490348AFF33A
:10016800008008BD0000000050010020380C010884
:1001780014214160704714207047406A704700009E
:10018800790100087F01000883010008990100082F
:1001980010B5044604F1100000F05CFCC4F8F80047
:1001A8000148C4F87C0110BD88010008F8B5E6B024
:1001B80004460D4616461F460A4906A800F0CAFE20
:1001C80070996F9A05910492009733466E996D9ACB
:1001D800039102922A466C990191214600F060F839
:1001E80067B0F0BD94010008F8B5E6B004460D46C6
:1001F80016461F46094906A800F0ACFE6F996E9A8C
:100208000491039200976D996C9A0291019233467A
:100218002A46214600F087F867B0F0BD940100082F
:1002280038B500281CBF01680029184A23D1184B8B
:100238001C684FF6F0710C404CF24025AC421FBFD1
:100248001B6819404CF27024A14212D1114D296843
:1002580079B911490B68C3F30B03B3F58A6F1FBF54
:100268000968C1F30B0140F28343994204BF01219D
:10027800117028B905E0094B994204BF012111709A
:100288004068BDE8324001F09FBE00BF6801002011
:1002980000ED00E0002004E00010005C000037489A
:1002A8002DE9F04104460D46216816464A681F4666
:1002B80090478046B8F5403F2ED122680A99936846
:1002C800204698478046B8F5403F25D12368089ACC
:1002D8000799D3F80CC02046E0478046B8F5403F60
:1002E8001AD12368069A39461F692046B8478046BE
:1002F800B8F5403F10D1236829465D69324620464B
:10030800A8478046B8F5403F06D123680B9A09995B
:100318009D692046A847804621680A68204690477C
:100328004046BDE8F0812DE9F04104460D462168BC
:1003380016464A681F4690478046B8F5403F2ED17A
:1003480022680A999368204698478046B8F5403F46
:1003580025D12368089A0799D3F80CC02046E047AE
:100368008046B8F5403F1AD12368069A39461F6976
:100378002046B8478046B8F5403F10D12368294643
:100388005D6932462046A8478046B8F5403F06D109
:1003980023680999DD6900222046A847804621681C
:1003A8000A68204690474046BDE8F0814FF4403047
:1003B80070470000F0B50C4685B0114600281A4673
:1003C8001CBF0568002D0B4B11D082B104B971B95F
:1003D8000D9860B10F9E0E9F0A9B0290049603979A
:1003E8000B980C9E009001962046A8470346184695
:1003F80005B0F0BD020003002DE9F04F0646D0B06D
:100408000868F56DD6F860E0726EB76EF36E00BAE4
:1004180000906C46486800BA60600DF14008886832
:1004280000BAA060C86800BAE060086900BA206134
:10043800486900BA6061886900BAA061C86900BAF1
:10044800E061086A00BA2062486A00BA6062886A95
:1004580000BAA062C86A00BAE062086B00BA2063FA
:10046800486B00BA6063886B00BAA063C86B00BAB7
:10047800E063402058F80C1C58F820CC58F838ACE9
:100488008CEA010158F840CC8AEA01018CEA01099A
:100498004FEAF979401E48F8049BEBD187EA02003D
:1004A80000EA0E00784010EBF5610098DFF824C4EC
:1004B80041186144C81882EABE032B404FEAF06134
:1004C80053405918636859186144CF194FEAB50366
:1004D80083EABE01014081EABE0111EBF765A1681C
:1004E8004D196544A91883EAB0023A404FEAF1650C
:1004F8005A405519E26855194FEAB70282EAB0071F
:1005080065440F4005EBBE0E97EAB00717EBFE6592
:1005180027697D194FEAB10782EA0701654401EAB4
:100528000E01EB18514011EBF36561694D194FEA63
:10053800BE0187EA010E65440EEA030E15EBB00012
:100548008EEA070E0EEBF065D4F818E075446544A2
:10055800AA1881EAB30505404FEAF26E4D40AE4451
:10056800E569AE44E64477444FEAB00080EAB30E4A
:100578000EEA020E8EEAB30E0EEBF765D4F820E011
:1005880075446544691880EAB2053D404FEAF16E4A
:100598004540AE44656AAE44E6440EEBB3034FEA09
:1005A800B70787EAB20E0EEA010E8EEAB20E0EEB1C
:1005B800F365D4F828E075446544281887EAB1053E
:1005C8001D404FEAF06E7D40AE44E56AAE44E64415
:1005D8000EEBB2024FEAB30383EAB10E0EEA000E45
:1005E8008EEAB10E0EEBF265D4F830E0754465443E
:1005F800EF1983EAB00515404FEAF76E5D40AE4447
:10060800656BAE44E6440EEBB1014FEAB20282EAF2
:10061800B00E0EEA070E8EEAB00E0EEBF165D4F8B6
:1006280038E075446544EB1882EAB7050D404FEA97
:10063800F36E5540AE44E56BAE44E6440EEBB000B5
:100648004FEAB10181EAB70E0EEA030E8EEAB70E41
:100658000EEBF065D4F840E07544654481EAB30ECA
:10066800AA180EEA000E4FEAF2658EEA010E7544EA
:10067800DDF844E04FEAB000754480EAB30E654403
:100688000EEA020E15EBB7078EEAB30E0EEBF7650E
:10069800DDF848E04FEAB202754480EA020E65448C
:1006A8000EEA070E69188EEA000E0EEBF165DDF80A
:1006B8004CE07544654405EBB3034FEAB70E1427C5
:1006C8000DF1500CDFF810528EEA010B82EA0B0B89
:1006D8000BEBF36A5CF804BBDA44AA44504483EA9F
:1006E800B10B4FEAF06A8EEA0B0BDA445CF804BBF4
:1006F800DA44AA44524480EAB30B4FEAF26A8BEA1E
:10070800B10BDA445CF804BBDA444FEAB000AA44FF
:1007180080EA020BD6448BEAB30B0BEBFE6A5CF85B
:1007280004BBDA444FEAB202AA4482EA0E0B0AEB8F
:10073800B10180EA0B0B0BEBF16A5CF804BBDA44FD
:100748007F1DAA44282F0AEBB3034FEABE0EBBD382
:100758003C2F61D3502F4DD204EB870CC7F15407BF
:100768005E4CA7FB04A504465D4FA8088EEA010A63
:1007780082EA0A0A5CF804BB0AEBF3655D447D195A
:100788002C1983EAB10A4FEAF4658EEA0A0A55443D
:100798005CF804AB5CF804BB55447D19AA1884EADC
:1007A800B30A4FEAF2658AEAB10A55445D444FEA52
:1007B800B4047D1984EA020AAE448AEAB30A0AEB51
:1007C800FE655CF804AB55444FEAB2027D1982EA33
:1007D8000E0A15EBB10184EA0A0A5CF804BB0AEBBD
:1007E800F1655D447D1915EBB303401E4FEABE0E5B
:1007F800BCD12046F46D1B19F365336EC9183166F8
:10080800716E71447166B36ED218B266F16E40189B
:10081800F06650B0BDE8F08F4EEA010B0EEA010A0F
:100828000BEA020B4BEA0A0A0AEBF36554F827A015
:10083800DFF8B0C0554443EAB10B654403EAB10A96
:100848000BEA0E0B28184BEA0A0A7F1C0AEBF06524
:1008580054F827A0554440EAB30B654400EAB30AAC
:100868000BEAB10BAA184BEA0A0A7F1C0AEBF265DD
:1008780054F827A055444FEAB00040EA020B6544FB
:1008880000EA020A0BEAB30BAE444BEA0A0A7F1CE1
:100898000AEBFE6554F827A055444FEAB20242EA33
:1008A8000E0B654402EA0E0A0BEA000B15EBB101C8
:1008B8004BEA0A0A7F1C0AEBF16554F827A0554455
:1008C8007F1C65443C2F05EBB3034FEABE0EA3D350
:1008D80040E700BF9979825AA1EBD96ECDCCCCCC38
:1008E800D6C162CADCBC1B8F00B581B00168074A5B
:1008F800914200D110B9064801B000BD7C2110F02A
:10090800FFF84FF4003001B000BD00BFFC0900083B
:10091800030002002DE9F0410B4A92E8F85188B033
:10092800694681E8F8510268084B9A4200D118B923
:10093800074808B0BDE8F0811422083000F04FFBEA
:1009480008B0BDE8F08100BFDC090008FC09000818
:1009580003000200152904D20268044B9A4200D110
:1009680008B903487047083000F048BBFC09000884
:100978000300020010B481B013460268074CA2427B
:1009880000D118B901B010BC0548704701B000F19A
:10099800240210BC083000F035BB00BFFC09000879
:1009A8000300020010B481B013460268074CA2424B
:1009B80000D118B901B010BC054870470A4601B00B
:1009C80000F1240110BC083000F070BBFC090008DD
:1009D800030002000123456789ABCDEFFEDCBA981E
:1009E80076543210F0E1D2C300000000000000008D
:1009F80000000000F10800081D0900085D09000852
:100A08007D090008AD09000801040008790F0008F5
:100A1800C50F0008810F0008F0B5A3B004460B48C5
:100A280002900D4616461F46094B0822402104A88D
:100A380000F0D1FA28980190009733462A462146BB
:100A480002A800F01BF823B0F0BD00BFFC090008A5
:100A5800100A000810B5040008BF002408D0054893
:100A6800054B20600822402104F1080000F0B3FA89
:100A7800204610BDFC090008100A00082DE9F041C5
:100A880004460E46216817464A681D469047804628
:100A9800B8F5003F19D1226806999368204698470F
:100AA8008046B8F5003F10D123683146DE683A46E3
:100AB8002046B0478046B8F5003F06D12368079A1C
:100AC80029461D692046A847804621680A682046AD
:100AD80090474046BDE8F08110B500F033FA4FF476
:100AE800403400280EBF034C4FF4C07110F008F8D2
:100AF800204610BD0200030010B5044600F022FA9B
:100B080008B9054810BD0021A160D0F87C21116802
:100B180088474FF4403010BD0200030070B504460A
:100B28000D4600F00FFA064E40B1D0F87C0141683E
:100B38008847A84224BF65604FF44036304670BDF0
:100B4800020003002DE9FF4715000C4600D02CB128
:100B5800064600F0F7F95FEA000801D16448C3E0EF
:100B6800D8F8F80001684A689047B0F5003F17D1F7
:100B7800D8F87C118A68404690478146B9F1810FC0
:100B880080F09E80A94508F1FC0A17D2D8F8F80031
:100B98000368D3F80CC02A462146E047B0F5003F69
:100BA80040F08E80D8F8F8000368D3F810C06A4681
:100BB8005146E047B0F5003F76D10AE0002004E056
:100BC800215C0AF800100098401C00900098A84288
:100BD800F6D34FF0000C4749474A484B01AC009800
:100BE800844558D2D3E9007001ADC5E9007010788A
:100BF80000281ABF042086464FF0000E085854F803
:100C08000E5028443E4D05600127D0F800E087606B
:100C1800019D4F681AF80C007D408EEA050585F0A5
:100C2800040E65680F687D4085F0FC05754485F005
:100C3800A30568400AF80C000CF1010CCFE7D3E9D2
:100C4800004501A8C0E9004510782E4D002814BFC2
:100C58004FF0040E4FF0000E01A8744651F80EE054
:100C68000459A6440127CEF80050DEF80040CEF81B
:100C780008704D68019F40687D406C400D68684071
:100C880084F0040480F0FC00041984F057040AF886
:100C98000C400CF1010CCC45D1D3D8F8F800016810
:100CA8004A689047B0F5003F0AD1D8F8F8000368C1
:100CB800D3F80C804A465146C047B0F5003F01D0F2
:100CC800114811E0002006E05AF8201081F06A313E
:100CD8004AF82010401CB0EB990FF5D3B06840F0EB
:100CE8000100B0604FF4403004B0BDE8F08700BFA9
:100CF80002000300D00C010868010020240F00083E
:100D0800ADBE4ED70DBE75A10100030038B50C4627
:100D1800017A1546CA0702D500F014F908B908483F
:100D280032BDD0F8F80003682146DC682A46A0479F
:100D3800B0F5003F01D0034832BD4FF4403032BD1A
:100D480002000300010003002DE9F84191B00546B7
:100D58000E461746402101A80FF0D2FE297AC8078F
:100D680004D5284600F0EEF8040002D1DFF8A4808C
:100D78004BE0D4F8F800DFF8A0800368D3F810C07F
:100D88006A4601A9E047B0F5003F3ED1D4F8F80023
:100D980001684A689047B0F5003F36D1D4F87C1115
:100DA8008A6820469047D4F8F830024618461B68EF
:100DB800D3F80CC004F1FC01E047B0F5003F24D1A2
:100DC800D4F87C0141688847D4F8F83002461846C0
:100DD8001B68D3F80CC001A9E047B0F5003F14D157
:100DE800D4F8F8000268696893689847B0F5003F3E
:100DF8000BD1D4F8F80003681C693A463146A0477D
:100E0800B0F5003F08BF4FF44038404612B0BDE887
:100E1800F08100BF02000300010003002DE9F84142
:100E2800A5B0074688461646402115A80FF068FE6B
:100E380000220492402105A80FF062FE387AC1070B
:100E48005ED5384600F07EF8050059D0D5F8F80090
:100E58002D4C0368D3F810C06A4605A9E047B0F5E1
:100E6800003F3CD1D5F8F80001684A689047B0F5D2
:100E7800003F34D1D5F87C118A6828469047D5F8C8
:100E8800F830024618461B68D3F80CC005F1FC017F
:100E9800E047B0F5003F22D1D5F87C01416888478A
:100EA800D5F8F830024618461B68D3F80CC005A9D7
:100EB800E047B0F5003F12D1D5F8F800026879682C
:100EC80093689847B0F5003F09D1D5F8F800036852
:100ED8001D6904AA15A9A847B0F5003F01D020460E
:100EE8000FE00A4B0A490B4A0396029101924046C9
:100EF8001C68049B009415AA796800F0E5F900E0E5
:100F0800054826B0BDE8F08101000300D80C0108AF
:100F1800936E030026C703000200030004B001011A
:100F280000170145E10A0008010B0008250B00081D
:100F3800B50300084D0B0008150D0008510D0008F9
:100F4800250E00080168024A914218BF0020704728
:100F58002C0F000810B5040008BF002404D0034873
:100F68002060204609688847204610BD2C0F0008DD
:100F780020225C300FF0C2BDF0B58468A3080022BF
:100F880004F0030407E000F15C0555F8226035BA67
:100F980041F82250521C9A42F5D300220BE000F18E
:100FA8005C0502EB830755F82360D500C5F11805E9
:100FB800EE40CE55521CA242F1D3F0BD30B5C46804
:100FC80003690022E31AD5188C5C0544521C082AD0
:100FD8002C77F8D330BD0360C1600261704738B523
:100FE800044615460022626023685A68904700202C
:100FF8006061A061A5604FF4003032BD81604FF49C
:10100800003070472DE9F84304462079D4F80C8065
:10101800450748BF244845D466691D46A8F1010024
:1010280000EAD60306EBC506B6EBC50F666102D229
:10103800A669761CA6611746A66906EB5576A661D1
:101048000E46E918884225D2A8EB03094A463146DC
:10105800F8180FF053FD2268136839460FE042462E
:1010680038460FF04BFD23681A68394620469047EA
:1010780007E0311811F00300F1D122681368204607
:101088009847484600EB0809A9F10101A942F0D3A5
:10109800002300E000202A1A3118F8180FF02EFD5E
:1010A8004FF40030BDE8F283040002002DE9FC4F44
:1010B800024685B0D0681369DFF86CC1DFF86C812F
:1010C800A0EB030A506840F004005060002703A812
:1010D80002900DF10C0ED8E9003403A8544DC0E974
:1010E80000342878534D00280CBF00230423994668
:1010F8005CF803305EF80940234401261D601C6833
:101108009E60DCF80430039DDCF80090DEF8046093
:101118005D406540484C654089EA0606474C664094
:101128007519474C6540D8E9006B03AC0028C4E941
:10113800006B0EBF002404200424029E5CF800000B
:10114800345920183F4C04600126046886600398CF
:10115800029E43406340384C7068634089EA00004F
:10116800364C6040034438484340280018BF0120EB
:101178005B1E9B41042F2CBFC0B2D80F02F1140391
:1011880053F8200007F00303C3F10303DB00D84042
:101198000DF807007F1C082F9DD315460C466A6979
:1011A800AB69E868D20842EA4372401E00EA0207C7
:1011B800002302409B420AD8524508D28020E055BD
:1011C8007F1C574516D2AAEB0701E01910E08020D2
:1011D800E05500E0E355E8687F1C8742FAD32A68A7
:1011E800136828469847BAF1000F03D051462046A5
:1011F8000FF086FC2A68069E059F93686946284674
:1012080098472A68D2F8009021462846C8472B6894
:10121800DA683946284690470EB1A86830604FF41E
:10122800003007B0BDE8F08FD00C01085412000858
:10123800680100205FC5109304850012FC68017ADC
:10124800C0F524FF24AF33D426AF698B04B0010165
:1012580000170145F8B501240094002300240DE08F
:10126800009D065D0F5D7E40F643761CF60F86F006
:10127800010635400095641C009DEB189442EFD39D
:101288001846F2BDF8B5002301240094002A11E0A5
:10129800009C85188F1815F8016C17F8015C6E40D2
:1012A800F643761CF60F86F0010634400094009C45
:1012B800E318521EECD11846F2BD00005D1200087A
:1012C8008D120008010000002DE9F84F1D46DDF8D9
:1012D80028900B9F0D9C4FF0FF3300930E469246CB
:1012E800D9F800B0804632465146D847834664B3A1
:1012F800D9F8043032465146404698476FEA0B0207
:10130800521C42EA0B0200996FEAD2735B1C194027
:10131800C2430091521C024300996FEAD2735B1CCE
:101328001940009186F05531484087EA000181F064
:101338005531216080F05531C943491C0843009A52
:101348006FEAD070401C82430092D9F80800012847
:1013580009D17540E943491C0D4300986FEAD572DD
:10136800521C90430AE0F11C85EA9102D243521CB8
:10137800154300986FEAD5735B1C984386F0AA362C
:10138800009086EA0B0686F0AA33F243DB430C98FA
:10139800C2F3C0725B1C42EAD3720099D243521C5A
:1013A80091430091774000998843009987F0AA37C4
:1013B8000F403843BDE8F28F034613F8012B002A8B
:1013C800FBD1181A0138704781F0004102E000BFD4
:1013D80083F0004330B54FEA41044FEA430594EAED
:1013E800050F08BF90EA020F1FBF54EA000C55EA28
:1013F800020C7FEA645C7FEA655C00F0E2804FEAF9
:101408005454D4EB5555B8BF6D420CDD2C4480EADA
:10141800020281EA030382EA000083EA010180EA0A
:10142800020281EA0303362D88BF30BD11F0004F58
:101438004FEA01314FF4801C4CEA113102D040428E
:1014480061EB410113F0004F4FEA03334CEA1333C9
:1014580002D0524263EB430394EA050F00F0A780E1
:10146800A4F10104D5F1200E0DDB02FA0EFC22FADC
:1014780005F2801841F1000103FA0EF2801843FAD0
:1014880005F359410EE0A5F120050EF1200E012AC1
:1014980003FA0EFC28BF4CF0020C43FA05F3C018FF
:1014A80051EBE37101F0004507D54FF0000EDCF178
:1014B800000C7EEB00006EEB0101B1F5801F1BD321
:1014C800B1F5001F0CD349085FEA30004FEA3C0C25
:1014D80004F101044FEA445212F5800F80F09A801B
:1014E800BCF1004F08BF5FEA500C50F1000041EB1F
:1014F800045141EA050130BD5FEA4C0C404141EB23
:101508000101013C28BFB1F5801FE9D291F0000F1D
:1015180004BF01460020B1FA81F308BF2033A3F1CC
:101528000B03B3F120020CDA0C3208DD02F1140CC3
:10153800C2F10C0201FA0CF021FA02F10CE002F1FE
:101548001402D8BFC2F1200C01FA02F120FA0CFCF7
:10155800DCBF41EA0C019040E41AA2BF01EB045140
:10156800294330BD6FEA04041F3C1CDA0C340EDC3E
:1015780004F11404C4F1200220FA04F001FA02F381
:1015880040EA030021FA04F345EA030130BDC4F13F
:101598000C04C4F1200220FA02F001FA04F340EA34
:1015A8000300294630BD21FA04F0294630BD94F0E5
:1015B800000F83F4801306BF81F480110134013DCC
:1015C8004EE77FEA645C18BF7FEA655C29D094EA3D
:1015D800050F08BF90EA020F05D054EA000C04BFBB
:1015E8001946104630BD91EA030F1EBF00210020A6
:1015F80030BD5FEA545C05D14000494128BF41F045
:10160800004130BD14F580043CBF01F5801130BDA8
:1016180001F0004545F0FE4141F470014FF0000033
:1016280030BD7FEA645C1ABF194610467FEA655CE4
:101638001CBF0B46024650EA013406BF52EA033586
:1016480091EA030F41F4002130BD00BF90F0000F74
:1016580004BF0021704730B54FF4806404F13204B0
:101668004FF000054FF0000150E700BF90F0000F69
:1016780004BF0021704730B54FF4806404F1320490
:1016880010F0004548BF40424FF000013EE700BF60
:1016980042004FEAE2014FEA31014FEA02701FBFF0
:1016A80012F07F4393F07F4F81F06051704732F022
:1016B8007F4208BF704793F07F4F04BF41F4002179
:1016C800704730B54FF4607401F0004521F00041D7
:1016D8001CE700BF50EA010208BF704730B54FF061
:1016E80000050AE050EA010208BF704730B511F062
:1016F800004502D5404261EB41014FF4806404F19A
:1017080032045FEA915C3FF4D8AE4FF003025FEA1F
:10171800DC0C18BF03325FEADC0C18BF033202EBA3
:10172800DC02C2F1200300FA03FC20FA02F001FAFD
:1017380003FE40EA0E0021FA02F11444BDE600BFA0
:101748004FF0FF3C06E000BF4FF0010C02E000BF85
:101758004FF0010C4DF804CD4FEA410C7FEA6C5C68
:101768004FEA430C18BF7FEA6C5C1BD001B050EA0B
:10177800410C0CBF52EA430C91EA030F02BF90EAF6
:10178800020F0020704710F1000F91EA030F58BFB5
:10179800994208BF90422CBFD8176FEAE37040F017
:1017A800010070474FEA410C7FEA6C5C02D150EAB5
:1017B800013C07D14FEA430C7FEA6C5CD6D152EA70
:1017C800033CD3D05DF8040B704700BF8446104635
:1017D80062468C461946634600E000BF01B5FFF734
:1017E800B7FF002848BF10F1000F01BD4DF808ED04
:1017F800FFF7F4FF0CBF012000205DF808FB00BFD5
:101808004DF808EDFFF7EAFF34BF012000205DF82E
:1018180008FB00BF4DF808EDFFF7E0FF94BF01207B
:1018280000205DF808FB00BF4DF808EDFFF7CEFF7C
:1018380094BF012000205DF808FB00BF4DF808EDBB
:10184800FFF7C4FF34BF012000205DF808FB00BF8C
:101858004FEA410212F5001215D211D56FF47873D0
:10186800B3EB625212D94FEAC12343F0004343EA73
:10187800505311F0004F23FA02F018BF404270474E
:101888004FF00000704750EA013005D111F00040D8
:1018980008BF6FF0004070474FF00000704700BF6E
:1018A80080F0004002E000BF81F0004142001FBF0D
:1018B8005FEA410392EA030F7FEA226C7FEA236C16
:1018C8006AD04FEA1262D2EB1363C1BFD21841400B
:1018D80048404140B8BF5B42192B88BF704710F0A1
:1018E800004F40F4000020F07F4018BF404211F044
:1018F800004F41F4000121F07F4118BF494292EAAC
:10190800030F3FD0A2F1010241FA03FC10EB0C00D7
:10191800C3F1200301FA03F100F0004302D5494264
:1019280060EB4000B0F5000F13D3B0F1807F06D311
:1019380040084FEA310102F10102FE2A51D2B1F109
:10194800004F40EBC25008BF20F0010040EA0300FE
:101958007047490040EB0000013A28BFB0F5000F7E
:10196800EDD2B0FA80FCACF1080CB2EB0C0200FA34
:101978000CF0AABF00EBC25052421843BCBFD04083
:101988001843704792F0000F81F4000106BF80F4FD
:1019980000000132013BB5E74FEA41037FEA226CC0
:1019A80018BF7FEA236C21D092EA030F04D092F08B
:1019B800000F08BF0846704790EA010F1CBF0020BF
:1019C800704712F07F4F04D1400028BF40F000401C
:1019D800704712F100723CBF00F50000704700F03C
:1019E800004343F0FE4040F4000070477FEA226263
:1019F80016BF08467FEA23630146420206BF5FEA34
:101A0800412390EA010F40F4800070474FF0000333
:101A180004E000BF10F0004348BF40425FEA000CFA
:101A280008BF704743F0964301464FF000001CE0A2
:101A380050EA010208BF70474FF000030AE000BFF8
:101A480050EA010208BF704711F0004302D5404236
:101A580061EB41015FEA010C02BF844601460020A8
:101A680043F0B64308BFA3F18053A3F50003BCFAC3
:101A78008CF2083AA3EBC25310DB01FA02FC634470
:101A880000FA02FCC2F12002BCF1004F20FA02F277
:101A980043EB020008BF20F00100704702F120026A
:101AA80001FA02FCC2F1200250EA4C0021FA02F2CB
:101AB80043EB020008BF20EADC7070474FEA40029F
:101AC800B2F1FE4F0FD34FF09E03B3EB12620DD964
:101AD8004FEA002343F0004310F0004F23FA02F0CE
:101AE80018BF404270474FF00000704712F1610F75
:101AF80001D1420205D110F0004008BF6FF000404C
:101B080070474FF00000704753B94AB9002908BF21
:101B180000281CBF4FF0FF314FF0FF3000F070B9C4
:101B2800ADF1080C6DE904CE00F006F8DDF804E02C
:101B3800DDE9022304B070472DE9F047089E0D4601
:101B480004460F46002B4AD18A42944665D9B2FA18
:101B580082F343B102FA03FCC3F120029F4020FA4A
:101B680002F217439C404FEA1C4E1FFA8CF5B7FB54
:101B7800FEF1220C0EFB117742EA074201FB05F049
:101B880090420AD91CEB020201F1FF3780F01B8159
:101B9800904240F2188102396244121AA4B2B2FB90
:101BA800FEF00EFB102244EA024400FB05F5A542B4
:101BB8000AD91CEB040400F1FF3280F00681A5422B
:101BC80040F203816444023840EA0140641B00216A
:101BD8001EB1DC400023C6E90043BDE8F0878B4214
:101BE80008D9002E00F0EC800021C6E9000508465F
:101BF800BDE8F087B3FA83F1002949D1AB4202D39B
:101C0800824200F2F780841A65EB0302012017462E
:101C1800002EE2D0C6E90047DFE702B9FFDEB2FADC
:101C280082F3002B40F08F808A1A4FEA1C471FFA74
:101C38008CFE0121B2FBF7F507FB1520220C42EAC6
:101C480000420EFB05F0904208D91CEB020205F198
:101C5800FF3802D2904200F2CA804546121AA4B256
:101C6800B2FBF7F007FB102244EA02440EFB00FE29
:101C7800A64508D91CEB040400F1FF3202D2A645A0
:101C880000F2BA801046A4EB0E0440EA05409FE734
:101C9800C1F120078B4022FA07FC4CEA030C05FA35
:101CA80001F420FA07F3FD40234300FA01F94FEA53
:101CB8001C401FFA8CFEB5FBF0F81C0C00FB1855F5
:101CC80044EA054408FB0EF5A54202FA01F20BD9D5
:101CD8001CEB040408F1FF3A80F08780A54240F22B
:101CE8008480A8F102086444641B9DB2B4FBF0F33D
:101CF80000FB134445EA044403FB0EFEA64508D93D
:101D08001CEB040403F1FF306BD2A64569D9023BF2
:101D1800644443EA0840A0FB0283A4EB0E049C42FF
:101D2800C6461D4655D352D056B1B9EB0E0364EBE7
:101D3800050404FA07F7CB40CC401F43C6E90074FA
:101D48000021BDE8F087C3F1200102FA03FC20FA64
:101D580001F225FA01F19D402A434FEA1C471FFA78
:101D68008CFEB1FBF7F007FB1015110C41EA054199
:101D780000FB0EF58D4204FA03F408D91CEB0101AF
:101D880000F1FF382FD28D422DD902386144491B0A
:101D980092B2B1FBF7F507FB151142EA014205FBC8
:101DA8000EF1914208D91CEB020205F1FF3816D258
:101DB800914214D9023D6244521A45EA004139E77A
:101DC8003146304609E73946E7E61046FCE6C145A4
:101DD800AAD2B8EB020E63EB0C050138A4E745461E
:101DE800EAE7034695E74046D1E7D0467CE7023D5F
:101DF800624433E708460BE76444023843E700BF10
:101E0800704700BF1348144A08B54FF00043C0E9B3
:101E180000230422002342610122C2614FF4805151
:101E280007220383C0E90233C0E90933C0E90C1271
:101E38000361837680F8203080F82C30826380F844
:101E48003C30C36402F084F818B1BDE8084000F0E3
:101E58004BBB08BD6C010020002401400268084B00
:101E68009A4282B00AD14FF0B0431A6E42F400721F
:101E78001A661B6E03F400730193019B02B070474E
:101E8800002401400268054B9A4201BF4FF0B0425E
:101E9800136E23F400731366704700BF00240140DB
:101EA80030B585B000240546CDE901440394FFF719
:101EB800A9FF144802F0E4FB08B100F015FB114833
:101EC800039401A9CDE9015402F0A0F908B100F08A
:101ED8000BFB0C4802F0FEFA08B100F005FB4FF0CE
:101EE800FF31084802F034F9064802F0ABFB054818
:101EF80002F088F90446034802F04EFB204605B07C
:101F080030BD00BF6C010020014B024A1A607047C7
:101F18006C0100200024014008B50948FFF7C0FF04
:101F280068B1084BB3F8AA304FF6FF72934216BF58
:101F380040F6E442044B5343B3FBF0F398B208BDB8
:101F4800002000B40075FF1FD8084C0013B500230B
:101F5800ADF80630FFF7E0FF04461948FFF7A0FF89
:101F6800184BB3F8C820B3F8A8108A4204FB00F055
:101F780018D040F6E443B0FBF3F364205B1A434304
:101F8800521A93FBF2F31E331BB2ADF80630BDF8BC
:101F980006305BB21B02ADF80630BDF8060000B291
:101FA80002B010BD4FF47A7240F6FF73B0FBF3F342
:101FB8005343A3F53923A3F50C6340F6C412E0E7B5
:101FC800001000B00075FF1F4FF0B04382B09A6A4E
:101FD80022F480529A629A6C42F480529A649B6C02
:101FE80003F480530193019B002002B070474FF027
:101FF800B04307B59A6C42F004029A649A6C02F0F6
:1020080004020192019A9A6C42F001029A649B6C54
:10201800002203F00103009311461120009B02F0F7
:10202800CDFB112003B05DF804EB02F0F9BB000012
:1020380008B502F04BFE10B16FF0040008BD064B66
:102048009A6942F040429A614CF2FA321A6102F0FF
:102058004FFE0028F2D0EFE700400058F0B585B0F9
:1020680000230C4600930646A8B3FFF7E1FF054698
:1020780070BB02F02BFE88BB1A481B4A022301934F
:10208800D0F8E01506F1784302EA8121B3FBF1F7B5
:1020980001FB1733DB0A0293D0F8E00504F178411D
:1020A8000139314402EA8022B1FBF2F002FB10113F
:1020B800C3EBD1230133694601A8039302F098FECC
:1020C80020B102280CBF01256FF0010502F010FEB7
:1020D800284605B0F0BD6FF00505F9E76FF0040577
:1020E800F6E700BF0070FF1F00FCFF03014B1860FC
:1020F80000207047D00100202DE9F04F89B0B0F1E1
:10210800006F06460F460092C0F0C580DFF8988140
:10211800664DD8F8E03505EA832303F10063013BF7
:10212800984200F2B880002800F0B880002900F03A
:10213800B58040EA02035B0740F0B080FFF778FF04
:102148000446A0BB02F0C2FD002840F0AA80D8F8DF
:10215800E01506F1784205EA8121B2FBF1F301FBB3
:102168001322009B03F17843013B3344B3FBF1F0A6
:1021780001FB1033DB0A01334FEAD22AA3EBD22248
:10218800012A039388BFC6F30A050AF58038C6F109
:10219800080398BF009D069388BFC5F500654FEA00
:1021A800C828B346039B9A4505D302F0A1FD2046F3
:1021B80009B0BDE8F08FA6F10803069A1A449542C3
:1021C80019D804950197CDF814B04FF00009059B74
:1021D80009EB0301049B99453ED3009BAB442F4474
:1021E8005D1BB5F5006F28BF4FF400650AF1010AC1
:1021F80008F50068D6E753F8081F5A68B2F1FF3FA0
:1022080008BFB1F1FF3FD8D0294B186810B96FF05B
:102218000504CAE7B8F1000F04D04FF40062414644
:102228000EF008F8DFF88890D9F80030CBF30A00F0
:1022380039461844AAB20DF0FDFF4FF4006140463C
:10224800FFF70CFF08BBD9F8003001934FF4006387
:10225800CDF814800493B8E7019B07914B4402938F
:102268000120D3E9002302F07DFD88B90799019B7D
:10227800D1E9000259F80310029B5B689A4208BF33
:10228800884205D109F10809A1E76FF001048CE73C
:102298006FF0030489E74FF0FF3488E76FF0050417
:1022A80085E76FF0040482E70070FF1F00FCFF035E
:1022B800D0010020B1F1006F70B511D30B4BD3F8EA
:1022C800E0650B4B03EA862303F10063013B994267
:1022D80006D840B139B192B20DF0ACFF002070BD04
:1022E8004FF0FF30FBE76FF00500F8E70070FF1FC5
:1022F80000FCFF03B0F1006F10B40DD3084BD3F806
:10230800E045084B03EA842303F10063013B98424C
:1023180002D810BCFFF7A2BE4FF0FF3010BC7047C8
:102328000070FF1F00FCFF034FF0B04382B0DA6C6F
:102338000243DA64DB6C03400193019B02B07047EF
:1023480070B5012086B00024284ECDE90444FFF77B
:10235800EBFF0220FFF7E8FF0420FFF7E5FF0DEB96
:1023680000014FF6FF7203233046CDE901230394A1
:1023780002F08CFD01A91E4802F088FD01A94FF06A
:10238800904002F083FD4FF0B0420120D36C23F05F
:102398000403D364FFF7C8FF4FF44413CDE90230B8
:1023A8000546019001A94FF0904002F06FFD022010
:1023B800FFF7BAFF01A910233046CDE90135CDE971
:1023C800034402F063FD22462146062002F0F6F996
:1023D800062002F025FA22462146072002F0EEF9EF
:1023E800072002F01DFA06B070BD00BF00040048C7
:1023F8000008004800B59BB04822002108A80EF04C
:1024080051FB1822002102A80EF04CFB02F076FEC8
:102418004FF0B0420120D2F8903023F01803C2F8F0
:102428009030D2F8003423F4C06343F40073C2F848
:102438000034D2F8003403F4C0630193019B2423D1
:10244800089381230B930023CDE91003B02208A839
:10245800CDE9122303F01CF808B172B6FEE74F234A
:10246800CDE90230CDE90400CDE90600022102A839
:1024780003F0A8FA08B172B6FEE71BB05DF804FBDA
:1024880008B501F02BFDFFF7B5FFFFF759FFFFF780
:10249800AEFD0121002001F0B9FC0121002002F06D
:1024A8006FFE02F0A5FE0E4BD3F88820D2050ED59C
:1024B8000122C3F888204FF47A7000F041FA0948E5
:1024C8000022042102F008FE00F029FDFCE700F0DC
:1024D8001FFD04480122042102F0FEFDEBE700BFC6
:1024E800000400580004004872B6FEE70F4808B51B
:1024F8000F4B03601F2383604FF080420023C0E925
:102508000433C0E9072383614FF48073436203F007
:1025180003FD08B1FFF7E8FF044803F029FE18B1EE
:10252800BDE80840FFF7E0BF08BD00BFD4010020A8
:102538000028004010B5044690B03822002102A8B7
:102548000EF0B0FA2268194B9A422CD14FF480331E
:10255800029302A84FF480730F9303F057FB08B15E
:10256800FFF7C2FF4FF0B0430220D3F8902042F4A7
:102578000042C3F890209A6D42F480629A659B6D80
:10258800002203F4806311460193019B02F016F9BF
:10259800022002F045F900222A20114602F00EF925
:1025A8002A2002F03DF910B010BD00BF00280040FD
:1025B80008B501F0A9FCBDE8084002F0C7BD01F06C
:1025C800AABC000008B50F4804F020F900F0D6FBBB
:1025D8004FF6FF714FF0904002F004FD0A484FF6A5
:1025E800FF7102F0FFFC09484FF6FF7102F0FAFC98
:1025F80001F08AFC064B0120C3F88800BDE80840BA
:1026080002F026BEAC020020000400480008004882
:102618000004005808B501F07EFCFFF791FEBDE804
:102628000840FFF7E4BC08B501F06EFCBDE80840BF
:102638000121002002F06ABD01F06DBC7047FEE781
:10264800FEE7FEE7FEE7FEE7704770477047704712
:10265800014803F0B3BD00BFD4010020012002F0FF
:1026680041BD0000014802F0B5BA00BF4C0200208D
:10267800014804F087B900BFAC020020014803F00C
:10268800CFBB00BFD4010020014803F0C2BF00BF88
:10269800380200202DE9F04389B080460020109EC2
:1026A8000790894615461F46FDF7BAFDF0B9104C4C
:1026B800CDE90090CDE9020407AB0E480593142339
:1026C80004933A46434629460068FDF773FE2346BD
:1026D800324604F1140153F8044B42F8044B8B4280
:1026E800F9D1079B337509B0BDE8F0830120FAE7FB
:1026F8000C020020CC0C01081FB50E4C00233C2214
:1027080002A8CDE902336275237500F0BBF80423F3
:1027180003AA009412210848FFF7BCFF07491422B6
:1027280020460EF0AFF9B0FA80F35B09637504B088
:1027380010BD00BF20020020F40C01085E05002037
:10274800054808B50823036003F07EFD18B1BDE80D
:102758000840FFF7C9BE08BD380200204FF0B0435B
:1027680007B55A6E42F001025A665B6E002203F00A
:102778000103019311463220019B02F01FF8322019
:1027880003B05DF804EB02F04BB800000CB407B5D9
:10279800054A05AB102101930EF056F803B05DF819
:1027A80004EB02B0704700BF060D010830B585B0D4
:1027B800044602A80D460DF073FEBDF90C30064A1A
:1027C80000931021029B2046FFF7E0FF2046FEF70A
:1027D800F3FD288005B030BD060D01084FF0B0426A
:1027E80010B5936823F4004393600DF0E1FE0F4B9E
:1027F80001241C700DF0ACFB0D480DF0C3FB0D4B14
:102808004FF400421A6100200DF0C2FBFFF77CFB79
:1028180000F0B8F80DF0B8FC214620460DF0D4FCC5
:10282800BDE81040002102200DF0CEBC440200207B
:10283800B5270008004000580DF0DCBC08B5FFF7CC
:102848006BFB40F6B83398420CD8B0F5E16F0BD368
:10285800FE23A0F5E16058434FF49663B0FBF3F014
:10286800C0B208BDFE20FCE70020FAE77FB5684645
:1028780000F06CF80198FFF721F900B207B05DF895
:1028880004FB0000194A38B5D2F88035591C0446B3
:1028980019D101F047FB054601F050FB054401F052
:1028A80047FB2B0EE3712B0CA3712B0A6371030EEC
:1028B800E370C0F30742C0F307232571C0B2A270CA
:1028C8006370207038BD190AC3718171190C1B0E11
:1028D80041710371D2F88435C370D2F88405C0F30E
:1028E8000722C0F30743000EE9E700BF0070FF1F8F
:1028F80038B5094BD3F8803503600133054609D153
:1029080001F010FB044601F013FB444001F016FBF4
:1029180044402C6038BD00BF0070FF1F0121022019
:102928000DF03CBC002102200DF038BC002070479F
:10293800024B187808B100F05DB8704744020020D7
:1029480082B00190019802B000F0F0B810B50446CA
:10295800FFF7FCFA074BA36040F30F20FFF75AF884
:10296800054B064A2360064B6060C4E90323002038
:1029780010BD00BF0000484200007A440D093E0027
:10298800AB03050000207047014B1868704700BF73
:10299800480200200320704708B501464FF47A72B8
:1029A80000238002890DFFF7AFF808BD4FF47A7352
:1029B800A0FB0303800A40EA83507047034B9868E2
:1029C8009A689042FBD1C043704700BF002800407E
:1029D80008B5FFF7F3FF014B186008BD4802002057
:1029E80008B5FFF7EBFF024B1B68C01A08BD00BF14
:1029F80048020020024B187808B1FFF7DFBF704784
:102A08004502002010B5074B074C0122DA654FF448
:102A18008071204603F0CAF94FF0FF33236300208A
:102A280010BD00BF00280040D4010020024600214C
:102A3800014803F0D4BB00BFD401002002460121A5
:102A4800014803F0CCBB00BFD401002010B58CB006
:102A58002C220021044601A80EF024F8FFF7D2FF2B
:102A68000C4B0D481B681C440023089306934FF039
:102A78000053E443079301224FF4807301A90294A1
:102A88000B9303F0A9FA08B1FFF72EFD00200CB054
:102A980010BD00BF48020020D401002038B505460B
:102AA800FFF78CFF02210446074803F09FFBC4F39D
:102AB80009024FF47A71A2FB0121920AA30A2A8023
:102AC80043EA805038BD00BFD401002001480021EE
:102AD80003F08CBBD40100200148012103F086BB20
:102AE800D4010020F8B50F4D2E78CEB90E4C4FF01A
:102AF800FF372763FFF7FAFCFFF784FF4FF4807175
:102B0800204603F053F92046276303F013FB3246AF
:102B18002046022103F063FBFFF75AFF01232B70C5
:102B28000020F8BD45020020D4010020014610B560
:102B38004FF47A7200238002890DFEF7E5FF014603
:102B4800FFF73CFF0446FFF739FF031B8B4200D316
:102B580010BD00BFF7E70DF033BE000010B5064CFE
:102B68000221204603F042FB0221421C2046BDE818
:102B7800104003F034BB00BFD40100201348144AAE
:102B880008B54FF4E133C0E9002300230C22C0E963
:102B98000233C0E90523C0E90733C0E909330361FB
:102BA80004F0D1FC08B1FFF79FFC0848002104F0AD
:102BB80046FE08B1FFF798FC044804F020FE18B15F
:102BC800BDE80840FFF790BC08BD00BFAC0200207C
:102BD8000044004070B596B006461422002103A8B0
:102BE8000DF060FF3822002108A80DF05BFF326865
:102BF8002C4B9A4253D10223089308A82A4B0A93D4
:102C080003F004F808B1FFF76FFC4FF0B04300255C
:102C18009A6D42F400329A659A6D02F4003202927B
:102C2800029ADA6C42F00102DA64DB6C03F0010309
:102C380001930422019B0223CDE9032303240723E4
:102C480003A94FF09040CDE90554079302F01EF90F
:102C5800082303A94FF09040CDE903340595134CA0
:102C680002F014F9124925621423C4E90013102351
:102C7800C4E9023520468023C4E90435C4E9065571
:102C880001F02EFE08B1FFF72FFC2520F467002283
:102C98000221A66201F092FD252001F0C1FD16B0C7
:102CA80070BD00BF0044004004000C004C0200202E
:102CB8008000024002680C4B9A4210B5044612D1BB
:102CC8004FF0B0420C21936D23F4003393654FF01D
:102CD800904002F087F9E06F01F076FEBDE8104001
:102CE800252001F0ABBD10BD0044004008B50A46E0
:102CF8000146024803F0AAFD002008BDAC020020EE
:102D080013B5114B114C18604FF40013009302AB2C
:102D180013E90600204604F016FD2368DA69D1039A
:102D2800FCD4DA695202FCD59A68084842F4800259
:102D38009A6004F04EFD06490448012204F0BCFCE8
:102D4800002002B010BD00BF40030020AC020020EC
:102D58004803002008B5074B1860FFF748F9FFF74C
:102D68000DFF054AD2F8803043F00063C2F8803086
:102D7800002008BD440300200008005808B54FF0A3
:102D8800B04308489A6B42F400329A639A6B22F473
:102D980000329A63FFF78EFF0F2001F04FFD0020ED
:102DA80008BD00BFAC0200200268044B9A4203D160
:102DB800034B00201B681847704700BF00440040C1
:102DC8004403002002680B4B9A4210B504460FD109
:102DD800094B1B682BB1D0F8902012B90748012184
:102DE800984720460549BDE81040012204F064BC1C
:102DF80010BD00BF004400404003002048030020ED
:102E080010B50A4C23780BB9E37C6BB1FFF774FC5F
:102E18000038074B18BF0120400018701B78022BA0
:102E280002BF00232370E37410BD00BF5E050020BD
:102E38005103002038B5114C2378EBB9E37CDBB99A
:102E48000F4D2B68012B07D92B68042B04D80D4A8A
:102E58000421012000F008FA2B68042B0CD9FFF795
:102E68004BFC0038084B18BF0120400018701B7835
:102E7800022B04BF0023237038BD00BF5E0500206D
:102E88004C030020600D010851030020022804D8DB
:102E980002480122102102F01FB9704700040048BF
:102EA800022804D802480022102102F015B9704700
:102EB80000040048022808B50ED80122102107484E
:102EC80002F00AF93220FFF73BFDBDE8084003484D
:102ED8000022102102F000B908BD00BF000400481C
:102EE8007047000010B5012104464FF0904002F0F1
:102EF800EDF8054AB0FA80F35B0913701378A370F4
:102F0800024B01221A7010BD500300205D050020FD
:102F180008B5FFF763FCBDE8084000F045BB4FF07B
:102F2800FF300DF0CBB9704770470000014BD870E7
:102F3800704700BF5C000020014B1874704700BF49
:102F48005C00002020B1037813B102480DF0E6BB05
:102F5800704700BF9404002008B5022000210DF03E
:102F680075F9BDE8084001480DF0D8BBAC04002055
:102F7800002101200DF06AB910B5094C60B120603C
:102F880008480DF07DFB216806480DF001FCBDE8FE
:102F9800104004480DF0C2BB42F210732360EFE703
:102FA80074000020AC04002010B5094C2060236890
:102FB8000BB9084B236008480DF062FB21680648EE
:102FC8000DF0E6FBBDE8104003480DF0A7BB00BFBD
:102FD8000C000020A0860100C404002010B504469F
:102FE80060B190F906304BB907480DF049FB074B23
:102FF800E2791A70064B1868FFF7D6FFBDE8104053
:10300800002102200DF022B9480400207804002095
:103018000C00002038B504460D4607484FF40061FF
:10302800FFF768F930B92A4621460348BDE8384019
:10303800FFF762B838BD00BF00F003080A4601492F
:10304800FFF738B900F0030838B50C480DF018FB45
:1030580005F05AF860B90A4C0A480125257004F0B1
:10306800E5FE2078294604F037FC04480DF056FBAD
:10307800BDE8384004480DF051BB00BFAC04002047
:10308800000000205C0000207C04002005F0D8B877
:1030980030B585B0FFF7D2FB044604F013FD0546B2
:1030A80080B1002434480DF0EBFA344B32481968EB
:1030B800A14238BF21460DF06BFB2F480DF02EFBC7
:1030C80005B030BD01A8FFF70DFF2D4A2D49042397
:1030D800137053680878187053685D705368182126
:1030E800997053680121D970516823B203EB4303E7
:1030F80003EB4313FE24B3FBF4F30B71224B197853
:1031080011B31D70536860F07F00187005231370A9
:103118001E491F4C0978012988BF00235370637A20
:1031280033B104F0BBFC012802D120460DF0A8FA07
:10313800184B1348D978002204F0DAFCA8B9164BCA
:103148001870164B1870ACE7144B1B7813B9124B58
:103158001B7843B153680121597153689DF80610D3
:1031680099710723D4E70523D2E7063099D104F0F3
:103178008FFC044696E700BFAC04002074000020D2
:103188000400002044040020DC0400205103002037
:10319800480400205C0000205D0500207305002025
:1031A80008B5104B0122002102201A700DF04EF8CC
:1031B8000D480DF0B3FA0D4B1B788BB10C4B1A78F8
:1031C80072B9DB7C63B90B4B1A68042A9EBF1A6874
:1031D80001321A600021BDE8084010200DF036B811
:1031E80008BD00BFDC040020C404002078040020CF
:1031F8005E0500204C030020044B1B78022B03D1F2
:10320800002108200DF022B8704700BF0000002000
:1032180008B504F082FF80B904F040FC01280CD105
:10322800BFF34F8F0549064BCA6802F4E0621343A7
:10323800CB60BFF34F8F00BFFDE708BD00ED00E096
:103248000400FA05704770477047704770470128B7
:1032580002D0022804D07047002102200CF0F6BFEB
:1032680000210820FAE7000070B505460C4616460E
:1032780004F028FC0346002834D000241A480DF036
:10328800FFF91A4B18481968A14238BF21460DF0BA
:103298007FFABDE8704014480DF040BA4A68F05C07
:1032A800D0540133DAB29442F8D8114B0D701B7820
:1032B800012B88BF00244C700E4C637A33B104F0A4
:1032C800EDFB012802D120460DF0DAF90A4B0B4834
:1032D800D978002204F00CFC0630CED104F0D8FBDB
:1032E8000446CBE70549DDE7AC0400207400002064
:1032F80051030020480400205C0000200400002046
:10330800044B1B7823B9044A05210120FFF7ACBF01
:10331800704700BF51030020650D010810B5002457
:1033280090B03C22214601A800940DF0BBFB2C4B29
:103338002022DA7219788DF8001059788DF801106A
:1033480099788DF80210D9788DF8031019798DF8CD
:10335800041059798DF8051099798DF80610D979E6
:103368008DF80710197A8DF80810597A8DF8091018
:10337800997A8DF80A108DF80B2021460DF10B0271
:1033880058180131007B02F8010F1C29F8D193F875
:1033980028208DF8282093F829208DF8292093F8E3
:1033A8002A208DF82A2093F82B208DF82B200DF158
:1033B8002B0100229818013290F82C0001F8010F17
:1033C800142AF7D107484FF40061FEF793FF20B99C
:1033D800044840226946FEF78FFE10B010BD00BFBA
:1033E8007800002000F80308014940220CF022BFB1
:1033F80000F8030870B52A4D28796B794D2BC0B2B7
:1034080033D1C0EB001080000A2838BF0A204FF4DF
:103418007A735843234BAC791860EB794D2BE4B29F
:103428002BD1C4EB0414A40095F82C301E4E63BBBA
:1034380095F83F304BBB42F21070FFF79DFD3068A6
:10344800FFF7B2FD2B7A194A1949DBB213706B7A70
:10345800184ADBB213700023EA1892F82C20D2B273
:10346800CA540133142BF7D170BD6B79482B0ABFAE
:103478004FF461636B795843C6E7EB79482B0ABF71
:103488004FF46163EB795C43CEE7FFF775FD012CE0
:1034980038BF01244FF47A735C433460CFE700BF30
:1034A80078000020740000200C0000207205002025
:1034B8005E0500205103002010B590B000213C2289
:1034C80001A800910DF0EEFA4022344968460CF04C
:1034D800B1FE9DF800203AB99DF80100182803D1E3
:1034E8009DF8021001290ED0FFF718FF2C4814226E
:1034F80000210CF0A9FE4FF47A70FFF721FAFFF7CC
:1035080079FF10B010BD274B1A70587099709DF84C
:103518000310D9709DF8041019719DF805105971A0
:103528009DF8061099719DF80710D9719DF808103B
:1035380019729DF8091059729DF80A1099729DF830
:103548000B1001F03F01D972D87AD1B288421BD84A
:103558009DF8282083F828209DF8292083F8292021
:103568009DF82A2083F82A209DF82B2083F82B2009
:103578000DF12B0100229818013211F8014F80F843
:103588002C40142AF7D1BAE701F1400068441944E5
:1035980010F8340C08730132D6E700BF00F80308AE
:1035A8005E050020780000201FB5002403A92046EE
:1035B800039404F095FD03A9012004F091FD354B17
:1035C8003548009422464FF4FA710CF0FBFF334B58
:1035D8003348009422464FF4FA710CF0F3FF314B54
:1035E8003148009401224FF4FA710CF0EBFF2046A9
:1035F800FEF77CFD08B1FEF777FF2C4B0094002204
:103608004FF4FA612A480CF0DDFF2A4A0021012014
:103618000CF0D8FE284A002102200CF0D3FE274ADD
:10362800002104200CF0CEFE254A002108200CF0D1
:10363800C9FE00F039FB2349234804F007FD23485D
:1036480004F0F4FB18480DF069F8214B00211878B4
:1036580004F042F91F4900941F4B09681F480022D3
:103668000CF0B0FF1D480DF059F8FFF725FF1C4A74
:10367800002110200CF0A6FE1A4B1B4819681B4BA2
:10368800009400220CF09EFF17480DF047F804B094
:1036980010BD00BF513200089404002053320008C6
:1036A800600400204D320008480400200132000860
:1036B8007C0400202D7C0008993000089530000813
:1036C8005130000800000301100000205C000020B9
:1036D8000000002074000020612F0008AC040020C6
:1036E8003D2E00080C000020C4040020A931000869
:1036F80030B5A1B000217C2201A800910DF0D2F9CB
:1037080053238DF8003001254FF48C73ADF8023047
:103718008DF80450FFF792F80D4CFE23B0FBF3F040
:1037280000EB400000EB40108DF805002C228021B2
:10373800201D0DF0B7F90098BDF80430206022462E
:1037480006212846A380FFF78FFD21B030BD00BFBA
:10375800DD04002070B50378592B90B0044640F082
:10376800BE81052959D84378443B162B55D8DFE844
:1037780013F00F015400FF005400070154005400D7
:103788005400540073005400EA00540054005400DC
:103798007501540054008F00540054005400170061
:1037A8008578482D11D1A54A14210120FFF75CFD29
:1037B80041F28830FFF7C4F840F6B830FFF7C0F898
:1037C80010B0BDE87040FFF723BD532D0ED1302255
:1037D80080219B480DF066F9FFF78AFF41F2883097
:1037E800FFF7AEF8964A1521012064E0432D16D163
:1037F800002468468DF8004004F090FA904A4C2363
:103808001370182393709DF80030547001204133D1
:10381800D07013710521FFF727FD10B070BD442D3E
:10382800FBD1874C2C228021201D0DF03BF9002371
:103838002570637001251823A370E5702571FEF7C4
:10384800FDFFFE23B0FBF3F000EB400000EB40105F
:10385800607122460621C7E78378303BDBB2092B2B
:10386800DBD87849784A0B700B78DBB25372744A0C
:10387800592313704D2353700B7830339370032101
:103888000120FFF7F1FC10B0BDE87040FFF746BD1E
:103898008578482D14D16A4A562313700023537033
:1038A800032318210120137193710423917051711E
:1038B800D070D371082110B0BDE87040FFF7D4BCB8
:1038C800432DAAD15E4C00213C2201A800910DF0A5
:1038D800E9F86846FFF788FD2422802104F10C00EE
:1038E8000DF0E0F89DF8003063709DF80130A3708A
:1038F8009DF80230E3709DF8033023719DF8043081
:1039080063719DF80530A3719DF80630E3719DF849
:10391800073023729DF80830257063729DF80B50AC
:103928009DF80930A3729DF80A30E3722A4603A96C
:10393800257304F10D000DF0E6F805F10D0122469E
:10394800C9B2012067E7807839280CD83038C0B26E
:10395800FFF79CFA3A4A2378137063785370A37878
:103968009370032140E710B0BDE87040FFF7C8BC72
:1039780080783928F7D83038C0B2FFF791FAE9E7EC
:1039880080783928EFD83038C0B2FFF793FAE1E7EA
:103998008378303BDAB2092AE5D8C0783038C2B229
:1039A800092AE0D82179A1F14802D2B20B2ADAD843
:1039B800264D45FA02F2D207D5D40A224D2902FB38
:1039C800030036D13C2358434FF47A735843204BB5
:1039D8001860204B1860FFF7CFFA194A2378137044
:1039E80063785370A3789370E378D3702379137155
:1039F80005210120FFF738FC134B00221A7018220A
:103A08005A7001229A70DA70A278303A02EB820179
:103A1800E278303A02EB4102D2B21A7122795A7135
:103A28000D4A1278D2B21A72064A1278D2B25A7273
:103A380029E74829C8D14FF46163C4E76B0D010831
:103A4800DD0400205103002078000020DEF7FFFF8E
:103A5800740000200C000020720500208678A6F172
:103A68003003092B3FF67FAFC078A0F13003092B54
:103A78003FF679AF2179A1F14802D2B20B2A3FF67D
:103A880072AF5A4B134113F001057FF46CAF584ADB
:103A98005923137053235370D070117196700521F8
:103AA8000120FFF7E1FB534918230D704B700123E8
:103AB8008B70CB70A378303B03EB8302E378303B09
:103AC80003EB4203DBB28B712379CB714A4B1B7832
:103AD800DBB20B72494B1B78DBB24B72D3E6502B2F
:103AE80048D102297FF699AE4378303B012B3FF647
:103AF80094AE8378312B7FF490AE0B2904D8FFF76E
:103B0800FFFB00213A4A6FE63A4D0234002214F8CE
:103B1800013FA918303B0132DBB20C2A0B73F6D1F6
:103B2800FFF7DEF9324B502218211A7099700022E3
:103B380001215A70D97003F8041FA9180132097BB2
:103B48000C2A01F1300103F8011FF6D100232B7074
:103B580018236B700123AB70EB70274B1B78DBB21B
:103B68002B72264B1B78DBB26B72EA72FFF7D6FB1F
:103B78001121C7E7412B7FF450AE4378432B7FF4E4
:103B88004CAE16297FF449AE1D4D421C002312F895
:103B9800011FE9540133142BF9D1FFF731F9194BFF
:103BA8005B7D012B19D113490023EA5CC818013346
:103BB800D2B2142B80F82C20F7D1104B00221A70A7
:103BC8001B78DBB24B72FFF7A9FB094A631E153459
:103BD800A34206D1064A162106E6084B02221A70AD
:103BE800F3E713F8011F02F8011BF1E7DEF7FFFF07
:103BF800DD04002078000020720500205103002019
:103C08005E0500202002002037B504460D46002935
:103C180039D022480CF082FD2B78A3B39CB360689E
:103C2800237880B3032B0DD0042B2ED0022B2AD15E
:103C38006178012927D00B0625D403B0BDE83040B0
:103C4800FFF788BD6378012B07D10078012802D0DF
:103C5800022800D008B904F017F800240DF1070075
:103C68008DF8074004F05AF80D4A4C2313701823B6
:103C780093709DF80730547001204133D070137150
:103C88000521FFF7F1FA03B030BD6378012BFAD1B3
:103C98000378044A03F001031370F4E7600400207A
:103CA800DD04002044040020034B0022C3E9022263
:103CB8000122C3E9002270477405002000487047BC
:103CC800740500204FF0B04382B0DA6C0243DA6426
:103CD800DB6C03400193019B02B070472DE9F04172
:103CE80086B000240220154D0594FFF7EBFF042051
:103CF800FFF7E8FF124F03944FF4807601230DEB92
:103D08000001CDE901632846032304934FF40058CA
:103D180001F0BCF801A93846CDF8048001F0B6F8E6
:103D280022464146384601F0D7F928462246314610
:103D380001F0D2F9204606B0BDE8F0810004004841
:103D480000080048032810B50ED8012810D868B913
:103D580002460B484FF4807101F0BEF90022094871
:103D68004FF4005101F0B8F9002010BD0122F0E72E
:103D7800002203484FF4807101F0AEF90122EEE70A
:103D880000040048000800480220704700207047DF
:103D98000120704700280CBF0F2016207047000034
:103DA8000D48854600F098F80C480D490D4A002347
:103DB80002E0D458C4500433C4188C42F9D30A4AD8
:103DC8000A4C002301E013600432A242FBD30CF03A
:103DD80071FEFEF755FBFEE7000001200000002001
:103DE8004C010020A01801084C01002028230020C5
:103DF800FEE74FF0B04382B0DA6C0243DA64DB6C62
:103E080003400193019B02B07047000030B587B0B2
:103E180004460D461022002102A80CF043FE012C96
:103E280015D80120FFF7E5FF1C4B33F81430019338
:103E380001220223CDE90323194B53F8240055B975
:103E480001A9029501F022F8002007B030BD022C2C
:103E5800EAD10420E6E74FF4041301A9114D0293B7
:103E680001F014F8104B05EBC40553F8241028464C
:103E780000F00DFF0D4B002153F82420284600F0D8
:103E8800FFFE0B4B1D570B4B284653F824100022FE
:103E980000F094FC284600F0C3FCD5E7840D010827
:103EA8008C0D010884050020A40D0108980D010857
:103EB800800D0108B00D0108704708B50220FFF712
:103EC800FBFF08BD08B50120FFF7F6FF08BD08B5E0
:103ED8000020FFF7F1FF08BD7047000010B5032070
:103EE80000F05AFC01F0C4FA064B18600F20FEF7E8
:103EF8001DFD044618B9FEF7A1FB204610BD01249C
:103F0800FBE700BFB80000204FF0E022136923F060
:103F18000203136170474FF0E022136943F0020374
:103F280013617047014BD3F8900570470070FF1F6D
:103F3800014BD3F8940570470070FF1F014BD3F86D
:103F4800980570470070FF1F8068C0F380007047B5
:103F5800F7B5002301930446002800F0E980856D39
:103F680025B9FDF77BFFE56584F8545023689A6806
:103F7800D00040F1A1809A68D10000F1B480A26D10
:103F880042F01002A265E26D42F00102E2650125ED
:103F98001846FFF7D9FFA26D02F01002024340F065
:103FA800C980A26D206922F4817242F00202A265E2
:103FB8009A68D2075DD4226BA67E94F82CC0003A8A
:103FC80018BF01221703D4E902120A43217E42EAEC
:103FD8008132617E42EAC13242EA4632002842EA30
:103FE8004C02B4BF20F000414FF400113A430A4399
:103FF80094F82010012903D1002E76D142F48032A2
:10400800616A21B1A66A01F4E07131430A43D968B3
:10401800E66C21F4FE3121F4FF711143D96094F864
:104028003C206168012A01F0404C4CEA060609D19F
:10403800D4E910273A433243A66C324342EA0C02D1
:1040480042F001061F693E4A3A4032431A6121F0A4
:104058000042B2F1804F0CD0B1F1004F09D0394E77
:10406800D6F8082701F4701122F470120A43C6F832
:1040780008275A69666BA16B22F0070232435A611E
:104088005A6922F0700242EA01125A61002835D1B9
:104098009A6A62F00F029A625B6903F007039E4214
:1040A8003CD10023E365A36D23F0030343F0010330
:1040B800A365284603B0F0BD9A68234922F0104250
:1040C80022F0170242F080529A60204A1268B2FB2E
:1040D800F1F2013252000192019A002A3FF44BAFEB
:1040E800019A013AF7E7002552E7A16D41F0200156
:1040F800A165E16D41F00101E16581E7B0F5001FBF
:10410800CAD19A6AE269013A92006FF00F0102F08F
:104118001C0201FA02F2216E0A43BCE7A36D23F0E8
:10412800120343F01003A365E36D43F00103E36555
:104138000125BEE7A36D43F01003A365F8E700BFB0
:1041480002FCFF1F00200140400D0300B8000020C2
:10415800F8B54569082D04460E460AD00368DB68A1
:10416800D80705D5A36D43F02003A3650120F8BD4A
:104178000425FEF7DDFB074623681A682A4221D08A
:10418800A26D42F40072A265DA6812F4406F14D18D
:10419800A27E92B91A6812070FD51846FFF7D4FE07
:1041A80028BB5A6822F00C025A60A26D22F4807271
:1041B80022F0010242F00102A265207E00BB0C221F
:1041C8001A60D4E7711CD8D0FEF7B2FBC01BB0420E
:1041D80001D8002ED0D123681B682B40CCD1A26D0A
:1041E80084F8543042F00402A2650320BFE7A26DB0
:1041F80042F02002A265E26D42F00102E265DCE7CE
:104208000020B4E70368186C70470000F7B5002376
:10421800019390F85430012B044600F0C5800568DE
:104228000669012380F854302846FFF78DFE0028E0
:1042380040F0B480D1E90020022826F0040300F001
:104248008280B3F1004FC2F3110E13D1AB6A43EA77
:104258000E03AB628B68686903EA022323F07C4390
:1042680023F0FF0320EA02210B43002A6B6126DBBF
:10427800002055E0236E00F01F074FF00F0C0CFADA
:1042880007FC6FEA0C0623EA0C0CBEF1000F11D1F3
:10429800C2F38463BB4043EA0C0323668008E369E6
:1042A80001309842D6D8A86AC2F38363BB4006405F
:1042B8003343CEE792FAA2F3B3FA83F3EAE73B4932
:1042C8003B48D1F80837824203F0E07519D11B0248
:1042D800CED4D1F8083723F0E0732B4343F400031E
:1042E800C1F80837334B1A68334BB2FBF3F20C238F
:1042F80002FB03330193019B002BB9D0019B013BC7
:10430800F8E72E48824210D113F08070B0D1D1F86E
:10431800083723F0E0732B4343F08073C1F8083764
:10432800002384F8543003B0F0BD254882429FD161
:1043380013F480009CD1D1F8083723F0E0732B43A5
:1043480043F48003EAE7B3F1004F01BFAB6AC2F35D
:1043580011018B43AB62002A8ADA1548134982425D
:10436800D1F8083709D1D1F8082703F0A07322F053
:10437800E0721343C1F808377AE71048824204D143
:10438800D1F8082703F44003F1E70D4882427FF48F
:104398006FAFD1F8082703F0C073E8E7A26D42F0C9
:1043A8002002A2651846BBE70220BCE700200140B6
:1043B800001000B0B8000020400D0300004000B815
:1043C800002000B4026838B504461046FFF7BCFD6B
:1043D80008B9002038BD9368990707D4936823F07B
:1043E800004323F0170343F010039360FEF7A0FA8D
:1043F800054623689B685B07EBD5FEF799FA401BD7
:104408000228F6D923689B685A07F2D5A36D43F0B2
:104418001003A365E36D43F00103E3650120D9E7C9
:1044280073B50023026801939368DD07044602D53B
:10443800002002B070BD9168214B194209D0A36DCC
:1044480043F01003A365E36D43F00103E365012026
:10445800EFE7936823F0004323F0170343F00103C9
:104468009360184BD3F8083718021CD4637E012BCD
:10447800DED0FEF75DFA144E054622681368DB07A6
:10448800D6D49368D9075FBF9368334043F00103DC
:104498009360FEF74DFA401B0228EED923681B688B
:1044A800DA07EAD4CBE7094B094A1B68B3FBF2F3F6
:1044B80001330193019B002BD8D0019B013BF8E706
:1044C8001700008000200140E8FFFF7FB8000020AF
:1044D800400D030038B504460068FFF735FD054672
:1044E80020BB94F85430012B20D0012384F8543099
:1044F8002046FFF795FFB0B9A36D226823F47063D7
:1045080023F0010343F48073A3651C23E065136063
:1045180084F85400936823F0004323F0170343F012
:104528000403936038BD84F85450FBE70220F9E790
:10453800026838B5936891680446C80701D400201A
:1045480038BD9907FBD4936803F00503012B19D1F3
:10455800936823F0004323F0170343F002039360AA
:1045680003231360FEF7E4F9054623689B68DB071D
:10457800E5D5FEF7DDF9401B0228F6D923689B68CC
:10458800DA07F2D5A36D43F01003A365E36D43F09A
:104598000103E3650120D3E770B5044600284BD03A
:1045A800836D43F002038365FFF70CFF054668B986
:1045B8002046FFF7BDFF054608B90123A365226819
:1045C800936823F0104323F01703936023685A6815
:1045D80022F4677222F003025A6040F29F321A6096
:1045E800D968164A0A40DA601A6922F040421A610C
:1045F8005A6922F007025A611A6A02F0F0221A6216
:104608005A6A02F0F0225A62DA6A02F0F022DA629A
:104618009A6A0B4A00269E62D2F8083723F0FE7386
:10462800C2F808372046FDF72DFCE6652666A66524
:1046380084F85460284670BD0125FBE700023E83DC
:104648000020014010B590F85430012B044615D0D5
:10465800012380F85430FFF7B5FE58B92046FFF71C
:1046680067FF38B9A36D23F4807323F0010343F087
:104678000103A365002384F8543010BD0220FCE731
:10468800F7B50023019390F85430012B04467FD0EE
:10469800012380F85430FFF74BFF23689A6812F023
:1046A8000102054607D0A36D43F01003A36500235C
:1046B80084F854302DE0A16D364F21F4817141F01A
:1046C8000201A165DE68D96826F4FF4626F07C065B
:1046D80021F40041360421F00301360CD96008208A
:1046E8009968394041F0004199609968002913DAC6
:1046F8000199013101910199B1F52E3FF5D3A36DCF
:1047080023F0120343F01003A365002384F8543008
:104718000125284603B0F0BDD3F8B410013801F0E4
:104728007F010A44DCD199681A48014041F001012F
:104738009960D3F8B41021F07F0141EAD202C3F89E
:10474800B4209A68024042F002029A60FEF7F0F83C
:10475800074623689A68D20708D4DA683243DA60D1
:10476800A36D23F0030343F001039FE7FEF7E0F88E
:10477800C01B0228EDD923689B68D907E9D5A36D2A
:1047880043F01003A365E36D43F00103E365BFE75E
:104798000225BEE7E8FFFF7F0749CA6822F4E06206
:1047A8000302120403F4E063120C134343F0BF63E3
:1047B80043F40033CB60704700ED00E0164B30B592
:1047C800DC68C4F30224C4F10703251D042B28BFA9
:1047D8000423062D4FF0FF358CBF033C002405FA57
:1047E80003F321EA0303A54022EA0502A3400028B7
:1047F80043EA0203ACBF00F16040084A4FEA0313E2
:10480800B8BF00F00F00DBB2AABF00F56140135437
:1048180080F8003330BD00BF00ED00E014ED00E08B
:10482800002807DB044A4109012300F01F008340E8
:1048380042F82130704700BF00E100E000280CDB9F
:104848004309064900F01F0020330122824041F845
:104858002320BFF34F8FBFF36F8F704700E100E055
:1048680070B5D0E913456560446D14B1D0E91645BB
:104878006560D0E9105404F01C060124B4406C6053
:10488800046863608368102B0BBFA260A160E160BD
:10489800E26070BD0268416CD3B210B5083B1424C5
:1048A800B3FBF4F30B4CA24288BF0B4A21F003017F
:1048B80099BF01F1804202F502325218073382642F
:1048C800064AC26403F01F03012202FA03F30365D8
:1048D80010BD00BF070402401C08024080080240C7
:1048E80038B500285ED002682F4B9A424FF0140169
:1048F8004CD82E4B1344B3FBF1F32D499B00C0E970
:104908001013022380F825301368056923F4FF4348
:1049180023F070031360D0E9024323432B43456916
:1049280011682B4385692B43C5692B43056A2B43C3
:104938000B431360FFF7AEFFB4F5804F04BF0023AD
:1049480043604268816C02F07F030B60D0E9131466
:10495800013A032A4C6020D8164A174981651A443F
:10496800013B9200012103F0030301FA03F3002144
:104978004265C3651160114A536400230122C36371
:1049880080F8243080F82520184638BD0C4B134495
:10499800B3FBF1F30B499B00B1E70023C0E91533E2
:1049A800C365EAE70120F0E707040240F8FFFDBF0E
:1049B800000002403F820010400902400009024006
:1049C800F8FBFDBF0004024038B5002841D002685A
:1049D800136823F0010313601F4B9A424FF0140130
:1049E80030D81E4B1344B3FBF1F31D499B00C0E9BB
:1049F8001013012403F01C0304FA03F300251560C7
:104A08004B60FFF747FF836C41681D60D0E91332A4
:104A18005A604A1E032A06D8124B0B449B00944046
:104A28001D60114B5C640023C363C0E91533C0E902
:104A38000B33C0E90D33C36580F8253080F8243086
:104A4800184638BD094B1344B3FBF1F308499B00E2
:104A5800CDE70120F5E700BF07040240F8FFFDBFDE
:104A6800000002403F82001000090240F8FBFDBF31
:104A78000004024070B590F82450012D04463BD044
:104A880090F825600125AE4280F824504FF00006CA
:104A98002CD1022580F825500568C6632E6826F0BB
:104AA80001062E60FFF7DCFE036BBBB12B6843F0F9
:104AB8000E032B60A36C1A68D20342BF1A6842F433
:104AC80080721A60636D1BB11A6842F480721A60B2
:104AD8002B6843F001032B60002070BD2B6823F086
:104AE80004032B602B6843F00A03E2E78023C363C7
:104AF80080F824602846F0E70220EEE7034640B13C
:104B080090F82520022A06D00422C263002280F8E9
:104B18002420012070470268806C116821F00E0182
:104B28001160016821F480710160116821F00101B0
:104B38001160D3E9100202F01C0101228A40426090
:104B4800D3E9132151605A6D32B1116821F4807193
:104B58001160D3E9162151600122002083F8252035
:104B680083F82400704710B590F82530022B03D045
:104B78000423C363012010BD03681A6822F00E02E3
:104B88001A601A6822F001021A60826C136823F412
:104B980080731360D0E9101303F01C0201239340C3
:104BA8004B60D0E913325A60436D33B11A6822F46E
:104BB80080721A60D0E916325A60012380F82530D5
:104BC800836B002480F8244013B198472046D2E72D
:104BD8001846D0E770B4426C046C036826681D68F8
:104BE80002F01C020421914031420FD015F0040F4D
:104BF8000CD01A6892065EBF1A6822F004021A6086
:104C0800036B6160002B33D070BC184702219140C0
:104C1800314217D015F0020F14D01A68940606D442
:104C28001A6822F00A021A60012280F82520114A27
:104C380093428CBF104B114B5960002380F82430ED
:104C4800C36ADFE708219140314211D029070FD507
:104C5800196821F00E011960012303FA02F262605B
:104C6800C36380F82530002380F82430436BC9E7FC
:104C780070BC7047800002400004024000000240FF
:104C88000346084609B95A6070470120704710B1B9
:104C98000160002070470120704700000A4A5369EC
:104CA80043F4802330B55361EFF3108472B60023C8
:104CB800CD58C5500433B3F5807FF9D11369DB03B0
:104CC800FCD484F3108830BD00400058064B5A6964
:104CD800002ABFBF054A9A6002F188329A60BABFBB
:104CE8005869C00F002070470040005823016745ED
:104CF800044B5A6942F000425A615869C043C00FD8
:104D0800704700BF0040005870B50546FDF710FE1B
:104D1800124E04463369D90313D43369DA0744BF02
:104D2800012232614CF2FA32134011D10B4E306934
:104D380010F480200BD0FDF7FBFD001BA842F6D332
:104D480004E0FDF7F5FD001BA842E3D3032070BD86
:104D5800024A1361024A01205360F8E700400058F4
:104D68009C0500202DE9F041184D98462B78012B21
:104D780006460C46174626D001232B704FF47A704E
:104D880000236B60FFF7C0FFA0B9012E16D1104AAF
:104D9800536943F0010353612760BFF36F8FC4F871
:104DA80004804FF47A70FFF7AFFF094A536923EA8A
:104DB8000603536100232B70BDE8F0813946204675
:104DC800FFF76CFFEDE70220F6E700BF9C05002027
:104DD80000400058054A536923F47E7343EAC00033
:104DE80040F4803040F002005061704700400058A5
:104DF8002DE9F041234F3B78012B054688463FD0EB
:104E080001233B704FF47A7000237B60FFF77CFF2F
:104E1800044688B92B68042B13D11B4A536943F401
:104E2800803343F0040353614FF47A70FFF76CFF4B
:104E38000446154B1A681B6800233B702046BDE8E2
:104E4800F0814FF0FF33C8F800306E68D5E90132C1
:104E58001344B3420AD93046FFF7BCFF4FF47A70C7
:104E6800FFF752FF50B1C8F800600446064A53697C
:104E780023F47E7323F002035361DAE70136E5E792
:104E88000224DBE79C050020004000582DE9F04F84
:104E9800524C00234FF00F090A6832FA03F501D18A
:104EA800BDE8F08F012505FA03F818EA020200F0C0
:104EB8008E804E68032706F003054FEA430E07FA73
:104EC8000EFC6F1E012F6FEA0C0C32D8876807EAB8
:104ED8000C0ACF6807FA0EF747EA0A07876047689F
:104EE80027EA0808C6F300179F4047EA0807476003
:104EF800C76807EA0C088F6807FA0EF747EA080739
:104F0800022DC76017D14FEAD30800EB880803F0D9
:104F1800070AD8F820704FEA8A0A09FA0AFB27EA32
:104F28000B0B0F6907FA0AF747EA0B07C8F8207056
:104F380001E0032DDCD1076805FA0EF507EA0C0736
:104F48003D4316F4403F056041D023F0030707F1C5
:104F5800804707F5803703F0030CBD684FEA8C0CD7
:104F68004FF0070E0EFA0CFEB0F1904F25EA0E0E28
:104F78002FD01B4DA8422ED005F58065A8420CBF46
:104F88000225072505FA0CF545EA0E05BD602568DA
:104F9800D74316F4801F0CBF3D4015432560656854
:104FA80016F4001F0CBF3D4015436560D4F88050CF
:104FB80016F4803F0CBF3D401543C4F88050D4F828
:104FC8008450B60354BF3D401543C4F884500133A0
:104FD80062E70025D6E70125D4E700BF000800589E
:104FE80000040048374A2DE9F04F00234FF0010A2A
:104FF8004FF0070B4FF00F0931FA03F401D1BDE868
:10500800F08F0AFA03FC1CEA010654D023F00304CB
:1050180004F1804404F5803403F00307A568BF0059
:105028000BFA07F8B0F1904F08EA050E45D0264D67
:10503800A84244D005F58065A8420CBF0225072583
:10504800BD40754517D1D2F8805025EA0605C2F84B
:105058008050D2F8845025EA0605C2F884501568B5
:1050680025EA06051560556825EA06055560A56810
:1050780025EA0805A560056803265C0006FA04F41D
:1050880023FA06F6254300EB8606056003F00705BC
:10509800376AAD0009FA05F527EA0507376285681A
:1050A80025EA04058560456825EA0C054560C5685C
:1050B80025EA0404C46001339EE70025C0E7012502
:1050C800BEE700BF00080058000400480369194201
:1050D80014BF0120002070470AB1816170478162C6
:1050E80070470000044AD168014208B502D0D06078
:1050F800FEF7ADF808BD00BF00080058024A136863
:1051080043F4807313607047000400580D4B10B5CA
:105118005B690C4628B99A0507D500F079F820B1E3
:1051280010BD9B0501D400F06BF8074A1369012CE8
:1051380023F00403136101D130BFF1E740BF20BF62
:1051480020BFEDE70004005800ED00E0064A1368B0
:1051580023F0070343F003031360044A136943F081
:105168000403136130BF70470004005800ED00E0ED
:10517800024B186800F4C060704700BF0004005874
:10518800072830D8DFE800F0040E172F2F2F2F2420
:10519800164B1A6A0A431A625A6A22EA01025A62CA
:1051A80000207047114B9A6A0A439A62DA6A22EA27
:1051B8000102DA62F4E70D4B21F4FC511A6B090481
:1051C800090C0A431A635A6B22EA01015963E7E79B
:1051D800064B9A6D01F008010A439A65DA6D22EAD6
:1051E8000102DA65DCE70120704700BF00040058BF
:1051F800024A936843F48063936070470004005840
:10520800024A136843F4804313607047000400584F
:105218000C4A136823F4804313600B4B1B6832213C
:105228004B430A49B3FBF1F35169890500D533B9FA
:10523800536913F4007F14BF032000207047013B1B
:10524800F2E700BF00040058B800002040420F00F9
:105258000B4A136823F0070343F002031360094B5A
:105268001A69012842F004021A6105D130BF1A698F
:1052780022F004021A61704740BF20BF20BFF6E742
:105288000004005800ED00E04FF0B0431868C0F388
:10529800404070474FF0B0431868C0F34000704773
:1052A8004FF0B042536823F47F4343EA002353602E
:1052B80070474FF0B0431868C0F340607047000073
:1052C8007FB54FF0B0432C4AD3F80831C0F3031030
:1052D80003F00F0352F82040284A52F82330B4FB59
:1052E800F3F4FFF745FF264B054693E80700B5F5AD
:1052F800007F04AB03E9070010D0224B9C4218D36F
:1053080003F5B70303F67F539C4229D903F57413B9
:1053180003F510639C4225D802230BE01A4B9C42EC
:1053280007D91A4B9C421BD903F5370303F5D85309
:10533800F0E7002304AA02EB830353F80C4C144D46
:105348002B6823F0070323432B60FDF7F1FA064689
:105358002B6803F007039C4206D1002004B070BDFF
:105368000123E7E70024EAE7FDF7E2FA801B0228B9
:10537800EED90320F2E700BF1C0E0108BC0D01089E
:10538800500C0108C0CF6A00BFEA21013F933402E4
:10539800004000584FF0B04310B59A68D96812F031
:1053A8000C0205D00C2A4AD101F00303012B50D17D
:1053B8004FF0B0412B480B6813F0080306D00B6878
:1053C80013F0080337D1D1F8941007E00C682407CC
:1053D80056BFD1F894300968C3F3032350F823303B
:1053E800002A0CBF184600204FF0B0418A6802F02E
:1053F8000C020C2A1ED1CA6802F00302022A2ED01F
:10540800032A06D10B68184A13F4801F174B18BFDC
:1054180013464FF0B042D068D168D268C0F3062076
:105428005843C1F302130133B0FBF3F0530F0133B8
:10543800B0FBF3F010BD0B68C3F30313CEE7042AE7
:105448000AD0082A05D11B6813F4801304D1074831
:10545800CAE700231846C7E703480023C4E7024BFE
:10546800D7E700BF1C0E01080024F4000048E8013B
:1054780008B5FFF78FFF4FF0B043044A9B68C3F3AA
:10548800031352F82330B0FBF3F008BDBC0D01083C
:105498002DE9F0410446002853D04FF0B0439D68F1
:1054A800DE6803689B0605F00C0506F0030668D560
:1054B800026A1DB10C2D46D1012E44D1002A40D0DC
:1054C8004FF0B043A16A1A68170756BFD3F8943053
:1054D8001B681B0903F0F00399421FD90846FFF720
:1054E800EFFE00282DD14FF0B042136843F00803B7
:1054F80013601368A16A23F0F0030B431360606A1A
:10550800FFF7CEFEFFF7B4FFAB4B1860AB4B186844
:10551800FDF70CFA002834D0BDE8F0814FF0B04216
:10552800136843F008031360136823F0F0030B4378
:105538001360606AFFF7B4FE0846FFF7C1FE002853
:10554800E0D00120E8E74FF0B043002A54D01A68B1
:1055580042F001021A60FDF7EBF90746FFF79AFEE1
:10556800002842D04FF0B042136843F0080313609C
:105578001368A16A23F0F0030B431360606AFFF716
:105588008FFE2368D80748D42368990700F18C80D8
:1055980023681E0740F1FA80A3694FF0B046002B3C
:1055A80000F0E180D6F89430E16903F010029142EE
:1055B80000F0C48003F00302022AC2D0D80740F1E9
:1055C800B380D6F8943023F00103C6F89430FDF781
:1055D800AFF90746D6F89430990740F1A580FDF752
:1055E800A7F9C31B112BF5D904E0FDF7A1F9C01BDE
:1055F8000228B3D903208FE71A6822F001021A6043
:10560800FDF796F90746FFF745FE0028B9D0FDF7E4
:105618008FF9C01B0228F6D9ECE7082D03D00C2D12
:1056280005D1032E03D16368002BADD189E74FF074
:10563800B043A1681A6822F480120A431A606268AB
:10564800B2F5803F10D11A6842F480321A60FDF733
:105658006FF90746FFF718FE002895D1FDF768F99E
:10566800C01B6428F6D9C5E7B2F5041F04D11A682F
:1056780042F400121A60E6E7196821F480311960D3
:10568800196821F400111960002AE0D1FDF750F9DA
:105698000746FFF7F9FD00283FF476AFFDF748F914
:1056A800C01B6428F5D9A5E7042D236903D00C2D68
:1056B8000ED1022E0CD1002B3FF443AF4FF0B04275
:1056C8006169536823F0FE4343EA016353605FE76F
:1056D8004FF0B046BBB1336843F480733360FDF7D5
:1056E80027F9074633685A0507D57368626923F0B6
:1056F800FE4343EA026373604AE7FDF719F9C31BE7
:10570800022BEFD976E7336823F480733360FDF713
:105718000FF9074633685B057FF53AAFFDF708F9DF
:10572800C31B022BF6D965E74FF0B042E169D2F806
:10573800943023F010030B43C2F894304FF0B04775
:10574800D7F8943043F00103C7F89430FDF7F0F828
:105758000646D7F894309A0718D4FDF7E9F8831B62
:10576800112BF6D946E7D6F8943023F00103C6F892
:105778009430FDF7DDF80746D6F894309B0705D539
:10578800FDF7D6F8C31B112BF6D933E72368580762
:1057980054D50B4F3B68D90514D4FFF7AFFCFDF780
:1057A800C7F806463B68DA050CD4FDF7C1F8831B39
:1057B800022BF7D91EE700BFB8000020BC0000206C
:1057C80000040058E3684FF0B046002B58D023F08F
:1057D8008003052B02BFD6F8903043F00403C6F8C7
:1057E80090304FF0B046FDF7A3F8D6F8903043F06C
:1057F80001030746C6F8903041F28838D6F8903051
:105808009B0705D4FDF794F8C31B4345F6D9F1E689
:10581800E36823F00403812B1BD1FDF789F8D6F840
:10582800903043F08003C6F8903007464FF0B046FA
:1058380041F28838D6F89030180504D5E06A002877
:105848004AD1002068E6FDF773F8C01B4045F1D93E
:10585800D0E6FDF76DF8D6F8903023F08003C6F84F
:10586800903007464FF0B04641F28838D6F890306D
:105878001905E3D5FDF75CF8C01B4045F6D9B9E634
:10588800FDF756F8D6F8903023F080030746C6F89F
:10589800903041F28838D6F890301A0516D4FDF7C2
:1058A80047F8D6F8903023F00103C6F89030074641
:1058B8004FF0B04841F28836D8F890309B07BDD5F4
:1058C800FDF736F8C31BB342F6D993E6FDF730F877
:1058D800C01B4045DFD98DE60C2D4ED04FF0B043AC
:1058E80002281A6822F080721A6033D1FDF720F876
:1058F8000546FFF7DEFC38BBD4E90C314FF0B04267
:105908000B43D0682D4901400B43E16B0B43216CDD
:105918000B43616C0B43A16B43EA0123D36013680B
:1059280043F080731360D36843F08053D360FCF76F
:10593800FFFF0446FFF7BDFC002882D1FCF7F8FF03
:10594800001B0A28F6D955E6FCF7F2FF401B0A2887
:10595800CFD94FE6FCF7ECFF0446FFF7AAFC30B9B5
:105968004FF0B042164BD1680B40D360D4E5FCF73A
:10597800DFFF001B0A28F0D93CE601283FF4CCAD34
:105988004FF0B043226BDB6803F0030191427FF4D0
:10599800D8AD616B03F070028A427FF4D2ADA16B7F
:1059A80003F4FE42B2EB012F7FF4CBAD626C03F03F
:1059B800604393423FF445AFC3E500BF8C80C111FB
:1059C800FCFFFEEE2DE9F0410D46044610B901201A
:1059D800BDE8F081684E336803F007038B4216D3A5
:1059E80023689A0727D54FF0B047A268BB6823F011
:1059F800F0031343BB60FCF79BFF0646BB68DB0361
:105A080019D4FCF795FF831B022BF7D911E03368F3
:105A180023F007030B433360FCF78AFF074633681C
:105A280003F00703AB42DBD0FCF782FFC01B022860
:105A3800F5D90320CCE72368580617D54FF0B047AF
:105A48006269D7F8083123F00F0343EA1213C7F845
:105A58000831FCF76DFF0646D7F80831D90305D49D
:105A6800FCF766FF831B022BF6D9E2E723685A0787
:105A780013D54FF0B047E268BB6823F4E0631343E3
:105A8800BB60FCF755FF0646BB689B0305D4FCF7D3
:105A98004FFF831B022BF7D9CBE72368180714D5D0
:105AA8004FF0B0472269BB6823F4605343EAC2034E
:105AB800BB60FCF73DFF0646BB68590305D4FCF7FD
:105AC80037FF831B022BF7D9B3E72368DA070FD414
:105AD800294C236803F00703AB4239D8FFF7C8FC09
:105AE800264B1860264BBDE8F0411868FCF71EBF2E
:105AF8006268022A1DD1FFF7C7FB00283FF467AF91
:105B08004FF0B04641F28838B36823F003031343DB
:105B1800B360FCF70DFF0746B368626803F00C0337
:105B2800B3EB820FD4D0FCF703FFC01B4045F3D979
:105B38007FE7032A02D1FFF7BCFBDEE712B9FFF7C4
:105B4800A9FBDAE74FF0B0431B685B05D8D43EE702
:105B5800236823F007032B432360FCF7E9FE06467E
:105B6800236803F00703AB42B8D0FCF7E1FE801BC3
:105B78000228F5D95DE700BF00400058B8000020B2
:105B8800BC00002008B5FFF773FC4FF0B043044A8F
:105B98009B68C3F3022352F82330D84008BD00BFE6
:105BA800FC0D010808B5FFF763FC4FF0B043044A49
:105BB8009B68C3F3C22352F82330D84008BD00BF06
:105BC800FC0D01084FF0B043D3F89000C0F340003B
:105BD80070474FF0B0410209D1F8883002F47F22B3
:105BE800000123EA020300F47F200343C1F8883050
:105BF80070474FF0B041020CD1F88830120423EA04
:105C0800020343EA0040C1F88800704770B506688F
:105C180016F48036044638D0FFF770FAFCF788FE91
:105C2800614E05463368DB0529D54FF0B043616BFB
:105C3800D3F8902002F44072914214D0D3F8901017
:105C4800D3F8902042F48032C3F89020D3F8902003
:105C580021F4407022F480328D07C3F89020C3F8F5
:105C6800900000F190804FF0B042616BD2F8903014
:105C780023F440730B43C2F89030002605E0FCF78C
:105C880057FE401B0228CDD903262568E8070AD508
:105C98004FF0B0416268D1F8883023EA124392B2DB
:105CA8001343C1F88830A9070AD54FF0B041A2685C
:105CB800D1F8883023EA124392B21343C1F88830EE
:105CC800AA0609D54FF0B0422169D2F8883023F4EA
:105CD80040630B43C2F88830AB0502D5206AFFF752
:105CE80088FF680502D5606AFFF783FF290502D59A
:105CF800A06AFFF77EFF6A0602D56069FFF769FFB1
:105D08002B0602D5A069FFF764FFE80502D5E06914
:105D1800FFF75FFFE90610D54FF0B042E168D2F80F
:105D2800883023F440730B43C2F88830B1F5807F84
:105D380002BFD36843F08073D3602A040ED54FF0B6
:105D4800B042216BD2F8883023F040430B43C2F8AD
:105D5800883019B9D36843F08073D3606B0410D5C9
:105D68004FF0B042E16AD2F8883023F040530B4339
:105D7800B1F1005FC2F8883003D1D36843F48033AF
:105D8800D360304670BDFCF7D3FD41F28836054636
:105D9800FFF718FF01283FF466AFFCF7C9FD401B69
:105DA800B042F5D970E700BF0004005830B590F84C
:105DB8002C30012B02464FF0020022D0174B82F8FC
:105DC8002D00CA24012582F82C505C6253245C62A1
:105DD800B1F5807F146B996914D121F488519961C8
:105DE800596C24F0010421F0004159641463DD6505
:105DF8000A4BFF2159620020012382F82D3082F8D6
:105E08002C0030BD21F408519961D96C24F00204AA
:105E180021F00041D9641463D865E9E700280040FF
:105E280070B50B4E036B756D1D40EA07044603D52C
:105E38000123F365FCF78FFEAB0704D50223F36556
:105E4800204600F0CBF9012384F82D3070BD00BF47
:105E58000028004038B50A4CE36823F02003E360CB
:105E6800FCF766FD0546E3689B0601D5002038BDB2
:105E7800FCF75EFD401BB0F57A7FF4D90320F6E706
:105E8800002800402DE9F041114DEC6814F0400461
:105E980007461AD1EB6843F08003EB60FCF748FD36
:105EA8004FF003080646EB685B0601D4032C02D1C9
:105EB8002046BDE8F081FCF73BFD801BB0F57A7FFA
:105EC80084BF87F82D800324EDE70024F0E700BFA6
:105ED8000028004038B50F4CE36823F08003E360E6
:105EE800A3699B06054606D4FFF7B4FF10B103204B
:105EF80085F82D0038BDA36923F02003A361FFF7BF
:105F0800A9FF10B1032085F82D00A36943F02003F1
:105F1800A361EFE70028004038B5044600284BD0BD
:105F280090F82D3003F0FF021BB980F82C20FCF705
:105F380001FB0223214D84F82D30EB68DB0632D4B7
:105F4800CA236B6253236B622046FFF79BFF78BB23
:105F5800AB6923F08E6323F04003AB61216963686A
:105F6800AA690B431343A2691343AB61D4E9022323
:105F780043EA02432B61D4E90931EA680B4322F46E
:105F8800F8521343EB602046FFF7A4FF80B9D4E929
:105F98000713AA690B4322F0604213436269134353
:105FA800AB61FF236B62012384F82D30002002E0EF
:105FB800024BFF225A6238BD0120FCE7002800404E
:105FC8000023092803D840EA0310C0B270470A38F2
:105FD8000133C0B2F5E700002DE9F04790F82C3006
:105FE800012B05464FF0020069D0012385F82C30BB
:105FF8004E4B85F82D00DE6806F44076B6F5807FB6
:1060080078D04C69087891F8019091F802A091F83D
:106018002470002A55D19B6913F0400308BFCB7048
:10602800FFF7CEFF80464846FFF7CAFF02465046B4
:10603800FFF7C6FF81463846FFF7C2FF0B6ACF78E5
:10604800234343EA875343EA090343EA084343EAFD
:10605800022343EA0063354ACA2050625320506243
:106068008C6A8869B4F5807F946945D124F4885492
:1060780094610124D465B6F5807F09BFCB691364A8
:106088000343536418BF5064284B4A681A672A6B45
:1060980042F001022A639A6942F488529A61244ABA
:1060A800D2F8803043F40033C2F880301F4BFF220F
:1060B8005A620020012385F82D3085F82C00BDE8B0
:1060C800F087B4F1803F07D0B4F5000F04D09B6986
:1060D80013F0400308BFCB700B6ACA781C4344EA2C
:1060E8000A0444EA004343EA092343EA825343EAA1
:1060F8000763B0E70023AEE724F408549461022450
:10610800D465B6F5807F09BFCB6993640343D36434
:1061180018BFD064054B4A685A672A6B42F00202DE
:106128002A639A6942F40852B8E700BF0028004081
:106138000008005890F82C20012A03464FF002006E
:1061480012D00A4A83F82D00CA21516253215162A4
:10615800916941F020019161FF21516200200122E3
:1061680083F82D2083F82C00704700BF00280040DA
:1061780090F82C20012A03464FF0020019D00D4A4E
:1061880083F82D00CA2151625321516291690A484E
:1061980041F080019161D0F8801041F48021C0F86D
:1061A8008010FF2151620020012283F82D2083F8FE
:1061B8002C0070470028004000080058064B5A6D14
:1061C800520610B5044603D54022DA65FCF7C6FC32
:1061D800012384F82D3010BD002800407047890045
:1061E80001F1804101F531410A607047890001F1F0
:1061F800804101F53141086870470000034AD2F830
:10620800903043F40043C2F89030704700040058BF
:10621800034AD2F8903023F40043C2F89030704714
:1062280000040058074B1A6822F040021A6040F434
:1062380041704FF4B85218605A601A6842F0400230
:106248001A6070470000015837B5054600284ED03F
:10625800837903F0FF046BB1032C0BD0254B4FF46B
:1062680000629A612868FFF7DDFF002401232B7183
:10627800AC602FE000236B712846FCF76FFA1E4ACA
:10628800D2F8903043F48053C2F89030002CE5D116
:1062980002234FF0B042AB71D2F8943023F400439C
:1062A800C2F89430154B1B681C214B43DB0C64214E
:1062B8004B430193019B93B90124AC60FFF79EFF08
:1062C8000C4B9A6842F400629A604FF400629A613B
:1062D800002CC7D00123AB71204603B030BD019B11
:1062E800013B0193D2F894305B04E3D4E6E7012440
:1062F800F2E700BF0004005800080058B80000206A
:1063080037B5174D2B6802461C204343DB0C64202D
:10631800434314480193019B93B901209060114CA9
:1063280021732B681C214B43DB0C64214B430193E5
:10633800019B6BB9012090600A4BDB6803B030BD4C
:10634800019B013B019383689C07E4D50020E6E7A5
:10635800019B013B0193A368DB07E9D5ECE700BF8C
:10636800B80000200000015837B5184D2B680246C8
:106378001C204343DB0C6420434315480193019BD5
:10638800A3B901209060124CFF2323732B681C25AE
:106398006B43DB0C64256B430193019B73B90120AC
:1063A80090600B4BDB680B7003B030BD019B013B69
:1063B800019383689C07E2D50020E4E7019B013B39
:1063C8000193A368DB07E8D5EBE700BFB80000201E
:1063D800000001580F4B13B51B680F4C182253438C
:1063E8001B0D64225343014601936269019B02F02D
:1063F800040223B902238B60012002B010BD019B67
:10640800013B0193606910F00200F6D0002AECD13C
:106418001046F2E7B80000200004005807B50379D9
:10642800012B0FD10A4B1B68182253431B0C0193F5
:10643800FFF7EEFE019B013B0193019B002BF9D175
:10644800FFF7DCFE03B05DF804EBFFF7C3BF00BF46
:10645800B8000020F8B51E468379012B154604467E
:106468000F46DAB22DD14379012B2AD0022342718B
:106478008371FFF7D3FF0D212046FFF7C9FEFFF711
:106488003FFF390A2046FFF73BFFF9B22046FFF7E6
:1064980037FF2E44B5420ED12046FFF7AFFEFFF777
:1064A80099FFA06801230038A3714FF0000318BFBB
:1064B80001206371F8BD15F8011B2046FFF720FF86
:1064C800E8E70220F6E7F8B51E468379012B154662
:1064D80004460F46DAB22FD14379012B2CD04271F2
:1064E800FFF79CFF1D212046FFF792FEFFF708FFEC
:1064F800390A2046FFF704FFF9B22046FFF700FFEC
:1065080000212046FFF7FCFE2E44B5420ED120465E
:10651800FFF774FEFFF75EFFA06801230038A37140
:106528004FF0000318BF01206371F8BD29462046CB
:10653800FFF71AFF0135E8E70220F6E7F8B51F462E
:106548008379012B154604460E46DAB22CD14379DD
:10655800012B29D04271FFF761FF06F0EF03A3F189
:10656800840253425341237131462046FFF750FEBF
:10657800FFF7C6FE2F44AF4210D1FFF73FFE842E2F
:1065880002D02046FFF726FFA06801230038A37138
:106598004FF0000318BF01206371F8BD15F8011B07
:1065A8002046FFF7ADFEE6E70220F6E7F8B51E46FF
:1065B8008379012B154604460F46DAB227D1437971
:1065C800012B24D04271FFF729FF39462046FFF7F7
:1065D8001FFEFFF795FE00212046FFF791FE2E448F
:1065E800B5420ED12046FFF709FEFFF7F3FEA0687B
:1065F80001230038A3714FF0000318BF0120637115
:10660800F8BD29462046FFF7AFFE0135E8E702202E
:10661800F6E737B50023ADF8043001AA02231221AA
:106628000546FFF7C3FFBDF80440022364BA01AA78
:10663800A4B219462846FFF781FFE20702D528468B
:1066480009F088FBA30702D5284609F089FB6007F3
:1066580002D5284609F0AEFB210702D5284609F0E5
:10666800AFFBE20602D5284609F0B0FBA30602D527
:10667800284609F099FB600602D5284609F076FB02
:10668800210606D514F4807118BF0121284609F0A7
:1066980073FBA20502D5284609F07EFB630402D5E8
:1066A800284609F099FB03B030BDF8B51E4683793A
:1066B800012B154604460F46DAB227D14379012B40
:1066C80024D04271FFF7AAFE0E212046FFF7A0FD55
:1066D800FFF716FE39462046FFF712FE2E44B54254
:1066E8000ED12046FFF78AFDFFF774FEA06801234C
:1066F8000038A3714FF0000318BF01206371F8BD83
:1067080015F8011B2046FFF7FBFDE8E70220F6E736
:10671800F8B51E468379012B154604460F46DAB2B2
:106728002BD14379012B28D04271FFF777FE1E2128
:106738002046FFF76DFDFFF7E3FD39462046FFF7DA
:10674800DFFD00212046FFF7DBFD2E44B5420ED1C8
:106758002046FFF753FDFFF73DFEA06801230038F0
:10676800A3714FF0000318BF01206371F8BD2946DB
:106778002046FFF7F9FD0135E8E70220F6E7026851
:1067880052E8003F23F0C00342E8003102680029C4
:10679800F5D102F1080353E8003F23F4000302F1A6
:1067A800080C4CE800310029F3D12023C0F88830C8
:1067B8007047000010B5026852E8003F23F4907358
:1067C80042E8003102680029F5D10F4C02F10803B4
:1067D80053E8003F234002F1080C4CE8003100293F
:1067E800F4D1C36E012B07D152E8003F23F0100308
:1067F80042E800310029F7D12023C0F88C3000236B
:10680800C366436710BD00BFFEFFFFEF38B50546FE
:10681800C8B12423C0F8883003681A68002422F01D
:1068280001021A601C605C609C60FCF743FAC5F8C2
:10683800904085F88440C5F888402046C5F88C40CB
:10684800EC662C6738BD0120FCE70000F8B504466B
:106858001346D4F88850202D32D1F1B1EAB1E06F57
:10686800A4F85620A4F8542000262122C4F89060E9
:106878002165C4F88820226888B1124FC762124F78
:106888000763124F2832C0E90D76FEF7F3F830B1EE
:106898001023C4F89030C4F8885001200FE0236812
:1068A80040221A62226802F1080353E8003F43F0CD
:1068B800800302F1080141E800300028F3D1F8BD57
:1068C8000220FCE7D9680008216900082D69000842
:1068D80008B50346806A1B681B6813F0200317D1AC
:1068E800A0F85630026802F1080353E8003F23F08D
:1068F8008003083242E8003102680029F2D152E8E8
:10690800003F43F0400342E800310029F7D108BDB9
:10691800FCF74AFAFBE7704708B5806AFFF7FBFF08
:1069280008BD7047806A38B50468D0F88830D0F858
:106938008C50A268120606D5212B04D10023A0F89A
:106948005630FFF71CFFA3685B0606D5222D04D13D
:106958000023A0F85E30FFF72DFFD0F8903043F009
:106968001003C0F89030FFF7DCFF38BD08B5806A27
:106978000023A0F85E30A0F85630FFF7D2FF08BD1C
:10698800704700000368D9691A682DE9F04140F69C
:106998000F0631429D68044610D18E0640F197805B
:1069A80002F0200605F080573E4300F09080436FC8
:1069B800002B00F08580BDE8F0411847AB4EAC488D
:1069C8002E401040304300F08280CF0709D5D00513
:1069D80007D501201862D4F8900040F00100C4F8EF
:1069E80090008F0709D5E80707D502201862D4F868
:1069F800900040F00400C4F890004F0709D5E8075C
:106A080007D504201862D4F8900040F00200C4F8BA
:106A180090000F070BD502F02000304307D0082064
:106A28001862D4F8900040F00800C4F890000E05F1
:106A38000AD5500108D54FF400601862D4F8903098
:106A480043F02003C4F89030D4F89030002B37D0AE
:106A58008B0609D502F0200205F080552A4303D0A1
:106A6800636F0BB1204698472668D4F89020B36826
:106A780002F0280203F0400353EA0205204621D021
:106A8800FFF798FEB3685F0617D5226802F108037E
:106A980053E8003F23F04003083242E80031002960
:106AA800F3D1D4F8800040B1724B8363FEF75BF8F2
:106AB80030B1D4F88000836B7DE72046FFF731FFC3
:106AC800BDE8F081FFF72DFFC4F89050F8E7E06EBD
:106AD800012840F08980CE0640F18680D00640F13A
:106AE800838010221A629A6851064BD5D4F8802008
:106AF80011684A6892B2002AE2D0B4F85C00904269
:106B0800DED9A4F85E200A6892062FD453E8002F35
:106B180022F4807243E800210029F7D103F108022A
:106B280052E8002F22F0010203F1080040E800219A
:106B38000029F3D103F1080252E8002F22F04002A5
:106B480003F1080040E800210029F3D12022C4F80D
:106B58008C20E16653E8002F22F0100243E8002160
:106B68000029F7D1D4F88000FDF7C8FF0223236776
:106B7800B4F85E30B4F85C10C91A89B22046FFF741
:106B8800FFFE9DE7B4F85E20B4F85E00B4F85C1030
:106B980080B292B2002893D0891A89B200298FD086
:106BA80053E8002F22F4907243E800200028F7D120
:106BB800314D03F1080252E8002F2A4003F108067C
:106BC80046E800200028F4D12022C4F88C20606711
:106BD800E06653E8002F22F0100243E80020002866
:106BE800F7D102232367C9E7CF0209D56E0207D57B
:106BF8004FF4801220461A62BDE8F04100F0A0BDB3
:106C080008060BD502F0800005F40005284305D0DE
:106C1800A36F002B3FF454AF2046CCE64F0611D5A6
:106C280056060FD553E8002F22F0400243E8002112
:106C38000029F7D12023C4F88830A1672046FCF743
:106C4800B3F83DE70D0206D5500004D52046BDE84F
:106C5800F04100F077BDCB017FF532AF002ABFF6D7
:106C68002FAF2046BDE8F04100F06BBD01000010D9
:106C78002001000475690008FEFFFFEFD0F88C20A2
:106C8800B0F86010222A08B5036855D15B6A826D96
:106C98000B401370836D01338365B0F85E30013BA0
:106CA8009BB2A0F85E30B0F85E309BB2002B42D1A8
:106CB800026852E8003F23F4907342E80031036809
:106CC8000029F5D103F1080252E8002F22F0010251
:106CD80003F1080C4CE800210029F3D12022C0F868
:106CE8008C20184A41679342016705D1C26E012A78
:106CF8000ED0FCF767F81EE05A681102F6D553E883
:106D0800002F22F0806243E800210029F7D1EDE747
:106D18000022C26653E8002F22F0100243E8002147
:106D28000029F7D1DA69B0F85C10D20644BF102206
:106D38001A62FFF725FE08BD9A6942F008029A61B7
:106D4800F9E700BF00800040D0F88C20B0F8601050
:106D5800222A08B5036852D15A6A1140826D22F876
:106D6800021B8265B0F85E20013A92B2A0F85E205C
:106D7800B0F85E2092B2002A40D153E8002F22F4E6
:106D8800907243E800210029F7D103F1080252E884
:106D9800002F22F0010203F1080C4CE80021002921
:106DA800F3D12022C0F88C20174A4167934201672B
:106DB80005D1C26E012A0ED0FCF704F81EE05A680D
:106DC8001102F6D553E8002F22F0806243E8002133
:106DD8000029F7D1EDE70022C26653E8002F22F020
:106DE800100243E800210029F7D1DA69B0F85C10F5
:106DF800D20644BF10221A62FFF7C2FD08BD9A6985
:106E080042F008029A61F9E7008000402DE9F74F47
:106E18000368B0F86080DF691A689D68D0F88C1044
:106E280001922229044640F0B480B0F86890DFF857
:106E38006CA1DFF86CB10026B9F1000F01D0BB06D8
:106E480021D4B4F85E309BB2D3B1B4F868209A422A
:106E580016D9226802F1080353E8003F23F0805353
:106E6800083242E8003122680029F2D14D4B6367AD
:106E780052E8003F43F0200342E800310029F7D1EF
:106E880003B0BDE8F08F2368A26D5B6A03EA0803CC
:106E98001370A36D0133A365B4F85E30013B9BB258
:106EA800A4F85E302368DF6978072CD0F9070AD583
:106EB800019AD20507D501211962D4F8901041F042
:106EC8000101C4F89010B80709D5E90707D50221D0
:106ED8001962D4F8901041F00401C4F890107A07B0
:106EE80009D5E80707D504211962D4F8903043F092
:106EF8000203C4F89030D4F8903023B12046FFF74D
:106F080010FDC4F89060B4F85E309BB2002B93D1AA
:106F1800216851E8003F23F4807341E8003023687A
:106F28000028F5D103F1080252E8001F01EA0A011E
:106F380042E800100028F5D120215B45C4F88C10E8
:106F4800606720670AD05968090207D553E8001F0F
:106F580021F0806143E800100028F7D1E16E012993
:106F680013D1E66653E8001F21F0100143E8001032
:106F78000028F7D1D969CA0644BF102119622046F2
:106F8800B4F85C10FFF7FCFC56E72046FBF71AFF45
:106F980052E79A6942F008029A6171E7FEFFFFEF33
:106FA80000800040856C00082DE9F74F0368B0F8B1
:106FB8006080DF691A689D68D0F88C1001922229D8
:106FC800044640F0B280B0F86890DFF868A1DFF8B6
:106FD80068B10026B9F1000F01D0BB0621D4B4F87E
:106FE8005E309BB2D3B1B4F868209A4216D92268B1
:106FF80002F1080353E8003F23F08053083242E8C7
:10700800003122680029F2D14C4B636752E8003FF7
:1070180043F0200342E800310029F7D103B0BDE86E
:10702800F08F2368A26D596A08EA010122F8021B51
:10703800A265B4F85E20013A92B2A4F85E20DF6936
:1070480078072CD0F9070AD5019AD20507D501216E
:107058001962D4F8901041F00101C4F89010B807F3
:1070680009D5E90707D502211962D4F8901041F033
:107078000401C4F890107A0709D5E80707D5042158
:107088001962D4F8903043F00203C4F89030D4F871
:10709800903023B12046FFF744FCC4F89060B4F860
:1070A8005E309BB2002B95D1216851E8003F23F454
:1070B800807341E8003023680028F5D103F1080205
:1070C80052E8001F01EA0A0142E800100028F5D141
:1070D80020215B45C4F88C10606720670AD0596886
:1070E800090207D553E8001F21F0806143E800102A
:1070F8000028F7D1E16E012913D1E66653E8001F95
:1071080021F0100143E800100028F7D1D969CA0618
:1071180044BF102119622046B4F85C10FFF730FC18
:1071280058E72046FBF74EFE54E79A6942F00802FA
:107138009A6173E7FEFFFFEF00800040516D000881
:1071480038B5044603682169A2681D68C0690A4306
:1071580061690A437D49024329400A431A605A6813
:10716800E16822F440520A435A60794AA16993427D
:107178001CBF226A11439A6822F06E4222F43062E0
:107188000A439A60DA6A616A22F00F020A43DA62F5
:10719800704A93421CD14FF0B043D3F8883003F0C3
:1071A800030343F44033A3F54033013B022B00F2C1
:1071B800C780694A9B5CB0F5004F40F08980082B76
:1071C80024D8DFE803F061C08323802323236500EC
:1071D800624A934209D14FF0B043614AD3F88830EC
:1071E80003F00C0343F44023E4E7594A93420DD1DA
:1071F8004FF0B043D3F8883003F44063B3F5006F21
:107208001AD005D853B1B3F5806F12D0012009E028
:10721800B3F5406FFAD14FF400400EE0FEF7B2FC30
:1072280058B900204FF00113A3660023C4E91D33A9
:1072380038BDFEF7AFF8F3E74A4865684A4B626A1B
:1072480005EB450133F81220B0FBF2F39942DDD883
:10725800B3EB053FDAD800231946FAF755FC0902C3
:1072680041EA10616B080002C0182A464FF000037B
:1072780041F10001FAF748FC3C4BA0F540729A42F4
:10728800C4D82368D860CCE7FEF77CFC0028C8D0B7
:107298006168354B626A33F81220B0FBF2F24B0892
:1072A80003EB42034FF6EF72B3FBF1F3A3F11001C6
:1072B8009142ABD823F00F02216892B2C3F3420384
:1072C8001343CB60ADE7FEF765F8DFE72548DFE756
:1072D800082B9BD801A252F823F000BF2D73000899
:1072E8003973000845730008157200083F730008D9
:1072F8001572000815720008157200080973000855
:107308004FF400406368616A174A32F81120B0FBF5
:10731800F2F000EB5300B0FBF3F04FF6EF73A0F17F
:107328001002ACE7FEF72EFC00283FF47AAFE9E73D
:10733800FEF738FCF8E7FEF72DF8F5E70948E1E72E
:10734800B0F5004FF4D1FEF72DFC9FE7F369FFCFAE
:1073580000800040003801405C0E010800440040F5
:107368005F0EF5070024F4006C0E0108FFFC0F0007
:10737800836ADA0710B506D50168C46A4A6822F438
:10738800003222434A609C0706D50168046B4A68AC
:1073980022F4803222434A60590706D50168446BBB
:1073A8004A6822F4802222434A601A0706D50168F7
:1073B800846B4A6822F4004222434A60DC0606D500
:1073C8000168C46B8A6822F4805222438A60990655
:1073D80006D50168046C8A6822F4005222438A6048
:1073E8005A060FD50168446C4A6822F48012224379
:1073F800B4F5801F4A6005D14A68846C22F4C00243
:1074080022434A601B0606D50268C16C536823F400
:1074180000230B43536010BD2DE9F041DDF81880BF
:1074280004460E4615461F462268D36936EA03030A
:107438000CBF01230023AB4201D0002027E0B8F1A4
:10744800FF3FF2D0FBF774FAC01B4045206802D812
:10745800B8F1000F1DD150E8003F23F4D07340E885
:107468000032002AF7D100F1080353E8003F23F067
:10747800010300F1080141E80032002AF3D120237A
:10748800C4F88830C4F88C3084F884200320BDE820
:10749800F08103685A07C7D5C3691B05C4D54FF4E3
:1074A8000063036250E8003F23F4D07340E80032E1
:1074B800002AF7D100F1080353E8003F23F0010345
:1074C80000F1080141E80032002AF3D12023C4F872
:1074D8008830C4F88C30C4F89030D5E773B50446CA
:1074E8000026C0F89060FBF723FA23681B681A0788
:1074F800054619D423681B685B070AD56FF07E43DD
:10750800009300222B464FF480012046FFF784FFAA
:10751800B0B900202023C4F8883084F88400C4F867
:107528008C30E06620670CE06FF07E4300933246B3
:1075380003464FF400112046FFF76EFF0028D9D00C
:10754800032002B070BD10B5044650B3D0F888309F
:107558001BB980F88430FBF73DFB22682423C4F86C
:107568008830136823F0010313602046FFF7E8FD15
:10757800012816D0A36A13B12046FFF7F9FE236845
:107588005A6822F490425A609A6822F02A029A6055
:107598001A6842F0010220461A60BDE81040FFF761
:1075A8009DBF012010BD000030B581658168A0F83D
:1075B8005C200023B1F5805FA0F85E20436735D1D9
:1075C8000369002B40F2FF1318BFFF23A0F86030B7
:1075D8000023C0F890302223C0F88C30016801F1F4
:1075E800080353E8003F43F00103083141E8003441
:1075F8000368002CF2D1456E84680169B5F1005F1B
:1076080034D1B0F86850954230D8B4F5805F1DD1B8
:10761800254A264C002918BF22464267C1B153E8C3
:10762800002F42F4807243E80021F7E729B9036983
:10763800002B14BF7F23FF23C8E7B1F1805FC5D1BA
:107648000369002B0CBF7F233F23BFE7174AE4E7FA
:1076580003F1080252E8002F42F0805203F10800BB
:1076680040E800210029F3D1002030BDB4F5805F47
:107678000FD10F4A0F4C002918BF2246426751B15B
:1076880053E8002F42F4907243E800210029F7D113
:10769800EAE7084AF2E753E8002F42F0200243E8FD
:1076A80000210029F7D1DFE7B16F0008156E000847
:1076B800516D0008856C0008D0F88C30202B30B450
:1076C80015D1B9B1B2B100230468C3660A4B9C4214
:1076D8000AD063681B0207D554E8003F43F0806373
:1076E80044E80035002DF7D130BCFFF75DBF02201C
:1076F80030BC70470120FBE700800040436E30B586
:107708002BB90123A0F86A30A0F8683030BD0368AF
:10771800094D9A689968094C490FC2F342626B5C3B
:10772800615CDB00B3FBF1F3A0F86A30AB5CA25CF0
:10773800DB00B3FBF2F3E7E78C0E0108840E0108C7
:107748007047704770471FB504AB03E9060090F80F
:107758008430012B04463AD0012380F88430242356
:10776800C0F8883003681A6822F001021A609A6823
:1077780022F440120A439A6071B95A68BDF80C00A5
:107788009DF80E1022F0100202435A605A6822F047
:107798007F4242EA01625A601A6842F001021A60A6
:1077A800FBF7C6F86FF07E42034600924FF4800163
:1077B80000222046FFF730FE38B92023C4F888306D
:1077C800002384F8843004B010BD0320F8E70220B9
:1077D800F9E790F88430012B0FD0012380F884302A
:1077E800016851E8002F42F0020241E80023002B13
:1077F800F6D180F88430184670470220704710B5DB
:1078080090F88430012B044617D02423C0F8883020
:1078180003681A68196821F00101196042F00052E2
:107828004FF0005141661A60FFF768FF2023C0F847
:107838008830002084F8840010BD0220FCE770B571
:1078480090F88430012B044617D005682423C0F82B
:1078580088302E682B6823F001032B60AB6823F077
:1078680060431943A960FFF749FF20232E60C0F841
:107878008830002084F8840070BD0220FCE70000F6
:1078880038B5084D052455F8043B2BB9013C14F0D4
:10789800FF04F8D1204638BDDB6898470028F5D0AA
:1078A800F9E700BFD0060020034BD870034B1B68D4
:1078B8001B6C03B118477047E4060020CC06002073
:1078C800034B1874034B1B685B6C03B11847704774
:1078D800E4060020CC060020F0B5314D314B95F977
:1078E8000420314E91B00C46012795F905108DF80A
:1078F800047002288DF809208DF80A1010D18DF82F
:107908000800D8711C7202F09FFD337803B114B1DE
:1079180001A803F003FA254B059A1A6011B0F0BDCF
:1079280059714FF480711A71D9801C7233788DF8AF
:10793800087053BB1F2306A88DF81C208DF818303B
:1079480002F064FF20238DF8183006A82B798DF8F3
:107958001C3002F05BFF22238DF8183006A86B79E3
:107968008DF81C3002F052FF21238DF8183006A83C
:107978006B798DF81C3002F049FF29238DF81830F7
:1079880006A80B4B079302F041FF02F05DFD0123AF
:1079980006A88DF818308DF81C3002F037FFB4E7D0
:1079A800E4060020C0000020C0060020C406002015
:1079B800000400017FB5092301A88DF8043003F005
:1079C800ADF90038044B059A1A6018BF01204042EF
:1079D80007B05DF804FB00BFC406002070B504467C
:1079E8000B46134962784A700020A2780A72087020
:1079F8001A884A729A788A72DB780B746368CB604B
:107A08000C4B1B68DA6A2AB1237803F0FB030A2BB4
:107A180000D09047084E052556F8043B1BB15B6A19
:107A28000BB120469847013D15F0FF05F4D170BD14
:107A3800CC000020CC060020D006002070B50446FB
:107A480010480123037063784370A3788372E36856
:107A5800C360E378037623694376237943720A4B3C
:107A68001B689B6A03B19847084E052556F8043BE6
:107A78001BB19B690BB120469847013D15F0FF05E6
:107A8800F4D170BDE0000020CC060020D006002014
:107A9800014B1868704700BFC406002000B58BB0C2
:107AA800012368468DF8003002F088FD38B99DF84A
:107AB8000400003818BF01200BB05DF804FB00205B
:107AC800FAE7000008B501F073FE48B9FFF7E6FFD2
:107AD800012806D0054BD879197AFFF7FDFE012059
:107AE80008BDBDE80840FFF7CBBE00BFC0000020BE
:107AF8002DE9F04186B005460E46174601F058FEBE
:107B080000287FD101F06CFE044640B9FFF7C6FF9C
:107B1800012807D03D4B197AD879FFF7DDFE6FF0C1
:107B2800020462E0DFF8E88088F80860003E18BFC9
:107B380001268DF80460374E687833798DF8123055
:107B4800694602F0D9FC00283ED08DF80440039421
:107B5800ADF810406FF0060495E803002E4B83E85B
:107B68000300337988F80A30394601A803F0DAF9B6
:107B78002A4B059A1A60112841D801A353F820F01E
:107B8800E77B00080D7C0008077C0008077C0008DC
:107B9800077C0008077C0008077C0008277B000892
:107BA800077C0008077C0008077C0008017C0008A7
:107BB800077C0008077C00080D7C00080D7C000885
:107BC8000D7C0008FB7B00082B788DF808306B785B
:107BD800ADF810306B6803934FF0FF34BCE7104BDF
:107BE80000221A70E31D18BF1446204606B0BDE8EF
:107BF800F0816FF00404F8E76FF00504F5E74FF043
:107C0800FF34F2E76FF00104EFE700BFC000002087
:107C1800E0000020E4060020F0000020C406002058
:107C2800C806002037B501F0E5FD144D052455F8C8
:107C3800043B5BB11B694BB155F8043C9B682BB105
:107C4800984718B155F8043C1B699847013C14F053
:107C5800FF04ECD1FFF714FE68B9094D2B7853B136
:107C6800084BADF80040D978019422466846FFF7E2
:107C78003FFF00B92C7003B030BD00BFD006002014
:107C8800C8060020E406002030B58BB0054601F098
:107C98008FFD0446002839D1FFF700FF012838D1AD
:107CA80068468DF8004002F089FC10B14FF0FF30B3
:107CB80004E09DF80430AB4202D100200BB030BD87
:107CC800012DF3D0022D11D0002DF7D1002BF4D0C7
:107CD80068468DF8045002F099FD0028E6D10E4B55
:107CE8001B681B6B002BE8D09847E6E7002BDDD11B
:107CF80068468DF8045002F089FD0028D6D1064B5D
:107D08001B681B6B002BD8D02846EDE76FF00100ED
:107D1800D4E76FF00200D1E7CC06002010B5044686
:107D28008AB018B94FF0FF300AB010BD002368467A
:107D38008DF8003002F042FC0028F3D19DF80430A1
:107D48002370F1E77FB500220B4620498DF8072004
:107D580001220A7042784A700446002A33D1027917
:107D68000A721A884A729A788A72DB780B740369E5
:107D7800CB60C378164D8DF80830037B8DF8093039
:107D8800836803932B68DB6A0BB102A898472B68BA
:107D98009B6B13B1227E02B198470E4E052556F80B
:107DA800043B1BB1DB690BB120469847013D15F038
:107DB800FF05F4D10DF10700FFF7B0FF637913B1A8
:107DC800054B01221A7004B070BD00BFCC00002022
:107DD800CC060020D0060020C806002010B50446B6
:107DE8008AB018B94FF0FF300AB010BD202368469A
:107DF8008DF8003002F0E2FB0028F3D1024A9DF929
:107E0800043023701371EFE7E406002000B58BB04F
:107E18002323019068468DF8003002F0F7FC003803
:107E280018BF012040420BB05DF804FB70B5654CEB
:107E380001468EB01822204606F0FEF8624B00225A
:107E48001A70FBF73BFF23784068012202FA03F11E
:107E5800014004D15D4B084608F0E4F8FEE75C49B0
:107E68005C481A4602F032F918B14FF0FF300EB0F4
:107E780070BD272304A88DF8103002F0C7FC564EB9
:107E8800564D002870D1012333702B68DB690BB184
:107E980000209847272304A88DF8103002F08EFBA5
:107EA800059B93F84820227093F8182193F81A310B
:107EB8006270A370464BD3E9020105F0AFFF054697
:107EC8000028D2D1464E062304A88DF8103002F0BF
:107ED80075FB059B736104A802F098FC022304A8B3
:107EE8008DF81030059602F069FB0836032304A8C4
:107EF8008DF81030059602F061FB0F2606F052F857
:107F0800012304A88DF814308DF8106002F07EFC6F
:107F180010230DEB03008DF810308DF8145002F08B
:107F280075FC04238DF8103004A8A3788DF814305C
:107F380002F06CFC3A238DF8103004A863690593AD
:107F480002F064FC02A920788DF8086004F0E8F8D3
:107F5800003818BF0120E0711420FFF757FFE079BF
:107F680003F0A4F9284682E728238DF810302B68FF
:107F78001B6943B104A802F021FB2B6805981B6913
:107F880040F2C4519847272304A88DF8103002F016
:107F98003DFC50B9012304A88DF8103002F00EFB07
:107FA8009DF81430002B7FF46EAF3378002B7FF4EC
:107FB8006CAF052204A88DF81020059302F026FC6A
:107FC80078E700BFE4060020C8060020940E0108E8
:107FD8000C07002024070020C0060020CC06002043
:107FE800A806002037B500230D4601930446D0B9F2
:107FF80000F0A8FB0190019BD3B10F4A42F824304E
:108008000E4A9A620E4A1268916B1963916C596311
:1080180092690C49D9625A6128465B680A49F2227A
:108028009847002006E001A900F092FB0028E2D062
:108038004FF0FF3003B030BDD0060020E1780008D3
:10804800CC060020BD790008B4050020194B07B5FF
:108058001860194B194A1A60194A5A60194A9A60E5
:10806800194ADA60194B02681A6042685A608268D5
:108078009A60C268DA60164A1A6182695A61154BB9
:10808800C26B5A60144A019119609A601946134AE2
:10809800DA600020FFF7A6FF48B901A800F056FBF8
:1080A800003818BF0120404203B05DF804FB4FF0D0
:1080B800FF30F9E7CC06002024070020457A0008A5
:1080C8004D7D000865810008E57900080C0700204F
:1080D800D9C00008FC060020B1780008C97800085B
:1080E80051B118B1012804D000207047044B0B602F
:1080F8007047044B0B60F7E74FF0FF30704700BF45
:10810800000400010100010208B503F0EBF80028A3
:1081180014BF6FF00100002008BD08B502F0BCF9DB
:10812800002814BF6FF00100002008BD10B50446F8
:108138008AB018B94FF0FF300AB010BD2123684645
:108148008DF8003002F03AFA0028F3D1024A9DF97E
:10815800043023705371EFE7E40600202DE9F04165
:108168002E4D2F4F00232B7043786B703B689B6A12
:108178008AB004460BB128469847DFF8A880052640
:1081880058F8043B1BB11B6A0BB120469847013EC7
:1081980016F0FF06F4D12378052B2FD00B2B35D002
:1081A800012B25D1204C062368468DF8003002F0BB
:1081B80005FA0199E07905F077FE10B91B4B019A91
:1081C8005A611B48FFF70AFE1A48FFF7AFFF6B78A2
:1081D8008BB9A371184B5878FFF756FD3B685B6A5B
:1081E8000BB1114898476B7813B9E07905F0ECFEAC
:1081F8000AB0BDE8F081FF23A371EFE70F4B01221E
:108208005A74227A9A74627ADA74F1E76378002BE6
:10821800EED00AB0BDE8F041FFF7CCBBE00000208B
:10822800CC060020D0060020C0000020A8060020B0
:10823800C4000020C5000020E4060020CC00002077
:1082480030B58BB0FFF769FF0446F0B903F048FF7B
:10825800831C1DD0F8B9134D2B685B69DBB127234C
:1082680068468DF8003002F0A9F92B6801985B691F
:108278004FF4B961984703F045FF78B92CB9094B19
:108288001B68DB690BB10120984720460BB030BD55
:108298006FF00704EFE74FF0FF34ECE74FF0FF34DF
:1082A800F3E700BFCC060020014B1878704700BFE9
:1082B80038070020014B5878704700BF3807002066
:1082C80070470000044B9A7A0AB101225A70034B96
:1082D8005B6903B11847704738070020FC0000208D
:1082E80073B5224C6378002B33D008F085F96668A3
:1082F8000546FFF7CDFB0644AE4214D2A37A93B1EC
:10830800E0228DF800208DF80130217AE36801938E
:1083180001226846FFF7ECFB08B1073010D10023B3
:108328006370A372656094F83430EBB1002384F86D
:1083380034300F4B5B6BBBB102B0BDE870401847DF
:1083480040F2DC510B4808F023FA0A4808F0E6F935
:10835800E8E794F83520002AE5D094F8360084F848
:108368003530FFF791FCDEE702B070BD380700201A
:10837800FC0000207007002037B5104D104CC8B124
:10838800C1B10123627200222860E16023700D48A8
:108398000D4B00924FF0FF3108F014F900250B48FF
:1083A80025822022294605F05BFE6570A574A58606
:1083B80003B030BD00232B602370EFE734070020A3
:1083C8003807002070070020CD8200084C070020E5
:1083D8002DE9F0478E4C23788CB0002B56D0C2780C
:1083E8000AB9837B13B1238A01332382437B002B91
:1083F8004CD0E02A4AD10023A372876897F80080FE
:10840800B8F1220F27D8B8F1220F30D8DFE818F0DA
:108418004100FB0052005A0061006E0075008E009A
:108428009D00B400C7002F002F002F002F002F0041
:108438002F002F002F002F002F002F002F002F00BC
:108448002F002F002F002F002F002F002F002F00AC
:10845800C900D000D400B8F17E0F00F0CC80B8F18C
:108468007F0F00F0DF80B8F17D0F00F0AB80A57AB8
:10847800002D00F05B81674C637A3BB94FF47A7149
:10848800204608F085F9204608F048F90CB0BDE808
:10849800F087E36801220021A2721970A37AE168CB
:1084A8009818A0720620C854A37AE1689818A07298
:1084B800CA54DCE7584B9B6A002BD8D00121022014
:1084C8009847D4E77B7884F83630012384F8353030
:1084D800CDE704238DF804307B78003B18BF0123D7
:1084E80001A88DF8083002F091F9C0E778780038D3
:1084F80018BF012002F0DAFEB9E7484E0FCE01ADF1
:108508000FC50FCE0FC596E8070085E807007B78F2
:108518000A2BACD8424A12685268002AA7D00CA984
:1085280001EB830353F82C0C9047A0E77878431E9F
:10853800012B9CD83A4B01381B6818BF01202072C8
:108548009B68002B93D0984791E7E26801230821A4
:10855800A3721170627A057BA17AAA4228BF2A46C3
:10856800934284D285685A1CEB5CE56801334E1C43
:10857800A6726B54D3B2EDE7E3680122A272092216
:108588001A70A37AE268218A581CA072D154A27A80
:10859800238AE1681B0A501CA0728B5467E7238268
:1085A80065E705238DF8043001A802F0B7FB5EE704
:1085B800194BDB6A98475AE7194B78781B6860753E
:1085C800DB68BEE7037B072B7FF451AF06238DF8EA
:1085D8000430B7F80130ADF808307B793A791B04DC
:1085E80043EA0223FA781343642253430393BB7983
:1085F8008DF81030D8E73B2201A88DF804208DF8BB
:10860800083002F003F9012384F834302FE700BF63
:108618003807002070070020FC0000205C0C0108CF
:10862800340700202A2301A88DF8043001F0C6FF82
:1086380094F80A90E6689DF808009DF809509DF89E
:108648000A709DF80BC09DF80D309DF80E209DF81E
:108658000F109DF80CE009F1010A84F80AA006F849
:108668000980354E94F80A903668D4F80C8009F1E0
:10867800010A84F80AA096F803A008F809A094F85B
:108688000A90D4F80C8009F1010A84F80AA096F837
:1086980002A008F809A094F80A90D4F80C8009F10F
:1086A800010A84F80AA096F801A008F809A094F82D
:1086B8000A9009F1010A84F80AA096F80080E66891
:1086C80006F8098094F80A80E66808F1010984F838
:1086D8000A9006F808C094F80AC0E6680CF1010888
:1086E80084F80A8006F80C70A77AE66807F1010C8E
:1086F80084F80AC0F555A57AE6686F1CA77270550C
:10870800A07AE568461CA6722954A17AE0684D1C37
:10871800A5724254A27AE168501CA0728B54A37AC5
:10872800E268591CA17202F803E0A0E6034807F0CA
:10873800A7FF6570AAE600BF340700207007002075
:108748007047000000487047FC0000200020704778
:108758004FF0FF3070470000044B054A93F818317A
:10876800022B18BF062382F8903470474C0D002066
:1087780014130020034BD3F8483313B15B6903B1DA
:108788001847704714130020034A137843F0040372
:108798001370FFF7EFBF00BF101300201FB50A4B7F
:1087A8008DF8090093F87C208DF80A2093F88C2026
:1087B80093F848000D3202A98DF8082003F0B0FCA8
:1087C800C0B205B05DF804FB4C0D002010B5074C95
:1087D80004F5806007F054FF94F81A3413B10123AC
:1087E80084F81934BDE81040FFF7C4BF1413002003
:1087F80010B50C4CD4F8403343F08003C4F8403330
:1088080094F81A3413B10020FFF7E0FF94F891347C
:1088180023F0120343F0120384F89134BDE81040AA
:10882800FFF79ABF141300202DE9F041DFF8AC8060
:1088380098F81831022B06460D4602D0284BDB6A01
:10884800984702F0E9FD044628B1022002F0DAFD5B
:10885800002002F0DCFD98F81831012B17D102F046
:10886800DDFD074630B1002002F0CDFD002002F00A
:10887800CFFD3C4602F0D4FD48B1002002F0C4FD13
:10888800002002F0C6FDBDE8F041FFF765BF002CEF
:10889800F9D1144C94F8902494F81A34BAB90BB15D
:1088A80084F84164304602F065FFD8F82C0007F0E0
:1088B800ADFED4F8B4339842E5D30B4807F0E0FE98
:1088C80094F8913443F0100384F89134DBE70BB14A
:1088D80084F84154284602F04DFFF1E74C0D002082
:1088E8001816010814130020AC16002073B5164C96
:1088F800164D04F57A76EB6C95F8502095F97810BA
:1089080095F84800009603F031FC95F8303184F86A
:10891800FC3395F8480040F2012304F22442314622
:10892800A4F8FA3303F02EFC58B194F8243484F8F0
:108938006A34074B00205B6B984794F8FB3384F844
:10894800903402B070BD00BF141300204C0D0020FD
:1089580018160108074A10B5137843F0020313707C
:10896800FFF708FFBDE81040034B01220021022059
:1089780007F058BB10130020DD0E0108074A10B598
:10898800137843F008031370FFF7F4FEBDE81040B6
:10899800034B01220021022007F044BB10130020E2
:1089A800ED0E01082DE9F0410F4616461D4680469A
:1089B80007F022FE0B4A0C4C1378278123F0110391
:1089C80043F011031370C4E9000866812573FFF7AB
:1089D800D1FEBDE8F041054B01220021022007F03D
:1089E80021BB00BF10130020C0180020FD0E010895
:1089F80013B507F001FE0D4B6C461860204607F0D2
:108A08004FFD94E803000A4A0A4B83E803001378F1
:108A180043F020031370FFF7ADFE074B012200213E
:108A2800022002B0BDE8104007F0FCBAD0180020C0
:108A3800101300204C1600200A0F0108F8B5334D1A
:108A480095F81841012C06464BD0022C51D064B938
:108A580038B9D5E91B0105F1740383E80300204602
:108A6800F8BD01283DD0022801D00324F7E7284F9C
:108A780085F8180107F5747EBEE80F0007F57A7CC3
:108A8800ACE80F009EE8030095F8E9308CE8030095
:108A980087F8FB63E3B195F80031022B18D1D5F8BC
:108AA80004316B67C7F8EC3395F87D3095F80821E9
:108AB80087F8F83395F88C3085F8782087F8F933FB
:108AC80097F81B2487F8E82340F20133A7F8FA3314
:108AD800002387F81A340F4BDB6A9847FFF706FF25
:108AE800BDE702F0A4FC04460028B8D185F8186157
:108AF800B5E70028B9D1064B85F81801062283F896
:108B08009024044BDB6A98473446A8E74C0D0020B4
:108B180014130020181601082DE9F04192B00646FA
:108B280002F07AFC002840F05981AD4D95F81831D3
:108B3800012B09D02B6BAB4C93B194F80431BBB12A
:108B4800042B6FD0032003E002F068FC18B10F205B
:108B580012B0BDE8F08102F063FC0028EAD0F6E725
:108B6800B5F82031D4F81C24013B53432B63E4E7C8
:108B78009D4803F00CFA002840F02C8194F80C3141
:108B880023802B6B0C930DF1180895F839308DF86C
:108B98003830404695F81C318DF83A3007F0A6FC7D
:108BA800D5F82831009302AF98E80600D5F82431AB
:108BB800384607F032FC97E803000FAB83E8030060
:108BC800EB6A0D9300238DF844302388ADF84630C6
:108BD80095F8303101228DF839201BB98DF84420E1
:108BE8008DF83930814B0093814B95F84800A3F1FB
:108BF80079020CA903F009FBC0B10B28A8D1D4F85D
:108C0800941499B1002EA3D0D4F84033794843F096
:108C18002003C4F8403307F0BBFD764807F07EFD1B
:108C2800002095E7704803F0E6F9A4E795F8487046
:108C380095F9693095F9392095F87D106E4E3846CA
:108C480003F0F0FA009641B2EB6C95F850203846E4
:108C5800183603F08BFA0096EB6C95F8502095F9CE
:108C6800701095F8480003F081FAD4F8C413AB6D7E
:108C7800D4F8DC230B44C4F8B033EB6D1344C4F8C8
:108C8800B43394F80431042B07D02B6E0B44C4F88A
:108C9800B0336B6E1344C4F8B4330023089395F8CB
:108CA800303183B108A802F095FC00284ED195F91F
:108CB800390094F837629DF82070FFF76FFD3E4445
:108CC80080B2B04240D300238DF8133095F8393084
:108CD8008DF8213095F838308DF82230D5F880306D
:108CE8000993D5F884300A932388ADF82C3095F889
:108CF800303194F81B648DF82E3095F848003F4BBE
:108D08008DF820600DF1130208A903F043FA01233E
:108D180084F8413495F8393084F842349DF813309A
:108D280084F84334D4F81C34C4F85064C4F8483484
:108D3800C4F8583402F076FB50B1D4F81C0402F0A1
:108D480083FB28B1102003E7082001E71320FFE682
:108D580095F81831012B01D102F078FB02F065FB80
:108D68000023059394F8043195F9395094F81B645D
:108D78009BB1042B7FF4E6AE05A802F067FE58BB52
:108D880094F8183413B1059B013B0593164B0598CD
:108D98003246E9B202F0C0FE02E0134802F090FE4B
:108DA800C0B9D4F8403394F80C11218043F0020381
:108DB800C4F8403394F8183411480133DBB284F80E
:108DC800183484F845340F4B00259B6AC4F898542E
:108DD800984725E71120BBE61220B9E60E20B7E632
:108DE8004C0D0020141300201C1400207C0D0020C2
:108DF800A81700207C160020CC1600203017002071
:108E08001613002018160108F0B5504C504EB4F84F
:108E1800DC202287D4E92D0194F8B12084F8692058
:108E280004F16C0282E80300D4E92F0104F1740212
:108E380082E80300B4F8C420A4F87C2091B0D4F8E8
:108E4800CC20D4F8C810C4F884200025D4F8D02049
:108E5800C4F888200123A4F82031C4F8801084F8CD
:108E68003051A56284F81B5184F83A5084F81D519A
:108E780084F81E51C4F83451C6F89854A6F818540A
:108E880086F81A54A4F838518DF8183004F5097387
:108E9800039304F50A7394F84800A4F84651049320
:108EA80003A92C4B84F84551C4E94F55059303F0A9
:108EB80045F9E36EC6F8D43394F87D3086F8E0338C
:108EC80094F88C3086F8E1334FF48073A6F8E233D7
:108ED80086F8D05394F8303186F8E43306F5747781
:108EE8000FCF06F57A740FC497E8030040F2012308
:108EF80084E80300A6F8FA33D6F8483386F81B54FA
:108F0800CDE901551BB15A685B6901920293124B76
:108F18000793A3F148020892A3F1140209920F4A99
:108F28000B9229330A93A2F19C030C93A2F19803A4
:108F38000D93131D0E9301A902F14C0307A802F526
:108F480099620F9302F05DFA11B0F0BD4C0D00204C
:108F580014130020301800207C170020300E002049
:108F6800F8B50D4F0D4C0E4E0D4607F089FB3B6BC7
:108F7800984796F8480004F22442294603F002F97B
:108F880048B194F8243484F86A34706D7B6B984740
:108F9800EB7C84F89034F8BD1816010814130020EF
:108FA8004C0D00200F4890F81B3480F8B8330E4B56
:108FB80093F8692080F8BB2393F87D2080F8C823B4
:108FC80093F88C2080F8C92393F8303180F8CC339B
:108FD8000022A0F8CA2300F56E7100F56070FFF753
:108FE800BFBF00BF141300204C0D0020114890F89B
:108FF8009034EBB190F81B3480F8D0330E4BDA6E16
:10900800C0F8D42393F87D2080F8E02393F88C20CF
:1090180080F8E12393F8303180F8E4334FF480721C
:10902800A0F8E22300F5747100F56670FFF798BFA9
:10903800704700BF141300204C0D002070B5344C4D
:109048002421204605F00EF8636A984218BF606232
:109058004FF01C012F4814BF0125002505F002F828
:10906800636C984218BF60644FF480712A4818BF37
:1090780045F0020504F0F6FFD4F84831984218BFCD
:10908800C4F848014FF0D401244818BF45F004053E
:1090980004F0E8FFD4F82032984218BFC4F8200240
:1090A8004FF000011E4818BF45F0080504F0DAFF2C
:1090B800D4F82432984218BFC4F824024FF46071DF
:1090C800184818BF45F0100504F0CCFFD4F8A835AF
:1090D800984218BFC4F8A8054FF01401124818BFE9
:1090E80045F0200504F0BEFFD4F8C03598420F4B78
:1090F80018BFC4F8C005D3F8483318BF45F0400579
:109108002BB11B691BB12846BDE87040184770BDDC
:109118004C0D0020740D0020940D0020980E0020A6
:10912800700F0020740F0020F81200201413002084
:109138002DE9F04F91B04FF00008012B05460F467E
:1091480002928DF81580ADF8188003D8C84EC14634
:10915800B94502D311B0BDE8F08F15F8090002F047
:1091680077FA4844B842F5DC15F8093009F10104EA
:10917800023BE4B2112BEDD801A252F823F000BF54
:10918800D191000803920008039300082D9300086A
:10919800B5930008DD9300084F94000881940008F7
:1091A800FD9400085D9100085D9100085B9500083A
:1091B8005D9100085D910008199600084196000825
:1091C80085960008C3960008052002F0EDFA90B1D4
:1091D8000521002002F0ACFA2A5DA64B09F1030430
:1091E80009F102095FFA89F983F85C2415F8092066
:1091F80083F85D24E4B2A146AAE700238DF816306F
:109208008DF817308DF81C308DF82030B8F1000F2C
:109218006CD14FF0050896F87C208DF83920631E34
:1092280096F839208DF83B202B4496F838200D937A
:109238008DF83C2096F81A3196F868208DF83D2074
:10924800D6F82C218DF83A300C9273B37B1C1B1B7B
:10925800DBB28DF8383008AB019307AB009396F872
:1092680048000DF117030DF116020CA902F09EFF3C
:109278008DF8150000F00700072813D196F939205A
:109288009DF9163086F839309A429DF8173086F8DD
:109298003830B8BF01229DF81C30B8BF86F81D21B0
:1092A80086F868304FF0000909E00523D1E701226C
:1092B8000DF11501032002F0DBF809F101095FFA4D
:1092C80089F29DF82030B3FBF8F19142EFD823449E
:1092D800DCB2631EDBB29F420DD9EA5C032A9AD046
:1092E800A74288BF1C464FF0010884E709F1050929
:1092F8005FFA89F4F7E71C46F5E72B5D012203F0D6
:109308000F0309F1020986F81B3102FA03F35FFA29
:1093180089F9A6F82031002206A9042002F0A8F84D
:109328004C4668E707238DF815302B5D96F8480002
:10933800C3F3021203F00F038DF8303009F1030371
:10934800DBB28DF83120EA5C09F10403DBB209F1E4
:109358000504EB5C09F102095FFA89F91B0443EA89
:10936800022315F809201343642253430CA90D93D3
:1093780002F02BFF00F00703072BE4B28DF815006D
:109388000CD19DF8303086F8703086F878300D9B17
:10939800F36673679DF8313086F869308DF81800E8
:1093A800012206A9052002F063F824E7314BD3F81F
:1093B80048336BB11B685BB19847029B8DF8180066
:1093C80003F03F038DF81930022206A90620EAE7C8
:1093D800FF20F2E703238DF815302B5D8DF824303C
:1093E8000CAB089309F10303DBB209F10604EA5C4C
:1093F80096F8480009F10403DBB208A9EB5C1B04EA
:1094080043EA022309F10202D2B209F10509AA5C72
:109418001343642253435FFA89F90C9300230D9395
:1094280015F809308DF8383002F0D5FEC3B200289F
:10943800E4B28DF81530FFF6DEAE8DF81830012253
:1094480006A90720AFE72B5D03F00F03012B4FF4AC
:109458007A7238BF0123534309F10209B3651344F3
:109468005FFA89F9F365002206A9082056E700BFCC
:109478004C0D0020141300202B5D96F84800C3F310
:1094880040128DF81D2007A9C3F3001203F00F0343
:109498008DF81C208DF81E3002F0A3FE09F1020998
:1094A80001305FFA89F93FF43BAFBDF81C30914AAF
:1094B800A6F87C309DF81E309DF81C40D05CF8F76B
:1094C800A5FA0223C6F880000CA996F848008DF882
:1094D80030308DF8324002F023FE96F9393008908A
:1094E80040B29842B8BF184686F83900002206A94B
:1094F800092013E703238DF815302B5D8DF83030E4
:1095080009F10303DBB209F10504EA5C96F84800A7
:1095180009F10403DBB209F10209EB5C5FFA89F98E
:109528001B0443EA022315F809201343642253431A
:109538000CA90D9302F05BFEC3B20028E4B28DF8CB
:109548001530FFF658AE8DF81830012206A90A200A
:1095580029E7092002F028F9DFF89CA1002854D057
:109568000921002002F0E4F80023ADF8263009F1C3
:109578000203DBB24FF47A71EA5C09F10303DBB250
:109588000DF1300BEB5C1B0443EA02232A5D134305
:1095980009F10402D2B209F1060409F10509AA5C2D
:1095A8005FFA89F943EA026315F8092003934A43ED
:1095B80012125846ADF8242006F072FF039B03F1FF
:1095C800965303F5A91303F5EC530893DAF83C33E3
:1095D80000930DF1200999E80600DAF838330AA853
:1095E80006F01BFF0B9B00939BE806000A9B48466E
:1095F80006F0F8FE99E8030006F02AFF01F021FFC3
:109608000123E4B28AF83834F5E58AF83804F2E53B
:109618000C2002F0C9F800283FF4EDAD0C21002021
:1096280002F086F8344B93F89034043B012B7FF614
:10963800E2AD01F002FFDEE509F10203DBB22A5DCB
:10964800E95C09F10303DBB209F10504EB5C09F1FC
:1096580004095FFA89F91B0415F8090043EA012394
:1096680013436421594300F00F0001F0E7FEE4B210
:109678008DF81800012206A9112094E60D2002F0A9
:1096880093F800283FF4B7AD0D21002002F050F800
:1096980009F10203DBB2194AE85C2B5D126809F193
:1096A800040409F103095FFA89F943EA002015F86F
:1096B8000910E4B201F0C4FE9DE52A5D09F1020338
:1096C80009F1040409F10309DBB25FFA89F9E95CDD
:1096D80015F809301B0443EA012313436420584357
:1096E80001F0B0FEE4B28DF81800012206A913209B
:1096F80059E600BF170F010814130020C0180020F6
:109708000E4B93F89124920703D593F88F24012ADE
:1097180008D90B4991F81A2122B18A6A501C18BF3E
:1097280001328A620022A3F8182483F81A24D3F895
:10973800402322F00202C3F840237047141300208C
:109748004C0D002070B5184C184D04F55A7006F0F1
:1097580097FFD4F84033D4F89804D5F8906023F0F4
:109768002003C4F8403338B106F050FF864203D2D4
:10977800002385F83A3070BD0120FFF7CDF90028A5
:10978800F9D00B28F7D095F8393084F842340920FD
:1097980094F8183484F8453484F8410401F0EAFF59
:1097A800BDE87040FFF7ACBF141300204C0D00203B
:1097B800094BD3F84023012A0AD008490978C90778
:1097C80008D43AB993F89204013818BF01207047B9
:1097D8000020704701207047141300201013002048
:1097E800034BD3F84003431E58425841704700BF0B
:1097F800141300202DE9F04FA9B0EFF3108272B6D0
:10980800DFF8F4820021D8F80030C8F8001082F39D
:109818001088BA4C002B00F0E480DAB29B06039261
:1098280064D5B74D95F81831022B02D0B54BDB6AD9
:109838009847EFF3108972B6B34F06F0DDFE3E6825
:10984800D4F8B013361A3144B04806F0A1FFAF4837
:1098580006F064FFD4F8B413AD48314406F098FF1D
:10986800AB4806F05BFF89F3108894F81A34002B94
:1098780000F06D81152312A995F848008DF848303D
:1098880002F04EFCD4F8B4130F900144A14806F03E
:109898007FFFA04806F042FF3B6894F81B24EB6268
:1098A8000DAF38468DF870201D9306F01FFED5F8D1
:1098B8002831009306AE97E80600D5F824313046E3
:1098C80006F0ABFD96E803001FAB83E80300D4F86D
:1098D8001C341E9395F8303195F84800003B18BFAA
:1098E80001231CA98DF8713002F023FC039BDF06CD
:1098F8004BD5834DDFF820A2D5F8E420BAF90A3019
:10990800059298F800200493002363F300020A9359
:1099180088F8002084F84434049AA4F8223484F89F
:109928002534C4F82834A4F82C3484F82E34C4F828
:10993800303484F82034C4F8343484F83834C4F823
:109948003C34704B9AF90C90A4F88C2494F8902429
:10995800DB6A84F88E9484F88F24DAF80470BAF8F5
:109968000860984794F88F3413B9694806F088FE60
:109978003146384601F04EFD8346002800F0EA8063
:10998800049BA4F87E3484F88094039B19071AD5A5
:109998005B4B93F81831022B02D05A4BDB6A98477D
:1099A8000220FEF7D9FE84F8410401F0E3FE94F8A2
:1099B8001A3413B1012384F8193494F8913443F01C
:1099C800100384F89134039B5A0703D50621052018
:1099D800FEF72AFF039B9B0703D504210320FEF70C
:1099E80023FF01F035FD94F89124D7065FD50023B5
:1099F80084F89234D4F840331E0644BF23F082031F
:109A0800C4F8403312F0050F00F0FC820B2001F07F
:109A1800CBFE002800F0F68294F89134DD0700F1BF
:109A2800F182580740F10883D4F8403323F0020349
:109A3800C4F84033D4F8402382BB94F8915415F00D
:109A480001011EBF2B4662F3000384F8913494F899
:109A580091345E0744BF6FF3820384F89134012385
:109A680084F8923421B1D4F844332C481B689847C1
:109A78006D070BD52A4801F0A3FE01F0D1FE28B1ED
:109A880094F8913443F0040384F8913401F0CEFC47
:109A980094F891346FF3041384F89134012384F813
:109AA800923494F8913443F0200384F8913494F874
:109AB800913418070AD56FF3C3031A4984F891340F
:109AC800D4F84433A1F12400DB68984794F8913422
:109AD80099070AD56FF34103124984F89134D4F8F1
:109AE8004433A1F16C005B68984794F89034022BDA
:109AF8001AD1FEF7FBFE17E0101300201413002004
:109B08004C0D002018160108D018002094160020CB
:109B1800AC16002014170020C0180020541700208D
:109B280068170020A017002094F891349A0640F195
:109B3800C6826FF3451384F89134D4F84033002B70
:109B480040F0BD8229B0BDE8F04FFFF777BA84F83E
:109B58004134A1E695F81821012A0CD101F05EFCE8
:109B6800804668B1584601F04EFC584601F050FC5A
:109B7800042384F88F347EB9012384F8213450E11A
:109B880001F04EFC0028F6D0404601F03DFC40466E
:109B980001F03FFC0523ECE73B7804935B09013BAC
:109BA800062B00F21882DFE813F007001602950072
:109BB8001602920016020702102EDDD995F83031F0
:109BC8001297F6B28DF84C60002BD5D11CA804F082
:109BD8005DF912AA1CA9FF2002F0B2F89DF85830CE
:109BE800C3F3030307468DF82C3095F8480095F821
:109BF8007D308DF82D3007220BA902F0A4FA002F32
:109C08005DD100285BD09DF853309DF852201599FE
:109C1800C5F8E4101B0443EA02239DF851200220F2
:109C28001343C5F8E03004F03FF99DF8583095F833
:109C3800480085F82E71C3F30212C3F3030385F8B5
:109C4800703085F878309DF8593085F86920012BF7
:109C580038BF01234FF47A725343AB651344EB6565
:109C68000DF15A034FF001081093113E94F81B347C
:109C78008DF83C300FA985F868808DF8446002F0B3
:109C88006AFA0223404685F8303101F08DFD18B19B
:109C98004146384601F04CFD94F88F34012B00F210
:109CA800A88194F81A34002B40F09B8194F89134E1
:109CB80043F0100384F89134FEF74EFD65E6012069
:109CC80001F072FD0028E7D001210720E2E7012317
:109CD80084F8203495F87D308DF82E3094F82434AB
:109CE8008DF82D3095F88C3095F848000D330BA978
:109CF8008DF82C3002F014FAA6F10D031BB209906E
:109D080023EAE37300B283423FF736AF0B2E7FF6A8
:109D180033AFBB4B25931CA8FF231C978DF87460A9
:109D28008DF8983002F0D8F8074600287FF424AF61
:109D380095F81831012B13D101F070FB002873D06E
:109D4800384601F060FB384601F062FB04239DF8B9
:109D58007C101E9884F88F34C1F3001101F077FB52
:109D68009DF87C301E99C4F8341413F00F0203D008
:109D78009DF89000002863D19DF89800002862D0D3
:109D8800002A7FF4F9AE9DF89020002A0CBF4FF00E
:109D980002084FF0030800220A92D5F8EC209142FD
:109DA80054D195F8E910002950D0D5F80C1195F840
:109DB800EAB009680A9195F81811022902D103211D
:109DC80084F88F14B8F1030F7FF4D6AE13F0600F48
:109DD8007FF4D2AE0592012795F82E31BBF1000F22
:109DE80037D0BBF1010F38D1012B34D16FF0090600
:109DF80046FA08F606F00106C6F10206F6B2BDF804
:109E08007E100AAA304601F02DFE40B307280CBF89
:109E18000823012384F821340A9BC4F83034C4F899
:109E28006C34FEF7E5FCB0E501F0FAFA002897D0AB
:109E3800384601F0E9FA384601F0EBFA052386E7DF
:109E48004FF00008A7E74FF00108A4E74FF0010B17
:109E5800C2E70426D3E70326D1E70123DAE71CABE0
:109E6800009305990A9B3246584601F0BBFE20B183
:109E780002280CBF0A230B237FE60A9BC4F8303460
:109E8800C4F86C349DF87C3084F82104C3F3401383
:109E980084F82E3484F8443494F88F3484F8227487
:109EA800012B9EBF0122A86285F81E21012FC4F84C
:109EB800280484F82C0484F8410438D1022284F858
:109EC800202495F83A20002A4AD19DF87C20D6060D
:109ED80046D4012B94F840149DF87C2005D801291C
:109EE80001D1900601D501F05FFBB8F1020F94F89B
:109EF8008F3443D0B8F1030F0AD09DF87C10B8F125
:109F0800010F4A4601F00F0120A83BD0FFF710F9D6
:109F18009DF8903084F82334259BC4F828349DF8A4
:109F2800983084F82C34012384F82D3430E0049AD6
:109F380002F0E002A02A1BD195F82E11012285F823
:109F48003A2009B927996963012B84F8202407D995
:109F5800D5F89020C4F83C24DAF80020C4F89824F6
:109F680095F81821002AB4D1012284F82524B0E7F5
:109F7800002285F83A2084F82024A6E79DF8981056
:109F880025984A46FFF7D4F89DF8903084F8233492
:109F98009DF89020E02A08D195F81F312BB984F854
:109FA8002324C4F82834A4F82C3494F8913443F0CA
:109FB800020384F891346FE6114D013EB2B2791C68
:109FC800284604F039F80323A4F82034C4F82854A8
:109FD80084F82C64E9E7012384F82134FEF708FCAF
:109FE8005AE694F84434002B3FF460AE0020FEF7A4
:109FF800EDFB94F88F34022B3FF45EAE56E600BFBB
:10A008004C15002094F89134590715D5012001F01A
:10A01800CBFB60B1012001F09DFB08B984F818045E
:10A02800D4F8403323F00203C4F8403304E0062098
:10A0380001F0BAFB0028F3D194F89134DA077FF5E0
:10A04800F9AC94F840240AB1032A18D11D4A94F8AF
:10A05800181492F86820914205D29B0723D594F8EA
:10A068008F34012B1FD8184806F00AFBD4F8403368
:10A0780023F02003C4F84033FFF742FBDAE4012A57
:10A0880011D194F81924002A3FF4D4AC0D4A94F85D
:10A09800181492F868209142E5D29F0703D594F8E6
:10A0A8004434002BDFD194F8913400206FF304136B
:10A0B80084F8913484F81904FFF744FBBAE429B012
:10A0C800BDE8F08F4C0D00207C1600202DE9F04FE4
:10A0D80089468DB090460746002800F08F810029F8
:10A0E80000F08C810368002B00F088814368002B06
:10A0F80000F084818368002B00F08081C368002B06
:10A1080000F07C81104602F007F8002800F0788102
:10A11800BD4CBE4D384601F0C1FA40F2C452002190
:10A12800204603F09DFF40F21C520021284603F010
:10A1380097FFB74BC4F82C3104F50973089304F55D
:10A148000A7300264046099308A9B24B84F8488050
:10A158000A9384F8186184F88C608DF82C6001F0FB
:10A16800EDFF0F2306A994F848008DF8183001F088
:10A17800D7FF801B18BF01204FF00A0B84F81C0181
:10A1880006A994F848008DF818B001F0C9FF4FF0FF
:10A19800060A84F8DC0006A994F848008DF818A08F
:10A1A80001F0BEFF102384F8DD0006A994F84800EA
:10A1B8008DF8183001F0B4FF1123C4F89C0006A9EB
:10A1C80094F848008DF8183001F0AAFF1223C4F85B
:10A1D800A00006A994F848008DF8183001F0A0FFF7
:10A1E8001323C4F8A40006A994F848008DF8183081
:10A1F80001F096FF1423C4F8A80006A994F84800B3
:10A208008DF8183001F08CFF1623C4F8AC0006A9AD
:10A2180094F848008DF8183001F082FF172384F86D
:10A22800B10006A994F848008DF8183001F078FFBD
:10A2380018230DEB0301C4F8B400C4F8BC0094F86B
:10A2480048008DF8183001F06BFFC0B21D2384F868
:10A25800B80084F8C00006A994F848008DF81830B2
:10A2680001F05EFF1E2384F8C40006A994F8480094
:10A278008DF8183001F054FF1F2384F8C50006A993
:10A2880094F848008DF8183001F04AFF2023C4F8EC
:10A29800C80006A994F848008DF8183001F040FF6E
:10A2A8000B23C4F8CC0006A994F848008DF81830A0
:10A2B80001F036FF0C2306A9A4F8D00094F8480052
:10A2C8008DF8183001F02CFFD4F89C306365D4F871
:10A2D800A030A365D4F8A430E365D4F8A830236689
:10A2E8004FF00108D4F8AC300590A4F8D2006366AA
:10A2F80084F8B080C4F894B084F898A0C4F84CB03E
:10A3080084F850A084F8688084F81F81C5F84893C1
:10A31800FEF77AFD404B009632464FF0FF3105F5C7
:10A328005A70C5F84473C4E90B6684F8198185F836
:10A338009164C5F8408306F045F9384B00963246DB
:10A348004FF0FF3105F5607006F03CF9344B00968C
:10A3580032464FF0FF3105F5667006F033F902AF6B
:10A36800304B009632464FF0FF3105F5806006F01D
:10A3780029F9384606F0BAF897E8030004F592730D
:10A3880083E80300284B294F1E60294BC5F84C333E
:10A39800284BC5F85433284BC5F85C33274BC5F810
:10A3A8005033274BC5F8583305F553703B68984729
:10A3B80004F5A67003F088FB20B1112630460DB0D5
:10A3C800BDE8F08F204601F01DFB0028F5D101F013
:10A3D80041F8B8B91B4801F067FB06460028ECD1E4
:10A3E8007B69984703F006FEBB6D94F819019847FE
:10A3F800FB6A9847012385F89234DFE70326DDE7F7
:10A408000926DBE71326D9E74C0D0020141300209A
:10A4180000040001301800204D970008AD8F000897
:10A42800F58F0008D58700081013002018160108BA
:10A43800F9890008AD890008918700088589000816
:10A448005D890008340E002008B5034B0020C3F8CE
:10A458004003FEF781F908BD1413002010B5FFF77B
:10A46800A7F90A4C60B90A4B93F81831022B02D1AC
:10A47800084BDB6A98470123C4F84033002010BD1D
:10A48800D4F84003013818BF0120F8E7141300205E
:10A498004C0D00201816010838B5134C04F55A70F5
:10A4A80006F0EEF804F5607006F0EAF804F5667058
:10A4B80006F0E6F804F5806006F0E2F800F0B5FF73
:10A4C8000A4B0025DB6A9847C4F84053FEF7B6FDEF
:10A4D8000749084840F2C45203F0AEFD0123C4F80E
:10A4E8004033284638BD00BF141300201816010851
:10A4F8004C0D00208807002070B52E4B8AB0054609
:10A5080093F8DD008DF8090093F8DC008DF80A0057
:10A5180029489A6A90F81804039200268DF80B00CF
:10A5280004960C46002940D00692D3F8882007925A
:10A538001A8F93F81A118DF8151052BAADF8202019
:10A5480093F87C2093F848308DF8243003AB8DF8CD
:10A5580022008DF8232000930DF10A020DF10B0360
:10A568000DF1090105A88DF8146000F0DDFE9DF9D4
:10A578000900FEF713F9607004A801F02BF8B0B9D0
:10A58800049A0F2A0DD863789A420AD81544AB4228
:10A59800A3EB02012CBF002001202170C0000AB0EB
:10A5A80070BD002323700820F9E70320F7E7132084
:10A5B800F5E700BF4C0D0020141300201FB504461A
:10A5C800002800F012810078412800F20881DFE8B5
:10A5D80010F0420048004D00520056005A005F003B
:10A5E800060106010601060106010601060106012B
:10A5F80066006A006E0079008000830086008B0088
:10A6080089008D009100940097009A009D00A00099
:10A61800AF00B300BB00B700BF00C200C600CF0048
:10A62800CB00CD000601D300060106010601060194
:10A6380006010601060106010601060106010601DA
:10A64800060106010601DB00DF00E300E800EC007C
:10A65800F000F400FD00674B93F81831237104B043
:10A6680010BD644B93F83031237102E0606803F049
:10A67800C7FB0020F3E7606803F008FCF9E75D4BCF
:10A6880093F81A31F0E75B4BD3F8E0306360F0E7FA
:10A69800584B211D93F8300103F010FCE9E7554BA6
:10A6A80093F81931E0E7534B93F88C30DCE71C231F
:10A6B8008DF808304F4B02A993F8480001F030FD9F
:10A6C8006060D6E74C4B043493E8030084E8030049
:10A6D800CFE74A4B0434F7E7494B0434F4E7494BD6
:10A6E8000434F1E71A23E3E71923E1E7414B93F830
:10A6F8006830B9E73F4B5B6DC8E73E4B9B6DC5E7DC
:10A708003C4BDB6DC2E73B4B1B6EBFE7394B5B6EC7
:10A71800BCE702238DF80830364B02A993F87C2059
:10A7280093F848008DF80A2001F0FAFC2071A0E7A0
:10A73800304B93F8DD3097E72E4B93F8393093E799
:10A748002C4B93F8DC308FE72A4B93F838308BE7A3
:10A75800284BDB6C9AE7274B93F8503084E7254B5E
:10A76800D3F88430636084E7224B8FE7264B8DE76C
:10A77800204BD3F8CC30F5E71E4BD3F82C3163606F
:10A7880001F05CFDA06074E71A4BD3F890307DE7C8
:10A79800184B93F81F3167E7164BB3F88830A3803E
:10A7A80067E7144BB3F88A30F9E7124BB3F8D030A7
:10A7B800F5E7104BB3F8D230F1E70E4B93F8482089
:10A7C8000AB1062A13D1B3F8A035E8E7094B93F884
:10A7D80048200AB1062A0AD1D3F8A43556E72046FC
:10A7E80004B0BDE8104000F024BE032037E718206D
:10A7F80035E700BF4C0D0020B80D0020000E0020EA
:10A80800C00D0020080E0020880700207FB50446F0
:10A8180010B9032004B070BDA44DD5F840339A0791
:10A8280000F171820278412A00F26A82DFE812F0B0
:10A838004200480056005C00600065006A0077002E
:10A84800820088008E0094009A00A000A600AC0048
:10A85800B6006802BB00DD00F000170139012A01CB
:10A8680044014D015101550159015D016802610121
:10A8780073019B018901AD01B301BA01BF01C40194
:10A8880068022A02680268026802680268026802AE
:10A898006802680268026802680268026802680260
:10A8A8006802680236023B02400245024A024F0231
:10A8B80054025E020079FEF7C1F80028AAD105E02B
:10A8C8000379022BA5D07A4A82F8303195F8913471
:10A8D80043F0200385F8913400209BE7406803F09B
:10A8E80081FA0028F2D094E7406803F0BFFAF8E74D
:10A8F8006F4B027983F81A21E8E76D4B4268C3F879
:10A90800E020E3E76A4E416896F8300103F0CCFA9C
:10A9180000287FF47EAF6368C6F8E430D6E7416864
:10A9280000293FF476AF002001F0EEF90028CDD0E1
:10A9380011206FE7416800293FF46BAF0120F3E76E
:10A94800416800293FF465AF0820EDE74168002918
:10A958003FF45FAF0920E7E7416800293FF459AFAA
:10A968000C20E1E7416800293FF453AF0D20DBE7F5
:10A97800416800293FF44DAF0E20D5E74168002912
:10A988003FF447AF0F20CFE74A4C494B007983F893
:10A998001901A36D9847E36A984797E7444B0279F2
:10A9A80083F88C2092E7424E037A8DF8043096F8AB
:10A9B800480096F87D308DF80530072201A901F08E
:10A9C800C2FB00283FF425AF636896F8480001935E
:10A9D800002201A901F0B7FB00283FF41AAF6C363A
:10A9E800D4E9010186E8030070E7314E037A8DF857
:10A9F800043096F8480096F87D308DF80530072227
:10AA080001A901F0A0FB00283FF403AFB436E7E743
:10AA1800274E037A8DF8043096F8480096F87D3072
:10AA28008DF80530072201A901F08DFB00283FF4BD
:10AA3800F0AED4E9010106F1740383E8030096F847
:10AA48001831022B7FF442AF96F83031002B3FF4D7
:10AA58003DAF184BDB6A9847FDF748FF36E7144EC1
:10AA6800037A8DF8043096F8480096F87D308DF812
:10AA78000530072201A901F066FB00283FF4C9AEA2
:10AA8800BC36ADE74368029301238DF80C30084BC0
:10AA980002A993F8480001F063FB00287FF416AF81
:10AAA800B7E6436802930023EFE700BF14130020C2
:10AAB8004C0D00201816010803795A1E0E2A3FF67D
:10AAC800A8AE934A82F8683000E7914B42685A650D
:10AAD800FCE68F4B42689A65F8E68D4B4268DA656A
:10AAE800F4E68B4B42681A66F0E6894B42685A6670
:10AAF800ECE6874C037994F848008DF80430062278
:10AB080001A901F020FB00283FF483AE9DF8043032
:10AB180084F8DD30DAE67E4C03798DF8043094F859
:10AB2800480094F87C308DF80630052201A901F020
:10AB38000AFB00283FF46DAE9DF8043084F83930E4
:10AB4800C4E6734C037994F848008DF804300A225F
:10AB580001A901F0F8FA00283FF45BAE9DF8043033
:10AB680084F8DC30B2E66A4C037994F848008DF832
:10AB78000430092201A901F0E6FA00283FF449AEA1
:10AB88009DF8043084F83830A0E6614B4268C3F879
:10AB98009420DA649AE65E4B027983F8982083F869
:10ABA800502093E65A4B4268C3F884208EE6584BEF
:10ABB8004268C3F8CC2089E6012B40F0A480554CAC
:10ABC8002421204603F04EFA636A984201D01720E8
:10ABD80020E61C2104F1280003F044FA636C984233
:10ABE800F5D14FF4807104F1480003F03BFAD4F832
:10ABF80048319842EBD1D42104F5A67003F032FA1B
:10AC0800D4F820329842E2D1002104F5097003F00B
:10AC180029FAD4F824329842D9D14FF4607104F556
:10AC28000A7003F01FFAD4F8A8359842CFD114213E
:10AC380004F2AC5003F016FAD4F8C0359842C6D1E5
:10AC4800334E2146304640F2C45203F0F5F920460F
:10AC580040F2C452002103F003FA95F81B3485F83A
:10AC6800E833736FC5F8EC3396F87D3085F8F83320
:10AC780040F20123A5F8FA33274B96F819019B6D8A
:10AC8800984723E68379012B3FF6C3AD204B4268F2
:10AC98004068C3F82C2100F0D1FE47E61C4B4268FF
:10ACA800C3F8902012E61A4B027983F81F210DE6AB
:10ACB800174B8288A3F8882008E6154B8288A3F8EA
:10ACC8008A2003E6124B8288A3F8D020FEE5104BB9
:10ACD8008288A3F8D220F9E50D4B93F848200AB1F1
:10ACE800062A12D1A288A3F8A025EFE5084B93F80D
:10ACF80048200AB1062A08D16268C3F8A425E5E508
:10AD080000F099FBD9E5012084E5182082E500BF11
:10AD18004C0D002088070020181601082DE9F04383
:10AD280087B00023ADF800300646002800F0ED801B
:10AD38000361FEF73DFD20B10124204607B0BDE8C0
:10AD4800F08300F073FD0028F6D100F069FD01469C
:10AD580018B96F48142203F083F96E4D95F89134B1
:10AD6800012243F0040385F8552485F8913433789B
:10AD78008DF804300021013B8DF80520ADF8061050
:10AD88000C2B00F2BA80DFE803F007B8B8B8788176
:10AD9800B8B88FB8AC99A800D5F8407317F0200759
:10ADA800CAD196F80480B8F1020F45D1DFF868815E
:10ADB8005A4CFEF729F896F9051098F848003A46D3
:10ADC80001F01BFA88F83900B37988F8383038462A
:10ADD80007238DF80530FDF731FEFF2304F5867053
:10ADE800A5F80C31C5F8084185F8047103F04EF850
:10ADF80004F58A7003F004F83846FDF78DFE044622
:10AE080040B196F9051098F84800012201F0F5F9CB
:10AE180088F83900D5F894343361002C71D000F0EB
:10AE2800FFFC002889D195F8913485F81A0460F35D
:10AE3800820385F8913480E7B8F1010F4FF00204DE
:10AE4800E8D1DFF8D4908DF8144099F8480089F8D3
:10AE58001D7102A901F072F9337989F830318DF842
:10AE680005708DF80680FDF785FC95F8913443F060
:10AE7800100385F891340024CCE7002269460220AB
:10AE880000F0F6FA0028F6D01324C3E7244BB28862
:10AE9800DB6B96F90C10B0689847D5F8403343F04F
:10AEA8000203C5F84033E6E702A90D2000F060FB75
:10AEB8000028E0D0002269460D20E1E7164B93F800
:10AEC8001831D3B9347904F0070000F0ADFA8DF8E1
:10AED8000040012269461020D2E70022694612206C
:10AEE800CEE78DF8072000F090FA044638B900F054
:10AEF80089FA204600F08BFA8CE702248AE70124BD
:10AF080088E701A800F0DEFB17E7032415E700BF78
:10AF180068170020141300204C0D00201613002081
:10AF2800181601082DE9F04F99B08046059118B917
:10AF3800032019B0BDE8F08F00230361FEF738FC49
:10AF48000646002840F0AB8045460FCD0EAC0FC436
:10AF58005A4C98F800A0B8F80C7098F90EB0142262
:10AF680004F58860314603F07BF8012284F8412417
:10AF7800534C94F83021022A35460BD194F8182105
:10AF8800022A07D194F81E2122B9BAF1010F38BF5D
:10AF98004FF0010ABAF1010F2DD0BAF1030F2CD0EE
:10AFA800BAF1000F35D102229DF83C30DDF840900F
:10AFB800029362F34715012694F87C108DF832103D
:10AFC80002220CA994F848008DF8302001F0A8F866
:10AFD80094F81A3194F830C194F81D1140B2022245
:10AFE800002B6FD0BCF1010F65D1002963D1002E71
:10AFF8006DD1104627E00422D6E70023DDF83C9007
:10B00800BDF840709DF942B0029365F01F05012616
:10B01800D2E74FF0000BD946CDF808B0CCE74FF097
:10B02800010084F81A04DDE005F29A420BA900F049
:10B03800DDFA002800F020811320049B33871F4B82
:10B04800002283F81A241D4BD3F89434C8F8103022
:10B058006FE705F29A452A460BA900F0C7FA0028BF
:10B06800EAD10B9B84F82801C4F82C5184F83031BC
:10B0780002E1B9F1000F00F0FF80002A00F0FC8027
:10B088004946E01C02F0D8FF94F837320133238098
:10B09800F2E01220D1E70220CFE70720CFE7012016
:10B0A80047E7064B93F8912483F840A442F0010245
:10B0B80083F89124C7E7EEB90220C4E714130020EF
:10B0C8004C0D0020002E94D05845B8BF584694F82F
:10B0D8007C308DF82000052294F848008DF8223045
:10B0E80008A901F030F800283FF422AF9DF820307D
:10B0F80084F83930694A6A4BD2F89804D3F89040FA
:10B1080038B105F083FA664B84423CBF002283F8CD
:10B118003A20198F1A8F93F830010491996A09918E
:10B1280052BA0028B9D093F81B0100B9186393F8F4
:10B138001801ADF85820013893F87C2093F81A418B
:10B148001491D0F1000BD3F888108DF85B204BEBED
:10B15800000B93F8482093F83A0093F868308DF87C
:10B168005A3009AB00934F4B03904FF001008DF814
:10B178004C0015918DF85C20A3F12F01A3F130024A
:10B1880013A88DF84D4000F0CFF8039B4FEA0B1B36
:10B198004BEA431B00264BEA801B4BEAC413B1451C
:10B1A8003E4C039308BF37463A46494604F59C701F
:10B1B800CDE90A669B46268084F81A6402F03CFFB3
:10B1C800E9B2A570C5F34215FAB2042D344E039BBB
:10B1D80084F837223FF423AF072D3FF44AAF022DFE
:10B1E8007FF459AF304D84F80D110420029984F88A
:10B1F8000401FF2084F80C0184F8281184F8143124
:10B20800D6F8E410C4F8085105F59B730AA8C4F8E9
:10B21800101184F83021C4F82C3100F017FC0028F4
:10B228007FF437AF0A9BA4F844040BA8A4F816319E
:10B23800C4F84C3400F0CEF900287FF4FDAE0B9B27
:10B24800D3B196F93900FDF7A9FA94F83732002BF3
:10B258003FF4FFAE0B9B0F2B3FF6E6AE05F58B7266
:10B268000BA90F2000F0C2F900287FF4E5AE0B9B74
:10B2780063F3030B84F814B10598FDF74DFC00281F
:10B288007FF4DBAE099B86F83A00B36200F07EF9E2
:10B2980000283FF406AF1320D1E600BF14130020A6
:10B2A8004C0D0020B40D00201613002037B50B4DAF
:10B2B8008DF8040004460F2295F8480001A900F013
:10B2C80042FF40B1064A85F81C4192F8913443F098
:10B2D800200382F8913403B030BD00BF4C0D00202C
:10B2E8001413002010B5FFF7B9F8044688B90A48C6
:10B2F80005F0C6F9094805F0C3F9094805F0C0F991
:10B3080000F093F8FDF780FD064BDB6A984720466E
:10B3180010BD0124FBE700BF7C1600209416002016
:10B32800AC160020181601082DE9F04F8BB04778AD
:10B338000093149B90F90C8090F90D6090F80E9092
:10B348008B464168196004469246002F57D0022365
:10B358008DF8103004A9C37B007C8DF8123000F002
:10B36800DFFEB4F808C0618943B260689845454675
:10B378006144B8BF1D46604534BF00270127884295
:10B3880009D30A218DF81010207C019304A900F03C
:10B39800C7FE019B46B2B4F808C0608961680CEB2F
:10B3A800400E714520D3A1EB0C01B1FBF0FC00FB72
:10B3B8001C11C9B998450ADC237833B10223207CD3
:10B3C8008DF8243006A900F0B9FE4FF001092123B9
:10B3D8008DF81030207CE37B8DF8115004A98DF88E
:10B3E800123000F09DFE45B2009B8BF800503846A5
:10B3F8008AF8006083F800900BB0BDE8F08F4546EE
:10B40800F2E77047704770477047002070477047F1
:10B418007047704700207047002070470020704731
:10B42800002070470020704770477047704702201F
:10B43800704702207047022070477047002070470D
:10B44800704770470020704700207047704770476A
:10B458007047000010B5054C4FF4037220460021D8
:10B4680002F0FEFD0020C4E9000010BDD418002041
:10B478002DE9F8438146174600293FD0244B002583
:10B4880003F1010C1A462801103312F8018FB8F1A4
:10B49800000F36D19A42F8D11E4E33680BB9C6F860
:10B4A80000C073680BB1C3F800C03318002401351D
:10B4B8009C6083F80C900D302B01BAB206EB051591
:10B4C8003044F750C6F804C002F0B6FDB9F1110FC8
:10B4D8004FF0000398BF104C6B71D6F8083298BF34
:10B4E80024FA09F403F1010398BF04F001043B4472
:10B4F8002C71C6F808324046BDE8F8834FF00108C1
:10B50800F9E70135202DBBD14FF00208F3E700BF62
:10B51800DB180020D41800202007020010B510B353
:10B52800124A1368984204D103681360002304E0A8
:10B538000B4613B119688842FAD15168884208BF8E
:10B5480053600BB101681960D2F808328168013B79
:10B5580000245B1A04602146C2F80832102202F067
:10B568007FFD204610BD0120FCE700BFD418002055
:10B57800054B1B6813B11A798242FAD1002B0B6074
:10B588000CBF032000207047D418002010B5054BCD
:10B59800186800B910BD037B04680BB9FFF7BEFF3C
:10B5A8002046F6E7D418002038B5084B084C186830
:10B5B80000B938BD03790568112B05D824FA03F3BF
:10B5C800DB0701D5FFF7AAFF2846F1E7D4180020CA
:10B5D8002007020028B1044BD3F80832036000208A
:10B5E80070470120704700BFD41800202DE9F041B2
:10B5F80007460E4615463AB331B3144B1C68002370
:10B608002CB93046FFF7E6FF0020BDE8F081A268BC
:10B61800F91A0132914210D32279EA54581C22892E
:10B628005FFA80F8611D55FA80F002F005FDA36805
:10B63800246898445FFA88F3E2E720462468FFF715
:10B648006DFF002CF9D1DCE70120DEE7D4180020DB
:10B658000238C0B211289ABF014B185C002070470D
:10B66800270F010830B50B4B93F8202004460846F5
:10B6780072B100211C330578A54208D001319842E7
:10B68800CDB20CBF04480430AA42F4D8002030BD23
:10B698001046FCE7E01A0020EC1A002010B5084C10
:10B6A80000232060142204F10C00FF2184F82030CC
:10B6B800C4E9010002F0D4FC012384F8213010BD54
:10B6C800E01A002010B50E4A92F82010042915D867
:10B6D800936804781C7044785C70C478807898709B
:10B6E8000131DC7082F8201002F11C018B4214BF7A
:10B6F800043302F10C039360012010BD0020FCE725
:10B70800E01A0020094B93F8200068B15A6803F149
:10B718001C018A4200F1FF3014BF043203F10C020D
:10B7280083F820005A600120704700BFE01A00200B
:10B7380010B5074B93F820200446084632B15968E3
:10B74800FFF790FF10B101234470837010BD00BF54
:10B75800E01A002008B5064B93F820202AB1596852
:10B76800FFF780FF08B1407808BD0120FCE700BF63
:10B77800E01A002030B50A4A92F82010536882F87F
:10B78800210061B1916801241C32DD78587005B937
:10B798009C7093420CBF034B04339942F5D130BDE2
:10B7A800E01A0020EC1A002008B5044B5968FFF78E
:10B7B80059FF003818BF012008BD00BFE01A00205B
:10B7C8002DE9F3410422154E044600210DEB020039
:10B7D80096F8208002F044FC0025EBB2984502D888
:10B7E80002B0BDE8F0817368197821705A786270E8
:10B7F8009F785FB1336820469B689847FFF782FFC0
:10B8080017B901A8FFF75EFF0135E6E7DB788DF889
:10B8180004108DF805208DF80730EFE7E01A0020B6
:10B82800014B93F820007047E01A0020034B93F86F
:10B838002000042894BF002001207047E01A00204F
:10B848001FB50024CDE90244C41F8DF800408DF8CF
:10B8580001100C0AADF80420090C120C8DF8031025
:10B868008DF806208DF8073002461B0A012168462C
:10B878008DF802408DF8083002F04FFA002818BF02
:10B888000E2004B010BD2DE9F04188B017460D46D2
:10B898000F9A064600284DD000240121CDE9044422
:10B8A8008DF810109DF838108DF81510ADF8163079
:10B8B800190CCDE900441B0ECDE902448DF819306E
:10B8C800ADF81A20130C120E07948DF818108DF885
:10B8D8001C308DF81D20E3B24FEA0318002D5FFAE3
:10B8E80088F803DC002008B0BDE8F081013310219E
:10B8F8008DF81F303A466B460DEB010002F0A3F9B4
:10B908000346C8B9102DAC46A8BF4FF0100CDAB2E8
:10B91800624503F1010303DB103D2DB20134DAE780
:10B9280008EB020020326A44315C12F8202C4A40AD
:10B938003254ECE70920D6E70E20D4E70138032873
:10B9480015D8DFE800F002080C100A4B1B681B69C9
:10B958000B6000207047074B1B685B69F8E7054BD5
:10B968001B689B69F4E7034B1B68DB69F0E705205C
:10B97800704700BF041B00202DE9F041C4B00C46FD
:10B988004A9E17461D468046B8B3B1F5807F36D823
:10B998004FF488720021684602F062FB4923009345
:10B9A8004FF48073ADF804302B0C8DF80830330C4D
:10B9B800ADF80650ADF80A608DF80C302246002329
:10B9C800414604A82D0E360E8DF80E308DF809501C
:10B9D8008DF80D608DF80F4002F02EFB04F1100178
:10B9E8004B9A3B4689B2684602F017F910B1012814
:10B9F80018BF0E2044B0BDE8F0810920FAE70D20F9
:10BA0800F8E7000010B590B10A4C28220021206008
:10BA180002F026FB2368084A1A6000204FF0FF3224
:10BA2800C3E90302C3E90522C3E9072210BD0820C0
:10BA3800FCE700BF041B002000010101024B1B684A
:10BA480018600020704700BF041B002030B1044B71
:10BA58001B68DB68013303600020704709207047CA
:10BA6800041B002013B500230C460193D2B101A991
:10BA7800FFF764FF18B9019B591C02D1146002B08A
:10BA880010BD99B2611A002902DD0B441360F6E774
:10BA980002D113600720F2E71B0C1B0403F5803367
:10BAA8002344F3E70920EAE728B1044B1B681C3359
:10BAB8004362002070470920704700BF041B002024
:10BAC8001FB5044600B3002303A8039302F07CF9D2
:10BAD800104ABDF80C30126820469380E38200F0CB
:10BAE80056FA98B904F11803009321680123132228
:10BAF80002F08AF860B9204600F049FA003818BF09
:10BB08000120000104B010BD0920FBE71020F9E76F
:10BB18000E20F7E7041B0020F0B5054687B01C4649
:10BB28003BB32F4E3368DB68834257D894F8202004
:10BB3800002A14BF09220822834205D3204600F0B8
:10BB48005AFA70B110200AE0002301900093A3680C
:10BB580094F82810606AFFF796FE0028EED007B028
:10BB6800F0BD23792168B4F808C0A768043B9AB2ED
:10BB780009B90920F3E7B2F5807F2DD8ADF80EC0DA
:10BB88008DF817304FEA174C04F12C033F0E8DF84F
:10BB9800117000932F0C08234FF0490EADF80C00DC
:10BBA8008DF814708DF816002F0E0DEB0300CDF8EC
:10BBB80008E08DF810C0ADF812508DF8157002F03D
:10BBC80023F808B10E20CAE7204600F014FA00282E
:10BBD800B8D13368DD60C2E70D20C0E70620BEE7B4
:10BBE800041B00202DE9FF410A9D80460F4616469A
:10BBF8001C46002D5AD0002303A910460393FFF7D3
:10BC08009DFE18B1062004B0BDE8F081039B9C425C
:10BC180001D80133F6D1284600F05EF9002847D153
:10BC2800264B1A78424503D01A79424542D1012061
:10BC3800AA68BA4240D103EB8002EB6A92F801800D
:10BC48002979CDE900430439927828683B4689B2BE
:10BC5800FFF792FE0028D6D195F820300194002BEA
:10BC68004FF00103009314BF4246082295F82810AC
:10BC7800686A3B46FFF707FE0028C4D1013E032E41
:10BC8800C1D8DFE806F002070B0F0D4B1B681C61DB
:10BC98001C62B8E70A4B1B685C61F9E7084B1B6834
:10BCA8009C61F5E7064B1B68DC61ACE70920AAE755
:10BCB8000F20A8E70B20A6E70220A4E73401002004
:10BCC800041B00201FB50A460B2A4FF00001CDE9DE
:10BCD8000011CDE9021107D00C2A13D00A2A0FD07F
:10BCE8000A2005B05DF804FB012802D120238DF855
:10BCF8000030684602F011F8002818BF0E20F0E75F
:10BD08003023F4E70B21F4E738B5054602F000F8D4
:10BD1800044678B97DB9094B1B680B219878FFF761
:10BD2800D1FF38B90C21FFF7CDFF18B90A21FFF769
:10BD3800C9FF00B10E24204638BD00BF041B0020F7
:10BD48002DE9F04380468FB00C461746002A6BD089
:10BD5800002969D0002529461D2206A8059504F06A
:10BD6800A1FE8DF81350344D2B680DF114099E88EF
:10BD7800CDF804900DF1130302933B7900933B68CF
:10BD880032462146404601F0E4FF00284ED138688B
:10BD98003A79494602F050F9384600F04FF8002841
:10BDA80046D13C7AFA79BB79240444EA02241C433C
:10BDB8002B689A6894423DD99C609DF813000B212A
:10BDC800FFF780FF034658BB0C21FFF77BFF0346B4
:10BDD80030BB0A21FFF776FF034608BB7B7ABA7AA5
:10BDE800FF7A3F0447EA02271F433A463346214673
:10BDF8000920FFF725FD034690B933463A46214608
:10BE08000820FFF71DFD034650B92A689DF8131056
:10BE180091700021D1604FF0FF31C2E904119161A6
:10BE280018460FB0BDE8F0830923F9E70E23F7E7BA
:10BE38000F23F5E70323F3E7041B002010B504469E
:10BE4800002845D00168002942D011F8013B437110
:10BE58000322063002F0F0F82046032250F8091BAE
:10BE6800043102F0E9F82168CB79E3600A7A43EA01
:10BE78000223E3604A7A43EA0243E3608A7A43EAA8
:10BE88000263E360CB7A23740B7B63742379212BE1
:10BE98001AD110220D3104F1120002F0CDF81D2242
:10BEA8002168501C8B5C6362085C43EA0023901C89
:10BEB8006362085C033243EA004363628A5C43EAD4
:10BEC80002636362002010BD112B03DC0D22E7E73B
:10BED8000220F8E70120F6E710B50446002854D000
:10BEE8000168002951D00B7843714B7883608A78B8
:10BEF80043EA02238360CA7843EA024383600A79EB
:10BF080043EA026383604B7903738B79C381CA79EF
:10BF180043EA0223027BC38102F00F02083110308A
:10BF280002F08AF8237B002203F00F0384F8202014
:10BF380084F82820227903F10800111A04290DDD5C
:10BF480021680933043AD21A085C84F82000D2B276
:10BF5800606A84F82820194402F06EF82379226870
:10BF68001A44002012F8043CE36212F8031C43EA66
:10BF78000123E36212F8021C43EA0143E36212F868
:10BF8800012C43EA0263E36210BD0220FCE710B50E
:10BF9800044660B3036853B30279162A29D9427953
:10BFA8001A700146082251F8060B013002F04EF8CB
:10BFB8002146082251F80E0B093002F047F8236891
:10BFC800E28A5A74E38A22681B0A93742368A26976
:10BFD800DA74A36922681B0A13752368628B5A7581
:10BFE8002368E27E9A7517232371002010BD012073
:10BFF800FCE70220FAE738B50446002863D0016858
:10C00800002960D0037B90F8282003F00F03002A52
:10C0180057D10833207904321344984255D36379B1
:10C028000B702368A2685A70A36822681B0A937071
:10C0380023686289DA702368E27A1A712368227B9E
:10C048005A712368E2899A71E38922681B0A21469A
:10C05800D371227B51F8100B02F00F02083001F067
:10C06800EBFF237B94F8282003F00F0303F1080566
:10C078002AB1226894F82010515503F10905206867
:10C0880094F82820616A284401F0D6FF94F82830F3
:10C098002268E16A2B44D1545A1CE16A206892B2A2
:10C0A800090A81549A1C2168E08D92B28854DA1CDE
:10C0B800216894F82F0092B2043388542371002029
:10C0C80038BD0933A6E70120FAE70220F8E70000A7
:10C0D800024B1A8810431880704700BF081B0020C5
:10C0E80008B5074B1B883BB1FEF7B8F900280CBF11
:10C0F80000206FF0020008BD6FF00100FBE700BFF1
:10C10800081B002010B5034B00241C80FEF79CF987
:10C11800204610BD081B0020B0FA80F04009704787
:10C1280082B018B9084602B000F0CAB8002002B0C0
:10C13800704710B9084600F077B9704710B908463B
:10C1480000F08EB970470346084611460BB900F057
:10C15800E5B90020704710B9084600F071BD704776
:10C1680010B9084600F006BA0020704710B404461B
:10C17800084611461A46019B14B910BC00F018BABB
:10C1880010BC70470346084611460BB900F042BA86
:10C198000020704710B40446084611461A4614B9E0
:10C1A80010BC00F0AFBA002010BC704730B4054690
:10C1B800084611461A46DDE902341DB9029430BC1E
:10C1C80000F02EBB002030BC704710B9084600F0C4
:10C1D800DFBB0020704710B9084600F06FBD002093
:10C1E800704710B9084600F0EEBB0020704710B940
:10C1F800084600F0EBBB002070470346084611468E
:10C208000BB900F005BC0020704710B4044608467E
:10C2180011461A46019B14B910BC00F0FBBB09205B
:10C2280010BC704710B40446084611461A4614B9A3
:10C2380010BC00F063BDC8B210BC7047004870471E
:10C2480001000102064B10B51B6A0446984730B13D
:10C258000448054B204498428CBF0020012010BDA3
:10C268001816010840C220C980B92A00F0B5114B40
:10C2780085B00C4610491F56054601F049F80F4B8A
:10C28800E4B25E6A072D4FF00103CDE9024301468F
:10C298000AD105220023CDE900234FF47A727A43AC
:10C2A8001846B04705B0F0BD08220020CDE90020AF
:10C2B8003A46F5E7630F01083C0F01081816010814
:10C2C8001FB5002300930378013B372B21D8DFE803
:10C2D80003F01C242020201E202020204143454E0E
:10C2E8002055585B5E6164206C1E6E73787A20203E
:10C2F8007D81262020202020202020202020202072
:10C3080083858A2020838A208C90C3780BB10223EE
:10C318000093009805B05DF804FB8378F6E743784E
:10C328008DF8043005238DF805308378003B18BF5D
:10C3380001235B008DF8063010238DF80730304B51
:10C348001B6801A803F55872CDE9022300F0C0FF6D
:10C358000090DEE74023DBE72023D9E7827890F9D5
:10C36800013012B9274AD35CD2E7274AFBE7827823
:10C3780090F90130002AF8D1244AF4E740F6B8339E
:10C38800C6E74FF47A73C3E74FF4FA63C0E741F2A4
:10C398008833BDE741F27073BAE71D484FF47A71EC
:10C3A80001F02EFE00F5FA60D2E71A4BB0E7144B05
:10C3B8001B6803F55873ABE7114B1B6803F55B73F8
:10C3C800A6E71023A4E70E4B1B68A1E74FF08343B1
:10C3D80000939EE7104BFBE7104B99E740F21113CF
:10C3E800ADF8003095E7032392E790F901300C4A45
:10C3F800B9E70C4990F9010000F08AFFA8E700BFEF
:10C40800101B0020EB0F0108F30F0108FB0F0108B8
:10C4180018FCFFFF00EA06379A99094040F70937E8
:10C42800630F01083C0F010837B50B4B02781B68F6
:10C438000C2101FB02335B7A03EB4304074B1D68B5
:10C4480003690093C3684278816805EBC40000F073
:10C45800DFFC03B030BD00BF101B00200C1B002008
:10C4680070B586B0027B6423ADF80030012A4FF026
:10C478000003CDE90133CDE903338DF802308DF89F
:10C48800143030D0022A39D05ABB03684BB3436802
:10C498003BB31F4D80682B601E4B182269461860FD
:10C4A80001F0CAFD1C4B2C6893E807000C3384E8A4
:10C4B800070093E8070004F10C06032386E8070049
:10C4C800A4F86C33012204F55B7104F5587000F090
:10C4D80090FC2B684FF6B072A3F878230522C3F8B6
:10C4E8007C2306B070BD0A4908684360036100F503
:10C4F8005B7100F5587000F07CFCF2E7044B1B6898
:10C50800B3F86023B3F86C130A43A3F86023E8E791
:10C51800101B00200C1B0020880C010808B50346DE
:10C528000A2924D8DFE801F006232323230B161B4E
:10C5380023212100BDE808400068FFF783BE90F979
:10C5480000009978052271B900F013FC003818BF73
:10C55800012008BD052293F900000021F4E790F9B5
:10C5680000005978EEE70221EEE70722F3E7002002
:10C57800EFE7000010B504791CB1012C0BD00020A6
:10C5880010BD0A4B01681B68012203F5587000F0C2
:10C5980030FC0120F4E7054B01681B68224603F5CF
:10C5A8005B7000F026FC2046EAE700BF101B002065
:10C5B800F7B50528144D1C46A8BF052058700E462F
:10C5C8002946174600F0A4FE94F90130A070072B05
:10C5D80013D1322000F09CFD0C4BDB6D05469847CB
:10C5E80004F10C0208340346019200943A4631469D
:10C5F800284600F092FD03B0F0BD054A55F8231017
:10C60800D05C00F07DFDE7E73C0F01081816010833
:10C61800630F01082DE9F04F344F90F901607B68F2
:10C62800D0F804908BB00446884698470546002801
:10C6380059D1E37C73B92E4A2378126803EB43037C
:10C64800990002EB8303D3F80490B9F1000F01D1EC
:10C6580052F80190274B484613F906B0FB689847F3
:10C66800A37CD7F818A022890993072E28D1002384
:10C678000121CDE90223204A0693CDE90431CDE911
:10C6880007330521CDE900214FF47A7202FB0BF242
:10C698004CF250311846D047637C13B3174B995D61
:10C6A8007B6D0D31C9B228469847E07C3246494631
:10C6B80000F040FE88F8006001200BB0BDE8F08F64
:10C6C800002101250823CDE90013CDE90715CDE99F
:10C6D8000511CDE903110292A1782B465A46284646
:10C6E800D9E7074BDBE70020E7E700BF181601088A
:10C6F800101B0020630F010885450100FB0F01088E
:10C70800EB0F01082DE9F04F8DB090F90130DFF8FB
:10C71800FCA0DFF8FC90CDE90A123E4A12F903B0FA
:10C728000278DAF800300C2505FB02333A4A5B7AC6
:10C73800126803EB430302EBC303044693F90210A8
:10C7480090F9020000F0DFFD3449064694F9010033
:10C7580000F0DEFDA26861688046304600F005FD05
:10C768002178DAF80020D9F80C3069430746505888
:10C778009847D9F81C309C4694F901300025072BBE
:10C788004FF47A63CDE90753CDE905552DD101233F
:10C79800CDE903530523CDE901534FF47A7303FB25
:10C7A8000BF300933946434646F2A81228466746DB
:10C7B800B8472378DAF800200C214B4394F901108C
:10C7C800D05800F0D9FDA18994F90100FFF74EFD7A
:10C7D8000B9B217B1860D9F85430284698470A9B50
:10C7E80001201E700DB0BDE8F08F01200823CDE9AF
:10C7F8000350CDE901032A46CDF800B0654643460B
:10C808003946A84701200546D3E700BF101B002082
:10C8180018160108630F01080C1B00203C0F0108C3
:10C828002DE9F04F8FB0002405468A469146984678
:10C838000494ADF81440ADF8024007264FF0010B00
:10C848002B7AA34206D9686804A9204400F0F2FBB9
:10C8580000285ED102238DF8083002A86B7A8DF883
:10C868000A30FFF72DFDAB7A8DF81D309DF8113099
:10C878008DF81E309DF812308DF81F309DF810305D
:10C888008DF82030EB7A8DF821302B7B8DF8223013
:10C898006B7B8DF8233010238DF81C608DF82430C5
:10C8A8003A4E8DF82C000DF102030A9305238DF8FA
:10C8B8002D3033680C930723ADF834302B6806937A
:10C8C8000DF1120204AB0DF1110106A800F0CCFB2A
:10C8D800072805460BD130680C22002100F5587056
:10C8E80001F0BEFB3368BDF80220A3F860239DF871
:10C8F80011308AF800309DF8123089F800309DF820
:10C90800103088F80030189B28461C700FB0BDE81E
:10C91800F08F9DF81330BDF81470ADF80270204404
:10C92800C4B2F3B917B3194A0020116807260246A2
:10C938004FF00C0C062B1BD10CFB00FE51F80EE03F
:10C94800BEF1000F04D00BFA00F23A4397B201226D
:10C9580001301028EED1002A3FF472AFADF8027012
:10C968006EE75A1E042A01D9062BDCD0062667E793
:10C9780047FA00FE1EF0010FEAD00CFB00FE51F84A
:10C988000EE0BEF1000F08BF0626E1E7101B0020ED
:10C9980038B505464068FFF755FC0522841D00217F
:10C9A80095F90000E4B200F0E4F908B904F0FD04D8
:10C9B80095F901000722002100F0DBF908B904F01D
:10C9C800FB04204638BD00207047000010B50378EE
:10C9D8000F2B044618D84068FFF734FC22780B491F
:10C9E80002EB42020968831C01EB820051F8222005
:10C9F800DBB21AB903F0FD0358B210BD032B06BF12
:10CA0800626842600223F7E70020F6E7101B002067
:10CA1800022070472DE9F04FDFF838810446D8F836
:10CA2800000099B08946174600211E4601220323BB
:10CA380000F55870CDE90611CDE908118DF81410EC
:10CA48008DF81510ADF8163000F0B5F938B9D8F8EA
:10CA58000020B2F8603343F00303A2F86033D8F83B
:10CA68000020637A8DF8283002F55871CDE90B1251
:10CA7800394A94F9083012680D920DF116020F9296
:10CA88002268109262681192D4E90301A27A8DF8A3
:10CA9800482001228DF8492013AA82E803001025B6
:10CAA800227DE18A8DF8293018468DF85420ADF89A
:10CAB8003850FFF7DBFB0AAB17930DF115031690FF
:10CAC80000933146019705AB06AA10A800F0BCFBFD
:10CAD800064698BB9DF81410204F013901F090FAD2
:10CAE8001F4B1B690393C4B24FF00C0B04F1600396
:10CAF8006B44D8F8000013F848AC9DF814300BFBD1
:10CB08000AFC01343946B4FBF3F203FB1244D0F8B3
:10CB18007C33B0F9782350F80C00DDF80CC0E4B28F
:10CB2800E04728B189F800A0304619B0BDE8F08F79
:10CB3800013D15F0FF05D9D10D26F5E70C2801BFF9
:10CB4800D8F80020B2F8603343F00303A2F860334A
:10CB5800EAE700BF101B00200C1B0020400D03005B
:10CB680018160108F8B50679012E054601D80620E1
:10CB7800F8BD0F2E2BD80368187A40F3030005225E
:10CB8800002140B200F0F5F82B680446187A40F30B
:10CB980003100522002140B200F0EBF8A8B1B4FA66
:10CBA80084F4640929680B7A086843F3030243F3A1
:10CBB800031352B25BB29A42C8BF0124FFF742FB8B
:10CBC80048B9002CD3D10420D2E70124EAE7032096
:10CBD800CEE70520CCE7002CFBD10C4F29683B6839
:10CBE80006EB460003EB80000C2201F025FA3A68B8
:10CBF8000C2303FB062320465C72B2F86013012362
:10CC0800B3400B43A2F86033B2E700BF101B00200B
:10CC180010B4017801290ED9084B18680C234B432E
:10CC2800C4180022C250C4E9012200F5587010BC93
:10CC3800102200F0A7B8002010BC7047101B00207D
:10CC48002DE9F04186B050238DF81430037A102B6B
:10CC5800074630D14368DD7B6DBB0224A8466426B5
:10CC6800062C14D87A68535D03932A44517843EA12
:10CC780001230393927843EA02437343CDE90338CF
:10CC880063B968468DF80040FFF7C2FF0DE0CDF8A4
:10CC98000C808DF81480CDF81080F2E703AB01A862
:10CCA80001938DF80840FFF75DFF0134E4B2102CC2
:10CCB80005F10305D4D106B0BDE8F0811FB50268BF
:10CCC8000379116851B901A88DF80430FFF7A0FF66
:10CCD80078B9002040B205B05DF804FB02A80292C2
:10CCE8008DF80C30FFF73EFF0628F2D8024B185C8F
:10CCF800F0E70320EEE700BF5C0F0108C90020B988
:10CD0800034B0B449856C0B27047024BF9E700BF7B
:10CD18006B0F0108AB0F0108F0B59A42069D03DBC3
:10CD28009DF914309A4220DD0020F0BD03EB430347
:10CD380031F814C005EB830300264CFA06F7FF0709
:10CD480007D51F7A07F00F0E724502DBB2EB171FEB
:10CD58000DDD0136102E03F10C03EED10134E4B2DF
:10CD68002301DBB29842E1D8DEE70024F8E701208E
:10CD7800DBE7884204DB9042CCBF002001207047EB
:10CD88000020704710B51409B4EB111F03464FEA91
:10CD980011100ED391420CD202B201F00F0133F8F8
:10CDA8001240012000FA01F124EA010123F81210CF
:10CDB80010BD0020FCE7F0B528B100EB41050127C4
:10CDC8000020914200D3F0BD002435F802CB234661
:10CDD80007FA04F636EA0C0608BF013304F1010429
:10CDE80008BFDBB2102CF3D118440131C0B2C9B26C
:10CDF800E7E710B500B149B910BD31F8134020F884
:10CE080013400133DCB2A242F7D8F5E70023F9E773
:10CE180082B030B5048804936AB9B3F5616F18D34A
:10CE280049F6AF2542F21072AB4298BF4FF47A72BE
:10CE3800944238BF1446012C38BF01246143BDE831
:10CE48003040C3688B428CBF5B1A0023C36002B0BA
:10CE580070476422ECE700002DE9F04F91B01546C9
:10CE6800DDF86C8004939DF8683009930C460646FB
:10CE780003F0C2FB684ADFF8A4B10590A8F5F633C1
:10CE8800303BB3FBF2F3534303F5F63203F5A83313
:10CE980003F5C0730393182313FB0543303206923E
:10CEA800089300254FF0FF3A089BA34207D1002DB5
:10CEB80014BF50464FF0FF3011B0BDE8F08FBDF9F8
:10CEC8007030ADF82C300B99CDF86C804046CDF819
:10CED800288003F021FBB4F800906EB9B8F5616FB3
:10CEE8005BD349F6AF2242F21073904598BF4FF4D6
:10CEF8007A73994538BF99464B46012B38BF0123B1
:10CF08000793002E52D1B9F1640F48D1A0605F4653
:10CF1800A1680EA803F022FB0F9B0093DDE90A121B
:10CF28000E9B0CA803F079FA049B0C9A0BB9099B89
:10CF38002BB12369BB4202D1394B9A420DD9394BE7
:10CF4800E760984509D90023ADF83430069B0D9960
:10CF58000C93184603F0E0FAA060606800B9E76037
:10CF6800276126B103F052FBE3680344E360D4E988
:10CF780003329342059B1D996360079B88BFE2605B
:10CF88004B43E168994202D20498A8B9A6B101239B
:10CF98001D442375EDB2183486E76423A9E7B9F573
:10CFA8007A7F0ABF204F214FA060B1E7049B0BB9DD
:10CFB800C4F80CB05F46D0E700209342207506D82D
:10CFC8005B1A9A4505F1010528BF9A46EDB2002E75
:10CFD800E1D1B9F1640F164AADF8346019D049F6B9
:10CFE800B023B9F57A7F18BF1346904584BF039ADA
:10CFF8009B180C931C9B00930CAF97E806001B9B97
:10D00800384603F00AFA97E8030003F085FA8246E7
:10D01800C1E74FF46163E8E78051010040771B00E6
:10D028007F5101002FEC010080A81201002E93020D
:10D0380030EC01000378032B14D1437803F00F027E
:10D048001B098A704B7083788B80C27843EA02236D
:10D058008B800379C3F3021203F00F03CA700B70BD
:10D0680005207047002070472DE9F347984643791B
:10D07800057990F907609146044690F906208A469A
:10D0880083B190F9087075B30F2A12D194F9092069
:10D098000F2E1ED194F90A60072D24D1002F08BF46
:10D0A800012720E090F90B7090F9092090F90A60A7
:10D0B800E9E7A369019394F915300093216994F97C
:10D0C8001430207BFFF728FE0028E1D105F0FD058C
:10D0D800DEE794F91D30B3420FDC94F91C30B342FB
:10D0E800DADA05F0FB0528468AF8002089F800609E
:10D0F80088F8007002B0BDE8F0871E46CCE7000053
:10D10800024B03FA00F0B0FBF1F0704740420F0009
:10D118004FF4FA53B3FBF0F0704730B54FF47A751B
:10D128000C1F6A4300FB042252001EBF00F1FF34AB
:10D138001219B2FBF0F2914238BF1146039A1160FE
:10D14800820048431CBF013040084FF47A71121A1C
:10D1580001FB1323002BCABF03F2E73393FBF1F162
:10D16800B3FBF1F1049B196030BD38B5400014469B
:10D178000D46F4F74BFC01462846F4F795FB21468B
:10D18800F4F792FBF4F784FA03F0D2FCF4F760FBAF
:10D1980040B238BD2DE9F74F019300231F469C4646
:10D1A8001C01058A5FFA84FE04F0F004A54206D843
:10D1B800019B82F800C01F7003B0BDE8F08F0EEB32
:10D1C8004E054FEA4309AD000024466836F8096069
:10D1D8002641F60727D5866806EB050A765916B361
:10D1E800067836B9466926B136F809602641F60749
:10D1F80019D59AF8086090F901B046F303084FFA78
:10D2080088F8D8450FDC46F3031676B25E450ADB8C
:10D218009AF8096006EB4608C66806EBC806367D2C
:10D228004EB90137FFB20134102C05F10C05CCD1F1
:10D238000133DBB2B4E70CF101060EEB040801F888
:10D248000C805FFA86FCEEE72DE9FF47044640684C
:10D25800DDE90C671D468A46914603F0D7F9236835
:10D268001B1A3B604FF000080123337085F80080DB
:10D27800636813B12368834224D8CAF80080D4F8BD
:10D288001CC0A3699CF800E00393D4E9030101AB37
:10D2980083E80300237D0093DCF80C10237A627A7C
:10D2A8007046FFF7D9FD334638602A46E06949469B
:10D2B800FFF770FF2B782BB1C7F80080002004B06F
:10D2C800BDE8F0873378002B14BF0B200C20F6E75D
:10D2D80037B590F9002090F90250954204460FD0D6
:10D2E800013A52B295420BD0A368019394F90130E8
:10D2F80000936168E0782B46FFF70EFD0028EFD019
:10D30800104603B030BD8842B8BF084670470000D9
:10D3180051F82000054B984205D0054BC31A5842D6
:10D328005841400070470120704700BF90D003006B
:10D3380020A1070005281FB50ED80C4B53F8203044
:10D348000093CDE901120A4B01220021022002F0CC
:10D3580069FE05B05DF804FBCDE90012054B01221A
:10D368000021022002F05EFEF3E700BF7010010802
:10D37800031001082210010807B5054BCDE900018B
:10D3880001220021022002F04DFE03B05DF804FBEB
:10D398003E10010810B5102204460021F13000F0BB
:10D3A8005FFE0021C4F814112046F022BDE81040A9
:10D3B80000F056BE02460846102100F0A5B92DE936
:10D3C800F0430446D0F8140185B00E46154604F221
:10D3D800011988B3C0F110089045474628BF174681
:10D3E800BAB2484400F028FED4F814313B440F2B5D
:10D3F800C4F814312DD9A8452BD204F1F00304F553
:10D40800807113F8012F187C8B4282EA00021A708F
:10D41800F7D104F1F10810224146684600F00CFEED
:10D4280022466946684600F0E9F9102269464046F6
:10D4380000F002FE3E44ED1B04F5807804F1F1078C
:10D44800102D09D8AAB23146484600F0F5FDC4F8B7
:10D45800145105B0BDE8F08304F1F003711E13F810
:10D46800012F11F8010F434582EA00021A70F6D124
:10D4780010223946684600F0DFFD224669466846B4
:10D4880000F0BCF910226946384600F0D5FD103688
:10D49800103DD5E7F0B589B00C46102200210546AD
:10D4A800684600F0DDFD22466946684600F0A6F9A8
:10D4B8009DF90030002B6A464FF0000143DA1378DB
:10D4C80012F8010F01315B0043EAD0130F2902F86B
:10D4D800013CF4D19DF80F305B0083F08703D4F84A
:10D4E8001401DBB210288DF80F303BD104F580739E
:10D4F800694604F5887013F8016F11F8012B9842FA
:10D5080082EA06021A70F6D104F1F00304F580717C
:10D5180013F8012F187C8B4282EA00021A70F7D1A7
:10D5280010220DEB020004F1F10100F085FD224606
:10D53800294604A800F062F910220021684600F08C
:10D548008FFD09B0F0BD137812F8010F01315B00AF
:10D5580043EAD0130F2902F8013CF4D19DF80F30AB
:10D568005B00BCE79DF90030002B6A464FF00001D4
:10D5780037DA137812F8016F01315B0043EAD613EA
:10D588000F2902F8013CF4D19DF80F305B0083F0BD
:10D598008703471CDBB28DF80F30102F04EB000314
:10D5A800C0F10F064FF0800288BF002600F5817099
:10D5B80083F801210021324620443E4403F072FAE8
:10D5C800C4F8146104F58073694604F5887013F88B
:10D5D800016F11F8012B984282EA06021A70F6D1FF
:10D5E80092E7137812F8016F01315B0043EAD61312
:10D5F8000F2902F8013CF4D19DF80F305B00C8E711
:10D608000A780378534003704A784378534043704C
:10D618008A78837853408370CA78C3785340C3703C
:10D628000A790379534003714A7943795340437126
:10D638008A79837953408371CA79C3795340C37116
:10D648000A7A037A534003724A7A437A5340437200
:10D658008A7A837A53408372CA7AC37A5340C372F0
:10D668000A7B037B534003734A7B437B53404373DA
:10D678008A7B837B53408373CA7BC37B5340C373CA
:10D68800704710B50B7814786340037054784B7862
:10D698006340437094788B7863408370D478CB78F8
:10D6A8006340C37014790B796340037154794B79E3
:10D6B8006340437194798B7963408371D479CB79D2
:10D6C8006340C371147A0B7A63400372547A4B7ABD
:10D6D800634043728B7A947A63408372D47ACB7AAC
:10D6E8006340C372147B0B7B63400373547B4B7B97
:10D6F80063404373947B8B7B63408373CB7BD27B88
:10D708005340C37310BD0000A1F11003DBB2102B0E
:10D718002DE9F04704D8374C24FA03F3DB0705D486
:10D72800002382F8F030FF20BDE8F087531E44182C
:10D73800A0424ED101F11C039B005FFA83F9C3F3A9
:10D748000313013B2C4D82F8F03001240B46D61808
:10D75800B3FBF1F001FB103010F0FF0016F804AC39
:10D7680016F803EC16F802CC16F8017C36D115F839
:10D778000E8015F80CE015F807C015F80A70E009D6
:10D7880000EB400084EA080800EBC0006400C0B267
:10D79800E4B24440C246581AC0B212F800808AEA7D
:10D7A800080A02F803A01044043390F801808EEAB6
:10D7B800080E86F801E090F802E08CEA0E0C86F874
:10D7C80002C0C078DBB247409945F770BFD8002047
:10D7D800AAE710F8015B03F8015FA9E71829DAD96D
:10D7E800102801BF15F80AA015F80EE015F80CC0AE
:10D7F800EF5DD0E701010100881201082DE9F04F23
:10D80800A3B092F8F0301D911B920193002B00F009
:10D81800538101461EA8FFF734FF1B9BA74CA84D58
:10D82800A84E10330293002303939DF87C000490C4
:10D838009DF886000590205C06909DF87B00079077
:10D84800205C089004989DF881C0205C099014F829
:10D858000C000A909DF880000B909DF885009DF8BB
:10D8680078809DF87DE09DF882A09DF887900C90C7
:10D878009DF87A00029B1C9314F80A2014F80930CA
:10D8880014F8081014F80E700D90205C0E909DF896
:10D898007F000F90205C10900B98205C11900C98E2
:10D8A800205C12909DF8840013909DF879001490E4
:10D8B8009DF87E001590205C16909DF883001790C7
:10D8C800205C18901398205C19901498205C1A908A
:10D8D8000398013003900298DDF804B010300290EC
:10D8E8009DF80C00834536D88DF878108DF87A208D
:10D8F80009990E9A8DF87C108DF882201199069A54
:10D908008DF880108DF87E201999169A8DF884105C
:10D918008DF886200A99189A8DF87D108DF8872041
:10D928001299109A8DF87B301B9B8DF881108DF819
:10D9380083201A99089A1D988DF885108DF87F20F4
:10D948001EA903EB0B128DF87970FFF79AFE0020E1
:10D9580023B0BDE8F08F15F808B082EA03008BEA1F
:10D96800000016F80EB080EA0B008DF8780015F864
:10D978000E004B40434016F80A0043408DF87930BA
:10D9880081EA070315F80A10594016F8093059407A
:10D9980016F808308DF87A107A40534015F80920A7
:10D9A80053408DF87B30089A069B5340049AAA5C32
:10D9B800534016F80C2053408DF87C30DDE90832CE
:10D9C8005A4015F80C305340059AB25C53408DF814
:10D9D8007D30DDE909325A40059BEB5C5340079ADC
:10D9E800B25C53408DF87E30069B0A9A5340049AE5
:10D9F800B25C5A40079BEB5C5A408DF87F200E9B27
:10DA0800109A53400B9AAA5C53400C9AB25C53404C
:10DA18008DF88030DDE910325A400C9BEB5C5340A6
:10DA28000D9AB25C53408DF88130DDE911325A40CD
:10DA38000D9BEB5C53400F9AB25C53408DF88230DB
:10DA4800129A0E9B53400B9AB25C5A400F9BEB5CA8
:10DA58001C995A408DF88320169B189A5340139AA4
:10DA6800AA5C5340149AB25C53408DF88430DDE9C7
:10DA780018325A40149BEB5C5340159AB25C5340E1
:10DA88008DF88530DDE919325A40159BEB5C53401F
:10DA9800179AB25C53408DF886301A9A169B5340F9
:10DAA800139AB25C5340179AAA5C1EA853408DF88B
:10DAB8008730FFF7A5FDB8E6FF2049E7881201087F
:10DAC800881001088811010808B538B1044A0549C9
:10DAD8001060D82200F0B0FA002008BD0220FCE750
:10DAE800141B0020B81701080A4B1A6870B50023E8
:10DAF80002F1180503EB03142E5D864204D1183495
:10DB080022440A60002070BD01330B2BF2D10320A0
:10DB1800F9E700BF141B00202DE9F041CCB0064600
:10DB2800DDF8488117461C460D4631B3B8F1000FA1
:10DB380023D006A8FFF72EFC204601A9FFF7D4FF43
:10DB48000446B0B9019906A80131FFF733FC26B1A4
:10DB58001022314606A8FFF732FC3A46294606A8A5
:10DB6800FFF72DFC06A902A8FFF794FC029BC8F852
:10DB7800003020464CB0BDE8F0810224F9E70000EF
:10DB880030B595B013A90446FFF7AEFF002830D191
:10DB98001B490C2303FB00F2555CA5422BD1139BB8
:10DBA800187C1090D87B0F90987B0E90587B0D9026
:10DBB800187B0C90D87A0B90987A0A90587A09902A
:10DBC800187A0890D879079098790690587905902E
:10DBD80018790490D8780390987802900A445B7872
:10DBE8000193936800930022064B1146022002F02D
:10DBF80019FA15B030BD01300B28CBD1F9E700BFB9
:10DC080000150108881301080B2B10B402D810BCAA
:10DC1800FFF782BF032010BC704730B50D4685B0B2
:10DC28001446014668B103AA002000922A460390D0
:10DC3800FFF772FF18B90398001B18BF012005B041
:10DC480030BD0220FBE72DE9F0430D46BFB0144676
:10DC58009946804620B31BB311F00F0122D1F02260
:10DC680001A800F0FDF920466946FFF73DFF04468C
:10DC780048B9009801AA10210130FFF745FD2E464A
:10DC8800AF1BFFB21EB920463FB0BDE8F08301AA22
:10DC980009EB070108EB0700FFF7B0FD103EEFE7BF
:10DCA8000224F0E70524EEE7F0B5184E3468024682
:10DCB80085B00846002304F1180103EB03154F5DF6
:10DCC80097421ED10D2A05F1190513D10023CDE97C
:10DCD8000033CDE902330C2210216B46FFF7B3FF66
:10DCE8000446306810226946284400F0A5F9204609
:10DCF80005B0F0BD01461022601900F09DF900241E
:10DD0800F5E701330B2BD8D10324F0E7141B0020CF
:10DD180009B1FFF7C9BF022070471FB51446A0B16B
:10DD28000C2A01D10B2912D10023CDE90033CDE90A
:10DD380002330A466B461021FFF785FF18B969467A
:10DD48002046FFF7B1FF04B010BD0220FBE7032017
:10DD5800F9E7F8B51E46DDE907479DF818505BB3AB
:10DD680054B34FB3212D29D819462A46204600F02E
:10DD780063F90122631C691EB018FFF764FFF8B944
:10DD8800E37ADB093B70EBB96319204613F8012CE1
:10DD980013F8021C120642EA014213F8041C0A4353
:10DDA80013F8031C012342EA0122291FFFF735FF5C
:10DDB800003818BF0120F8BD0220FCE70520FAE76B
:10DDC8000720F8E70420F6E710B5044628B1044B0D
:10DDD8005B6998472060002010BD0220FCE700BF67
:10DDE8001816010808B5014630B1044B0822186816
:10DDF80000F022F9002008BD0220FCE7141B0020D7
:10DE080008B530B1044B0822196800F015F9002054
:10DE180008BD0220FCE700BF141B00207FB5124E8E
:10DE28000023044602A801930D46FFF7E9FF336873
:10DE38005B6901936CB102AA082312F8011B41B96E
:10DE4800013B13F0FF03F8D102A8A04702A8FFF78F
:10DE5800C9FF35B1019B23B901A8A8473368019AC6
:10DE68005A61002004B070BD141B002008B501469B
:10DE780038B1054B18680822104400F0DDF800207E
:10DE880008BD0220FCE700BF141B002008B538B10C
:10DE9800044B19680822114400F0CEF8002008BD90
:10DEA8000220FCE7141B0020034B1B6802280CBF50
:10DEB8001961596100207047141B002041B1054BBE
:10DEC8001B6802280CBF1B695B690B600020704748
:10DED80002207047141B002030B58FB0002405467F
:10DEE8000CA80994FFF78CFF9DF8373007939DF82D
:10DEF800363006939DF8353005939DF834300493F9
:10DF08009DF8333003939DF8323002939DF83130F9
:10DF180001939DF830300093224621461E4B022083
:10DF280002F080F80AA8FFF7B1FF9DF82F30079399
:10DF38009DF82E3006939DF82D3005939DF82C30D2
:10DF480004939DF82B3003939DF82A3002939DF893
:10DF5800293001939DF82830009322460F4B214623
:10DF6800022002F05FF809A92846FFF7A7FF9DF8ED
:10DF7800243003939DF8253002939DF826300193B1
:10DF88009DF8273000932246054B2146022002F0D7
:10DF980049F80FB030BD00BFE4130108221401088E
:10DFA8006014010808B50020FFF7EAFD0120FFF71B
:10DFB800E7FD0920FFF7E4FD0820FFF7E1FD002059
:10DFC800FFF78AFF002008BD10B504460B20FFF7B5
:10DFD800D7FD0C20FFF7D4FD0920FFF7D1FD08205D
:10DFE800FFF7CEFD0A20FFF7CBFD2046FFF774FFB1
:10DFF800002010BD014B1860704700BF3C01002095
:10E008000B4A30B514680B4D43F2390305FB043352
:10E018001360091A6FF00042B3FBF2F2C2EBC2724E
:10E0280001319B1A93FBF1F201FB1233184430BD06
:10E038003C0100206D4EC64101380A44914200D18E
:10E04800704711F8013B00F8013FF7E710440A4414
:10E05800914200D1704711F8013B00F8013DF7E704
:10E0680002F020BD30B530B10A4D01444FF0FF3306
:10E07800814201D1D84330BD10F8012B534008220A
:10E0880043F30004013A2C4092B284EA5303002A75
:10E09800F6D1EDE72083B8ED01207047054B4FF42A
:10E0A80000529A62044B1B6813B15B6803B11847AE
:10E0B800704700BF00040048181C0020054B4FF4AF
:10E0C80080529A62044B1B6813B1DB6803B118478E
:10E0D800704700BF00040048181C0020012070474A
:10E0E8000120704701F048B901F036B910B501F0C8
:10E0F80019FE0E21044640F61F1001F02DF92046A6
:10E10800012101F0F9FDBDE8104001F0D7BA000087
:10E1180070B50C4E01EB40030D46B3654FF6FF7129
:10E12800002304461A46084601F05EFB96F856009E
:10E13800002101F0E1FD29462046BDE8704001F0CC
:10E1480095BA00BF341C002010B5044601F0AAFEA1
:10E1580001281CD101F0AEFE34B11248214602F06C
:10E1680017FB104802F0DAFA0F4C104B00214FF45D
:10E178008052A1659A6194F8560001F0BDFD63785C
:10E188006BB16FF07F40BDE8104001F053BA002337
:10E1980040F262211A46084601F026FBDCE7A06837
:10E1A8008001F0E71C1C0020341C002000040048FB
:10E1B800002001F0BFB9000008B501F0C7F8043825
:10E1C800C0B2032896BF024B0020185C08BD00BFF0
:10E1D8001416010808B501F0BAFD033008BD01F0B6
:10E1E80049B901F009B908B501F000FD00B208BD50
:10E1F80038B50D46144601F05DFB284601F092FD46
:10E208000E21054640F61F1001F0A6F82846012108
:10E21800074D01F071FD01F051FA4FF47A71614335
:10E22800284602F0B5FA2846BDE8384002F076BA2A
:10E23800901C002001F03EBB08B5084B002193F864
:10E24800560001F059FD00234FF4C0711A460846E4
:10E2580001F0CAFABDE8084001F024BA341C0020D5
:10E2680010B5044601F01EFE01281CD101F022FE63
:10E2780034B11248214602F08BFA104802F04EFAE7
:10E288000F4C104B00214FF48052A1659A6194F80D
:10E29800560001F031FD63786BB16FF07F40BDE847
:10E2A800104001F07DB9002340F262211A46084669
:10E2B80001F09AFADCE7A0688001F0E71C1C002056
:10E2C800341C00200004004808B54FF0040001F099
:10E2D80017F9BDE808400220F4F732BB08B500235F
:10E2E8001A461946184601F07FFABDE8084001F0C1
:10E2F8006DB900001D4B73B51D4D186000241D48F5
:10E308006C70C5E90144AC6501F098FAAC8101F084
:10E3180003FA2146204601F04BFC21460422012045
:10E3280001F0FCFA144E154D4FF6FF7123462246B4
:10E33800084601F059FAFFF7C7FF2246104B009430
:10E348004FF0FF31304602F03DF90E4B0094224663
:10E358004FF0FF31284602F035F9304602F090F9C7
:10E36800284602B0BDE8704002F08AB9181C0020A7
:10E37800341C002045F30008901C00201C1C0020C1
:10E38800A5E00008C5E000080128084805D1084BA9
:10E39800C17719700E3001F0A7BB437D012B03D163
:10E3A800034B81751970F5E7704700BF341C0020D6
:10E3B800400100200D4B10B5044618735873012016
:10E3C80000F016F85CB134214FF4E86000F0C4FFA7
:10E3D8004421BDE8104040F2417000F0BDBF142157
:10E3E8004FF4E86000F0B8FF2421F2E7341C002065
:10E3F80038B5114C0546207001F061FD052D04D893
:10E40800DFE805F0090B03171709032001F070FA7C
:10E418000023637338BD0020F8E7012001F068FA93
:10E42800207B637B8342F5D06073BDE83840FFF7FB
:10E43800C1BF0220EAE700BF341C00202DE9F043E9
:10E448001E4687B000230546CDE901330C46174622
:10E4580001F027FD032D61D8DFE815F07B00C3002C
:10E468000E010400A27C082A04D94FF0FF3007B03F
:10E47800BDE8F083A16801A801F0DCFE216800294D
:10E48800F3D042F210729142E37C864D51D80322B8
:10E49800AA7385F83820E96385F844304FF00208FC
:10E4A8006368A17DDB002B820423AB74A37CDB00B3
:10E4B800EB7402294FF000032B75637D02D0227D97
:10E4C800022A42D103F10F02D2B2012A01D9012B4B
:10E4D800CBD1754B754A196803944FF0010903A80D
:10E4E8008DF8149001F0DAFC0028BED1287685F862
:10E4F80017906875FFF75CFE4046FFF779FF6C4898
:10E5080001F086FA6B4801F0EFFA01A800F084FFE9
:10E51800208A00F055FFA08900F09AFF384601F0E4
:10E5280001FC604C84F8560001F0C0FC66600020D5
:10E538009DE74FF00008E963890885F80E8085F8A3
:10E54800388085F844302964AAE7EB7529766A751E
:10E55800D0E72368002B88D0A27C082A85D8514DA3
:10E56800A16801A801F066FE002385F8383022680A
:10E57800EA63E27C85F84420A269AB732A64626886
:10E58800A17DD2002A820422AA74A27C2B75D20013
:10E598000229637DEA7402D0227D022A1DD103F18B
:10E5A8000F02D2B2012A02D9012B7FF45EAF3E4B93
:10E5B8003E4A196803944FF0010803A88DF81480A7
:10E5C80001F06CFC00287FF450AF287685F817809E
:10E5D8006875FFF7EDFD00208FE7EB7529766A7502
:10E5E800F7E7304D012185F83810227885F850205A
:10E5F800637885F85130A37885F85230E3788B42F8
:10E6080002D0022B03D03BB985F8533004E00B3A13
:10E61800012A29D885F853104FF0010885F80E8093
:10E62800A388AB83A379AB77E37985F82030237A85
:10E6380085F82130FFF7BCFD4046FFF7D9FE1C489E
:10E6480001F0E6F91B4801F04FFA95F85130062B16
:10E6580040F689000AD100F08FFE00F0FB0140F679
:10E66800890000F079FE59E70023CDE700F084FE29
:10E6780040F00401C9B2F2E72368013BB3F57A7FA1
:10E68800BFF4F3AE0320FFF7B3FE0648022380F879
:10E69800383023688364162380F84C30383001F012
:10E6A800B7F93BE7341C0020181C0020901C002000
:10E6B8006C1C0020421C00202DE9F041002686B089
:10E6C8001F461446CDE9016680460D4601F0E9FB78
:10E6D800B442764C16BF0123334637466370B8F10F
:10E6E800000F06D0B8F1010F7CD0002006B0BDE8BD
:10E6F800F081AB68002B00F0D680EB68002B00F0AF
:10E70800D280AA7F082A00F2CE80296901A801F0E8
:10E7180091FD2868003818BF012000F0D9FF84F85F
:10E728003880AB68E36395F8203084F84430686833
:10E7380001F05AFB84F80E8084F84500EB68DB0092
:10E748002382EB7FA374AB7FDB00E37495F8213061
:10E75800237595F82230002B3ED12A7D95F8241098
:10E76800A275022995F8232001D0022B36D102F197
:10E778000F03DBB2012B02D9012A40F09480002359
:10E788008DF814304A4B4B4A1968049503A801F0D8
:10E7980085FB002840F0878001232076E3756075AB
:10E7A800FFF706FD0020FFF723FE434801F030F98C
:10E7B800424801F099F901A800F02EFEA88B00F05C
:10E7C800FFFD288B00F044FE4FF4FA53AA687B4300
:10E7D800B3FBF2F3A36088E7FF22BFE7E275217677
:10E7E8006375DDE72B8E002B5DD095F83230A86A73
:10E7F800012B0CBF95F814804FF0FF08003818BFA4
:10E80800012000F065FFF8B200F06EFF012184F8E6
:10E81800381095F82C2084F8502095F82D3084F87D
:10E82800513095F82E3084F8523095F82F308B42BD
:10E8380002D0022B03D03BB984F8533004E00B3AE2
:10E84800012A28D884F853102B8EA38395F83230E8
:10E85800A377AB8E23840126A67384F81F80FFF765
:10E86800A7FC3046FFF7C4FD134801F0D1F8134860
:10E8780001F03AF994F82130B34240F236700CD1E5
:10E8880000F07AFD00F0FB0140F2367000F064FD04
:10E898004FF6FF739EE70023CEE700F06DFD40F0D2
:10E8A8000401C9B2F0E74FF0FF301FE7341C002025
:10E8B800181C00201C1C00206C1C0020421C00207E
:10E8C8002DE9F04F85B082460E9DBDF840B09DF809
:10E8D80044709DF84890019288461E4601F0E1FA7E
:10E8E800BAF1010F524C54D0BAF1040F00F09180E4
:10E8F800BAF1000F3AD10B22304684F8442084F84C
:10E9080038A0E56301F070FA019B23644FEACB035A
:10E91800B9F1000F238241F60403638214BFF22386
:10E928000123E37587F001070123237684F8450066
:10E9380084F80EA084F814A06775FFF739FC5046D8
:10E94800FFF756FD04F1380001F062F804F10E00FB
:10E9580001F0CAF8374A1068516802AB03C302A82D
:10E9680000F05AFD40F2FF1000F02AFD404601F089
:10E97800D9F90E2184F8560040F61F1000F0ECFC7F
:10E9880094F8560001F092FA169B636005B0BDE852
:10E99800F08F294984F838A0EAB2895D84F85020BC
:10E9A80076BB0B3D012D8CBF00250125053A012AB8
:10E9B80004D8BBF10C0F38BF4FF00C0B1F4B9DF860
:10E9C8003C201B7884F85350E37701259DF8543098
:10E9D80084F8511084F8522084F82130A573A4F8E3
:10E9E8001CB0A77784F82090FFF7E2FB2846FFF7D2
:10E9F800FFFC134801F00CF8124801F075F8B5E770
:10EA0800012E04D1A5F10C035D425D41CEE700253E
:10EA1800CCE75046FFF7ECFC022384F8383004F1C9
:10EA280038001623A56484F84C3000F0F1FF9DE708
:10EA3800341C0020A00C0108E21501084001002048
:10EA48006C1C0020421C00202DE9F04F87B0DFF835
:10EA5800B4B29DF864A09DF84C90029314469DF8BA
:10EA680054309DF85020BDF84880039205468BF835
:10EA780001A0BDF8446001930F4601F012FABAF103
:10EA8800000F18BF4FF00008DFF87CA2039AB9F115
:10EA9800000F08BFFF22012D8AF8002000F0C8806F
:10EAA800052D48D0002D40F0C080284600F010FE0B
:10EAB8000B2238468BF844208BF83850CBF83C4072
:10EAC80001F092F9019B8BF8450041F60402002BF6
:10EAD800ABF812209AF800208BF8162014BFF22207
:10EAE80001228BF81720F600012289F001098BF822
:10EAF80018208BF80E50ABF810608BF814508BF878
:10EB08001590FFF755FB2846FFF772FC0BF138000C
:10EB180000F07EFF0BF10E0000F0E6FF7B4908686D
:10EB2800496804AA03C204A800F076FC40F2FF106A
:10EB380000F046FC71E0012000F0CAFD09224FF008
:10EB480000098BF8442038464FF44872CBF840202F
:10EB58008BF83890CBF83C4001F046F94FF48052DE
:10EB6800ABF812209AF800208BF845008BF8162095
:10EB780028460122F6008BF817208BF80E90ABF888
:10EB88001060ABF814908BF81890FFF731FC0BF17C
:10EB9800380000F03DFF0BF10E0000F0A5FF5B49C7
:10EBA8008868C96804AA03C204A800F035FC40F2CA
:10EBB800FF1000F005FC40F6B80000F0DDFB00F0A7
:10EBC800EF0140F6B80000F0C7FB042140F6B90099
:10EBD80000F0C2FB40F69B0000F0CEFB00F0E30122
:10EBE80041F0080140F69B0000F0B6FB40F2D1600E
:10EBF80000F0C2FB40F01801C9B240F2D16000F049
:10EC0800ABFB40F2AC6000F0B7FB00F08F0141F0C5
:10EC1800500140F2AC6000F09FFB4FF4FA5202FB47
:10EC280008F2B2FBF4F2CBF8082007B0BDE8F08F89
:10EC3800002000F04DFD36498BF83850E2B2C95D2E
:10EC48008BF85020002F4DD10B3C012C8CBF002499
:10EC58000124053A012A02D80C2E38BF0C26029B43
:10EC68009AF800208BF852308BF85340019B8BF8B0
:10EC78001F2001249DF860208BF821208BF851106B
:10EC88008BF820308BF80E40ABF81C608BF81E9088
:10EC9800FFF78EFA2046FFF7ABFB1E4800F0B8FEE0
:10ECA8001D4800F021FF5FFA88F000F01DFD40F6D6
:10ECB800A30000F061FB00EA040140F6A30000F0A5
:10ECC8004BFB9BF82120A24240F2367013D100F092
:10ECD80053FB00F0FB0140F2367000F03DFB4FF6AD
:10ECE800FF72A0E7012F04D1A4F10C035C425C4140
:10ECF800AFE70024ADE700F03FFB40F00401C9B2E4
:10ED0800E9E700BF341C002040010020A00C0108E6
:10ED1800E21501086C1C0020421C0020F0B58BB0E5
:10ED28000D46044617461E46FFF742FA0020FFF735
:10ED38005FFB204600F0BEFD00240123CDE9084317
:10ED480003234FF4167229462046CDE90644CDE93F
:10ED58000444CDE90244CDE900532346FFF774FE8D
:10ED68002046FFF77DFAFFF735FAF3F7E9FD01F0E2
:10ED780043FC0446204601F049FCB04205D3012477
:10ED8800FFF716FA20460BB0F0BD00F02FFF00B2D7
:10ED98008742EFDA0024F3E7F7B500230C4640F288
:10EDA80001211A460646084600F01EFD644B654DD3
:10EDB8004FF400529A6195F85600012100F09CFF2B
:10EDC8002B78012B40F6890013D195F85130062B8A
:10EDD8000FD100F0D1FA00F0FB0140F6890000F0F5
:10EDE800BBFA2B78042B6CD8DFE803F0524B527F28
:10EDF800090000F0C1FA40F00401C9B2EDE7524A37
:10EE0800731E1046C6F101074FF0000CF9188C422A
:10EE18006FDC0022E7001346BA4271D19A0142EA38
:10EE2800C3125B0183F020031343661C0355F6B23B
:10EE380002234648AB73AE7600F056FE0021F1205F
:10EE480000F08AFA0021F02000F086FAAB6C642BFF
:10EE580070D17021F32000F07FFA1D21F22000F01C
:10EE68007BFAE1008C1CF420090A00F075FA04F022
:10EE7800FE01F52000F070FA33486FF07F4231460A
:10EE88001DE0EC77314800F02FFE0022214615E006
:10EE980001F008F80128074625D121460DF107029F
:10EEA800304601F004F80446A0B99DF80730274819
:10EEB800AB7500F019FE9DF807102246304600F0A9
:10EEC80065FB6968224801F063FC214801F026FCD3
:10EED800002006E01F4B3A460021022001F0A2F86C
:10EEE800032003B0F0BDAC75CCE70223AB73AC765E
:10EEF800C8E713F8011FC943197002F801CB85E769
:10EF0800D1106FEA020C715C0CF0070C013241FA67
:10EF18000CF101F001014FEAE20C4B40D14310F82B
:10EF28000CE001F0070103FA01F141EA0E0100F8D3
:10EF38000C1071E7E121F32000F00EFA04218DE7AF
:10EF480000040048341C0020181B0020421C00202C
:10EF5800901C002084150108F0B5BDF814409DF8F8
:10EF680018709DF81CE09DF8205040B1012814D07D
:10EF78000122002398180138B0FBF2F0F0BD87F0A9
:10EF88000107E30003EBC70318330EEB450503EB5A
:10EF9800C5034FF47A714B43ECE7501F012803F186
:10EFA800040302D80C2C38BF0C24D1B9A2F10B0CE5
:10EFB800BCF1010F8CBF4FF0000C4FF0010C280181
:10EFC800002F00EBCE0014BF00251425A0EB820013
:10EFD800062A4FEA82062844A2F102070DD83546D0
:10EFE80010E0012906D1A2F10C00D0F1000C4CEB85
:10EFF800000CE4E74FF0000CE1E70830BCF1000F2B
:10F00800EDD0BD000028ACBF2E182E1C701E90FB42
:10F01800F5F003FB0044094B062A5A5C8CBF0C34FC
:10F028000E340A2A09D8A30001334FF47A71BB4081
:10F038004B43034951F822209CE7FFDEE215010803
:10F04800E815010808B5094B012193F8560000F0AE
:10F0580053FE4FF4D7602D2100F07EF900F033FB0A
:10F06800BDE80840024800F07BBA00BF341C00200D
:10F07800FFFF0F0073B5A44CB4F854300025202BC3
:10F088008DF80350019500F01B8114D8082B0DD87A
:10F098007BB1013B072B0CD8DFE813F042005B0083
:10F0A8000B00CD000B000B000B00FD00102B00F037
:10F0B800008102B070BDB3F5807F00F0988011D850
:10F0C800402B00F01081802BF3D1284600F032FA53
:10F0D8008E4B1B68002BECD09B69002BE9D028468F
:10F0E8009847E6E7B3F5007FE3D1894B012229462B
:10F0F800022000F097FF00F029F9042840F08580ED
:10F10800844B85484FF400529A6201F0B9FA2846B8
:10F1180000F010FA7D4B1B68002BCAD05B6814E026
:10F128007C4B7D484FF400529A6201F0A9FA002006
:10F1380000F000FA00F0B8FE012801D100F0BDFE91
:10F14800724B1B68002BB4D01B68002BB1D09847BA
:10F15800AFE7704B71484FF480529A6201F090FA11
:10F16800657895B9284600F0E5F9294640F6021079
:10F1780000F0F2F840F6441000F0FEF840F002010A
:10F18800C9B240F6441000F0E7F8FF220DF1030180
:10F1980063485E4D00F05AFD624800F071FD2B682F
:10F1A800002B86D09E68002E83D094F82430012B43
:10F1B80008D194F9313094F930209DF8031058485B
:10F1C800B04776E7E06B01A900F022FE019B9DF8AD
:10F1D800031053484FF47A7203F5FA7393FBF2F372
:10F1E8002A685BB2956894F92920A84761E7284600
:10F1F80000F0A0F9454B1B68002B3FF45AAF9B6900
:10F20800002B3FF456AF01206AE700F09FF805286D
:10F218007FF44FAF3F4B41484FF480529A6201F060
:10F228002FFA284600F086F9384B1B68002B3FF46C
:10F2380040AFDB6889E700213B4B0122022000F048
:10F24800F1FEA16D00293FF434AFC1F3074140F648
:10F25800031000F081F894F8591040F6041000F0FB
:10F268007BF894F8581040F6051000F075F840F651
:10F27800021000F081F840F00101C9B240F6021016
:10F2880000F06AF8002340F262211A460846A36596
:10F2980000F0AAFA0DE7254B01220021022000F018
:10F2A800C1FE00F0FFFD01287FF403AF00F006FE69
:10F2B800FFE61F4B01220021022000F0B3FEF8E612
:10F2C800164801F0DDF9607808B900F033F90F4B02
:10F2D8001B68002B3FF4EDAEDB68002B3FF4E9AE72
:10F2E8009847144BE6E7144B01222946022000F008
:10F2F80099FE607808B900F01DF9044B1B68002BD3
:10F308003FF4D7AE1B6920E7341C0020181C0020EE
:10F318009915010800040048901C00201C1C0020BE
:10F32800181B0020581C0020AD150108B61501084F
:10F33800C0150108C9150108D2150108024BA3F828
:10F348005400FFF797BE00BF341C0020014B18780B
:10F35800704700BFAE1C002007B501238DF80710C9
:10F368000DF1070201460348F7F774F803B05DF89A
:10F3780004FB00BF3802002007B5012301460DF148
:10F3880007020448F7F79FF89DF8070003B05DF8F7
:10F3980004FB00BF3802002010B50446F4F7F8FC5F
:10F3A80001280CD140F62310FFF7E6FF00F0F90121
:10F3B800214340F62310BDE81040FFF7CDBF10BD34
:10F3C80010B50C4B1B7804469BB94FF4D760FFF778
:10F3D800D3FFC4F3002100F0FE0001434FF4D760CF
:10F3E800FFF7BAFFE1B240F2B960BDE81040FFF79D
:10F3F800B3BF10BDAF1C002010B51346EFF3108447
:10F4080072B60A4601460348F7F724F884F31088D1
:10F4180010BD00BF3802002008B5014608224FF48D
:10F42800D860FFF7E9FF002008BD000007B5074BCB
:10F438001B7840BAADF804002BB9022201A940F2AA
:10F44800BC60FFF7D9FF03B05DF804FBAF1C0020D8
:10F4580007B5074B1B7840BAADF804002BB9022258
:10F4680001A940F2BE60FFF7C7FF03B05DF804FBD7
:10F47800AF1C002010B51346EFF3108472B60A468D
:10F4880001460348F7F71FF884F3108810BD00BF42
:10F498003802002010B51346EFF3108472B60A46FE
:10F4A80001460348F7F701F984F3108810BD00BF3F
:10F4B800380200200A4601460020FFF7EBBF000093
:10F4C80010B51346EFF3108472B60A460146034896
:10F4D800F7F71EF984F3108810BD00BF380200202A
:10F4E80010B51346EFF3108472B60A460146034876
:10F4F800F7F724F884F3108810BD00BF3802002005
:10F5080013B504460020F4F71DFC0220FFF744FF62
:10F5180004F0070401220DF1070184208DF807404B
:10F52800FFF7DEFF024B00221A7002B010BD00BFC9
:10F53800AE1C002007B501228DF807000DF1070168
:10F548008020FFF7CDFF9DF80730002B034B0CBF41
:10F55800012202221A7003B05DF804FBAE1C0020E1
:10F5680007B5094B8DF8060004221A70030C8DF8B4
:10F5780004300322030A01A983208DF80530FFF720
:10F58800AFFF03B05DF804FBAE1C002010B51446B5
:10F59800FFF790FF2046BDE81040FFF7E1BF0000ED
:10F5A80007B5094B8DF8060005221A70030C8DF873
:10F5B80004300322030A01A982208DF80530FFF7E1
:10F5C8008FFF03B05DF804FBAE1C002073B5002666
:10F5D80040F6E2000196FFF7CFFE00F0FE01054677
:10F5E80040F6E200FFF7B8FE40F6E500FFF7C4FE7C
:10F5F80000F07F01044640F6E500FFF7ADFE6FF02E
:10F608007F40FFF7CDFF04220DEB020140F6190001
:10F61800FFF730FF3046FFF78DFF294640F6E2003E
:10F62800FFF79AFE214640F6E500FFF795FE0198A0
:10F6380002B070BD13B50C4B04460522972140F665
:10F64800AC001A70FFF788FE230C8DF804300322F3
:10F65800230A01A982208DF805308DF80640FFF7AE
:10F668003FFF02B010BD00BFAE1C002007B5030C61
:10F678008DF80030030A8DF801300B0C49BA8DF86B
:10F688000200ADF804100622694694208DF8033074
:10F69800FFF726FF024B06221A7003B05DF804FB41
:10F6A800AE1C0020002208B51146C520FFF718FF40
:10F6B800014B07221A7008BDAE1C0020002211461B
:10F6C800D120FFF70DBF00221146D220FFF708BF57
:10F6D80007B501228DF807000DF107019F20FFF7FC
:10F6E800FFFE03B05DF804FB07B501228DF80700A3
:10F6F8000DF10701A020FFF7F3FE9DF807103F2941
:10F7080007D901F0F8010131C9B240F20670FFF7DC
:10F7180023FE03B05DF804FB07B5F4F739FB431E7D
:10F72800584258418DF8070001220DF10701962033
:10F73800FFF7D6FE03B05DF804FB07B500F07F00C5
:10F748008DF8070001220DF107018920FFF7C8FE97
:10F7580003B05DF804FB0000154B984207B51BD8B1
:10F76800144B98421BD8144B98421BD8134B984201
:10F778001BD8134B984295BF29226B222B236F234A
:10F788008DF8042001A9022298208DF80530FFF792
:10F79800A7FE03B05DF804FBE122E923F0E7D722D6
:10F7A800DB23EDE7C122C523EAE775228123E7E7DA
:10F7B80000E9A43580F8A9328044E52D000B6B1BC5
:10F7C80040FC541907B58DF8062004228DF8040072
:10F7D8008DF8051095200DEB02018DF80730FFF725
:10F7E8007FFE03B05DF804FB07B552BAADF80420FC
:10F7F80040BA082249BAADF80000ADF802105BBA69
:10F8080069461046ADF80630FFF76AFE03B05DF8AA
:10F8180004FB07B50B0C042200F0070049BA8DF869
:10F828000400ADF8061097200DEB02018DF80530A5
:10F83800FFF756FE03B05DF804FB000010B508B1F1
:10F84800194B1860F2F77CFF0220FFF7A5FD002492
:10F85800164B20461C70FFF76DFEF4F797FA012847
:10F8680017D14FF42071FFF7D4FF40F6111021464D
:10F87800FFF772FD4FF07F00FFF75FFF0E2140F6A4
:10F888001F10FFF769FDF4F729FA094B01221A70D6
:10F8980010BD102140F61110FFF75EFD102140F653
:10F8A8001210FFF759FDE9E7B01C0020AC1C00203E
:10F8B800AE1C002037B50C4D2B7804461BB9FFF75A
:10F8C8004BFF01232B700023084A6006E109F2F779
:10F8D8001BF9042200BA01900DEB02018620FFF704
:10F8E800FFFD03B030BD00BFAC1C00200048E8019C
:10F8F80007B5094B8DF807000146187018B940F292
:10F90800AC60FFF729FD01220DF107018A20FFF7FE
:10F91800E7FD03B05DF804FBAF1C0020012873B5B8
:10F928000C46164637D10020F4F734FAA042B8BF87
:10F9380044B20E2805461AD101231A460021042094
:10F94800FFF740FF6FF010039C42B8BF1C46182118
:10F9580040F6E700FFF700FD022201A98E208DF88E
:10F9680004408DF80560FFF7BBFD02B070BD0123B0
:10F978000A28E4B21A464FF0000105D11846FFF7ED
:10F9880021FF033464B2DDE70720C5F10E05FFF758
:10F9980019FF2C44F6E740F6D800FFF7EDFC40F0DD
:10F9A8001E01C9B240F6D800FFF7D6FC0120F4F7D3
:10F9B800F1F9A042B8BF44B2142805464FF001033C
:10F9C8004FF000020CD105210320FFF7FBFE0234A3
:10F9D80064B26FF008039C42B8BF1C463821B7E7F1
:10F9E800112805D103210220FFF7ECFE0534EFE7CB
:10F9F8000E2804D102210846FFF7E4FEE9E7C5F125
:10FA08001605072104202544FFF7DCFE6CB2E0E769
:10FA180013B5314A0446516810686B4603C32F4B2F
:10FA280020781B78834201D0FFF762FF2378032BED
:10FA380027D8DFE803F00239283C6268284BB3FB7B
:10FA4800F2F31A0CA1688DF800208DF802301A0A1A
:10FA5800237B8DF80330637B8DF801208DF804300B
:10FA6800204A00234806C909F2F74EF8030C40BAA9
:10FA78008DF80530ADF80600082269468B20FFF79F
:10FA88002FFD02B010BD2269154BB3FBF2F31A0C1F
:10FA98008DF800208DF802301A0A237D8DF8012098
:10FAA8008DF803300422E8E7A3690093FAE7626857
:10FAB8000B4BB3FBF2F31A0C8DF800208DF80230D3
:10FAC8001A0A237B8DF80330637B8DF801208DF8AB
:10FAD80004300522D1E700BFB00C0108AF1C00209C
:10FAE8000000093D0048E8011FB52E4A0446D168C8
:10FAF8009068127C01AB03C31A702B4B20781B78DB
:10FB0800834201D0FFF7F4FE2378032B26D8DFE8E1
:10FB180003F002383302637AF12B21D14FF6FF70DC
:10FB2800FFF784FC48F20500FFF792FC0223628885
:10FB3800A188ADF8061052BAE188ADF804208DF816
:10FB48000B30227AA37A8DF80A20ADF808108DF8C8
:10FB58000C30092201A98C20FFF7C2FC04B010BDAB
:10FB6800F22BE4D141F60F50FFF760FC41F221007F
:10FB7800FFF76EFC0623DAE7237B8DF804300122B9
:10FB8800E8E7E389094A5BBAADF80430237C1370CF
:10FB98008DF80630637C8DF80730638AADF808303D
:10FBA8000622D7E7B00C0108AF1C0020AD1C0020CE
:10FBB80007B502228DF804008DF805108F2001A9E1
:10FBC800FFF78EFC03B05DF804FB000010B5134688
:10FBD800EFF3108472B60A4601460348F6F7E6FCCE
:10FBE80084F3108810BD00BF3802002007B5012239
:10FBF80001A91520FFF7EAFF9DF8040040424010D4
:10FC080003B05DF804FB000037B505460C46022238
:10FC180001A91320FFF7DAFF0A4B1B78012B0DD13E
:10FC2800094B1B78012B09D140F20270FFF7A4FBA6
:10FC38009DF805302870237003B030BD9DF804008E
:10FC4800F6E700BFAF1C0020AD1C0020F7B50D463D
:10FC5800064600240DF10701284617468DF807408F
:10FC6800FFF7D2FF2A78BA4207D89DF80700314635
:10FC7800FFF726FC204603B0F0BD0120FBE700009B
:10FC880013B50322044601A91420FFF79FFF184B60
:10FC98001A7822704AB1012A17D01422002120466E
:10FCA80000F0D2FA0F2323700DE09DF80430237181
:10FCB8009DF80530A2605B425B10A3719DF8063089
:10FCC8005B425B10637102B010BD9DF804305B426B
:10FCD8005B1023739DF9053002339B1063739DF805
:10FCE80006305B425B10A373024B1B682361EAE793
:10FCF800AF1C0020A81C0020012908B503460846AF
:10FD08000ED1012B07D10420FFF746FB0220BDE8E6
:10FD18000840F4F717B8022B14BF08460320F6E78B
:10FD28000120F4E738B50446F4F72EF850B102285C
:10FD380014BF01250225284602222146FFF7EEFDC1
:10FD4800284638BD0F2CCCBF02250125F3E70A2031
:10FD580070470000014B01201B681847B01C0020A9
:10FD6800014B02201B681847B01C0020014B4020A3
:10FD78001B681847B01C002011B1012904D0704736
:10FD8800044B1B6880201847024B4FF480701B6897
:10FD9800F9E700BFB01C0020024B4FF400701B684D
:10FDA800184700BFB01C0020014B20201B681847D3
:10FDB800B01C0020014B04201B681847B01C002011
:10FDC800014B08201B681847B01C0020014B10206D
:10FDD8001B681847B01C0020024B4FF480401B687A
:10FDE800184700BFB01C002068B1084A002352F829
:10FDF8003310814203D902EBC302107970470133F3
:10FE0800162BF4D1FEE71F20704700BFA416010887
:10FE180073B51D4B0193044640F607000D46FFF7E6
:10FE2800ABFAC0F3C10308336B4413F8042C00F099
:10FE38000703013302FA03F3144AB2FBF3F2B2FBED
:10FE4800F4F007281ED8400003288CBF022304239F
:10FE58004FF4D66002FB03F4FFF78EFA060240F275
:10FE6800B160FFF789FA06F470663043030544BFB2
:10FE78006FEA00506FEA105063094343DB112B60AF
:10FE880002B070BD0123E3E704080A0C0048E8014A
:10FE98004FF0FF3070474FF0FF3070474FF0FF30A2
:10FEA80070477047002070470020704770474FF038
:10FEB800FF3070474FF0FF3070477047704770470A
:10FEC80070B5EFF3108672B6144B5C8A1A8A9442A6
:10FED80013D1C4F5806292B2904206D3844218D9F5
:10FEE80001229A7000221C805A825A8A0A8002448F
:10FEF800C2F309025A8200200DE006D9C4F58065D4
:10FF0800ADB28542F1D88242E9E7121B92B2824231
:10FF1800EBD84FF0FF3086F3108870BDB420002076
:10FF2800EFF3108172B6034AD38A0133D38281F387
:10FF380010887047B4200020EFF3108172B6034A8E
:10FF4800D38A013BD38281F310887047B420002004
:10FF580010B508481822002100F076F906484FF439
:10FF68008062002100F070F9044B05481B68BDE869
:10FF780010401847B4200020B41C0020500D010880
:10FF8800F9000108014B5860704700BFB4200020F9
:10FF9800014B1872704700BFB420002073B5EFF30F
:10FFA800108572B61C4CE08A00282FD1FFF7B8FFE5
:10FFB800218A628A914227D0A378012B12D1238803
:10FFC80020805B1A9BB20221A382A17063B9A3703F
:10FFD8002382238A9A428BBFD21AC3F58063A282F6
:10FFE800A38201E0002BF4D0238A0C4E1E4485F333
:08FFF8001088F2F793FC0A4B9C
:020000040801F1
:10000000A18ADB680193304602B0BDE87040184712
:10001000FFF796FF85F31088002002B070BD00BF87
:10002000B4200020B41C0020500D010808B4F0B525
:1000300086B00023ADF800302C4B0B9C1D7A854216
:100040004DD3D86881434DD15B681BB112B169466D
:1000500002A898470CAB22464FF400712448019344
:1000600000F0F6FBFFF760FFBDF8003018440DF11B
:10007000020180B2FFF728FF01302BD00022BDF82B
:100080000030BDF802701B480DF1080C164691B205
:1000900017FA82F58B42ADB216D83B449BB20EB133
:1000A000ADF80230BDF80250019B22464FF40071BA
:1000B000284400F0CDFBFFF743FFFFF773FF06B0C6
:1000C000BDE8F04001B070471CF8011B41550132FA
:1000D0000126DCE7FFF734FF6FF00200EFE76FF077
:1000E0000400ECE76FF00500E9E700BFB420002052
:1000F000CC200020B41C002013B5EFF3108472B69E
:10010000204B9A78588A022A1DBF1A8A998A521857
:10011000002214BFC2F309029A7090421A8228D0BA
:10012000D98A012925D19978012913D119888A1AE8
:10013000022192B2997000219A82198062B99A7054
:100140001A821A8A90428BBF801AC2F58062988206
:100150009A8201E00029F4D01A8A0B48104484F3F3
:1001600010880A4A998AD368019302B0BDE810400A
:10017000184784F31088F2F7D9FB02B0BDE81040AD
:10018000FFF7DEBEB4200020B41C0020500D010893
:10019000024A00231360024A13607047D0220020F5
:1001A000CC22002010B5EFF3108472B641B10129C2
:1001B00003D1064A13680343136084F3108810BD0B
:1001C000024A136823EA0003F6E700BFD0220020AA
:1001D00010B5EFF3108472B641B1012903D1064A7C
:1001E00013680343136084F3108810BD024A136838
:1001F00023EA0003F6E700BFCC22002038B5EFF376
:10020000108572B60A4B0B4C1B6833B123689847B4
:100210006368984785F3108838BD074B1B681BB18E
:10022000A3689847E368F4E7236998476369F0E7B0
:10023000D0220020DC0C0108CC22002001380A4426
:10024000914200D1704711F8013B00F8013FF7E7F8
:1002500000F02CBC10B5EFF3108472B6064A136898
:1002600003431360054A52F83130034342F83130FA
:1002700084F3108810BD00BF202300201823002025
:1002800070477047030C1B04C3B90004102310F01F
:100290007F4F02BF08330002DBB210F0704F08BF7F
:1002A00000014FEA1070064A08BF0433125C08BF11
:1002B000DBB2C3F11F03981AC0B270470023E6E710
:1002C000541701082DE9F84F384D394ED5F8008004
:1002D000DFF8E0B0DFF8E0A0DFF8E090D6F800C08B
:1002E000374FDBF80010374CDAF80020D9F800302F
:1002F00008EA00002860286800EA020E1EEA0C0FD7
:1003000001D019421ED04FF0FF333B60FFF7B8FF1A
:10031000EFF3108472B63368DBF80020DAF80010CF
:100320000B4029680B4205D1D9F80030134201D1A6
:10033000F2F786FA84F31088FFF7A3FFC5F8008070
:10034000BDE8F88F236823680340134062681A42AF
:1003500004BF4FF0FF32626060681840FFF792FF01
:1003600062683860012303FA00F022EA000262604A
:10037000EFF3108172B63A689340326822EA0302C2
:100380003260226822EA0303236081F310880E4A58
:100390003B6852F823309847D6F800C0DBF80010CD
:1003A000DAF80020D9F80030A5E700BF44010020AA
:1003B00020230020D822002048010020DC22002039
:1003C000D422002018230020E022002010B511467E
:1003D000EFF3108472B6FFF755FF034B43F820107C
:1003E00084F3108810BD00BFE022002082B082B0EC
:1003F0000DF1080C0CE90600BDF8042003930B4432
:10040000BDF810100A4491B212B2B2F57A7FA2BFC1
:10041000A1F57A72013312B20360828002B002B099
:10042000704782B082B00DF1080C0CE90600BDF8EF
:1004300004200393CB1ABDF81010521A91B212B2D5
:10044000002ABEBF01F57A7203F1FF3312B20360D6
:10045000828002B002B0704730B585B0114D6B4656
:1004600083E8030000230293ADF80C3003A82B6946
:100470009847009BBDF804400290181ABDF80C3054
:10048000E41AA3B224B2002CBEBF03F57A731CB2E7
:1004900000F1FF302B689847AB682046984705B0BD
:1004A00030BD00BF100D010873B5114E0023054685
:1004B0000093ADF8043001A833699847F3680090C1
:1004C0009847736804469847009B1844BDF8043069
:1004D00023449AB21BB2B3F57A7FA2BF0130A2F5D2
:1004E0007A731BB228602846AB8002B070BD00BF93
:1004F000100D010837B500230093ADF80430074B09
:1005000004461B6901A898476D46009095E80300D2
:1005100084E80300204603B030BD00BF100D010881
:1005200037B50F4D02AB03E90300EB6898476B68E2
:1005300004469847BDF80430009A1B1B99B21BB2C1
:10054000002BA2EB0002BEBF01F57A7102F1FF326F
:100550000BB24FF47A7000FB023003B030BD00BF25
:10056000100D01082DE9F0414FF47A75B1FBF5F556
:10057000C5EB4513DFF83C8005EB8303A1EBC30318
:100580009CB2D8F80C3006469847D8F80430074695
:100590009847E31999B21BB2B3F57A7F2844A2BFFA
:1005A000A1F57A7301301BB23060B3803046BDE8EC
:1005B000F08100BF100D0108024B00221A60024BAF
:1005C0001B68184724230020240D0108F8B50446B1
:1005D000174608461E467CB173B1084B00255B6A7E
:1005E00025609847069B60602581A572E6602361BF
:1005F000E77265612846F8BD0120FCE7240D01087B
:1006000010B5034CE3699847A36ABDE8104018474A
:10061000240D010870B5064DEB69064698476B6AD4
:10062000044630469847AB6A201ABDE87040184728
:10063000240D0108054B1B680BB91846704783420F
:1006400001D05B69F8E70120704700BF2423002038
:100650002DE9F3410B4E336A044698470123B769ED
:100660002372D4F800800546B8472844804502D25A
:10067000B84728442060B3682068019302B0BDE801
:10068000F0411847240D010870B520B3EFF3108630
:1006900072B6124D2B680122827253B1002242724F
:1006A00098425C690ED102723CB120462C60FFF783
:1006B000CFFF86F31088002070BD094BDB68984798
:1006C0002C60F6E71A465B69002BF2D09842F9D10C
:1006D00043695361EDE70120EEE700BF24230020CA
:1006E000240D0108084B10B51A685369516911B9F6
:1006F0005061416110BD046819688C4202D91A46E4
:100700005B69F3E71946F3E724230020044A1368E2
:100710000BB10021197243611060FFF799BF00BF50
:10072000242300202DE9F041044600282DD0FFF7B6
:1007300081FF50BB657A45BBEFF3108872B6144E4B
:100740006768336A984787422CBF27602060114F43
:10075000A5724FF4807323813B684BB93369984786
:100760002046FFF7D3FF88F310882846BDE8F081C4
:10077000B3699847236818443B6820601B68984217
:100780002046EED3FFF7AEFFEDE70125EDE700BF12
:10079000240D01082423002010B5044608467CB12E
:1007A000084B5B6A984760602046FFF743FF40B103
:1007B0002046FFF769FF2046BDE81040FFF7B2BFB3
:1007C000012010BD240D01082DE9F041EFF3108741
:1007D00072B61D4E1D4D736998473369044698479C
:1007E0002B684BB94FF000082B688BB9286828BBE1
:1007F00087F31088BDE8F081011B241A1A688A4229
:100800008CBF121900221A605B69002BF6D1E9E750
:100810001C681CB1B36998478442E7D22C686369AD
:100820002B60A4F80880D4E9033098476389B3F5B6
:10083000807FD9D12046FFF775FFD5E7037A002BDB
:10084000D6D1FFF705FFD3E7240D010824230020AC
:100850002DE9F04F97B000298046039140F30E81B7
:100860009A46044603991378A4EB0800013923B98A
:100870000023237017B0BDE8F08F8842F8DA252BEB
:1008800004D004F8013B1646721CEBE792F801C055
:10089000ACF13003D3F1000E4EEB030EACF130039C
:1008A000092B02F1010629D8324600254FF00A092A
:1008B000164612F8013BA3F13000092819D9337804
:1008C000692B00F09C801CD8632B28D0642B00F08F
:1008D0009680582B5BD0252B19D13378002B00F054
:1008E000928004F8013BA4EB08038B4280F28980DC
:1008F000CAE709FB0533A3F13005D9E74FF0FF350F
:10090000DDE7752B7DD0782B43D0732B1ED02523AC
:1009100004F8013BA4EB08038B4272DADDE7002DFB
:1009200005F1FF39D8BF4FF000094A462046202183
:1009300000F0BCF85346A144002D53F8042B89F86D
:100940000020D8BF01252C449A469DE74C4B5AF80D
:10095000047B002F08BF1F463846F0F731FDA5EB9A
:10096000000B8542B8BF4FF0000B5A46814620214C
:10097000204600F09BF8A34400234B4502DB0BEB21
:10098000090481E7FA5C0BF803200133F5E74EF028
:10099000400E1020DFF8EC903B4F1EF0400F08BFD8
:1009A0004F465346BCF1300F0197A4EB08020CBF31
:1009B000302720271EF0020FA1EB0202029753F806
:1009C000041B22D0002920DA4942013D4FF02D0EB0
:1009D00005AF009700278946DDF804A0B1FBF0F1D0
:1009E00000FB119B48451AF80BB0DDF800A00AF88F
:1009F00001BB07F10107CDF800A0ECD90EE04EF0E5
:100A0000020E0A20C6E7013E6DE711B14FF0000E5D
:100A1000DEE730208DF814008E460127BCF1300F40
:100A2000A5EB070504D02020002D05F1FF3509DCDA
:100A3000BEF1000F04D02D21013A04F8011B83D030
:100A400025440AE0013A04F8010BEDD17CE7029954
:100A500004F8011B013A3FF477AF291B0029F6DCAB
:100A600005A9394422442744A7423FF46DAF11F849
:100A7000010D04F8010B9442F6D165E70020F9E678
:100A8000641701086B1701089017010810B50139A8
:100A90000244904201D1002005E0037811F8014F93
:100AA000A34201D0181B10BD0130F2E702440346F7
:100AB000934200D1704703F8011BF9E770B50D4D63
:100AC0000D4C641BA4100026A64209D10B4D0C4C02
:100AD00000F0B2F8641BA4100026A64205D170BD38
:100AE00055F8043B98470136EEE755F8043B984724
:100AF0000136F2E7981801089818010898180108BB
:100B00009C18010800F003B8002200F00EB80A4457
:100B1000914200F1FF3300D1704710B511F8014B3D
:100B200003F8014F9142F9D110BD13460A46194608
:100B3000FFF7BCBF00000000C1F30A522DE9F843E3
:100B4000A2F2FF36132E0B4607460C46054632DC52
:100B5000002E14DA34A3D3E90023F0F73FFC00227F
:100B60000023F0F76FFE38B1002C56DA24F0004471
:100B7000254355D02E4C002523462F4625E02D4AEF
:100B800042FA06F801EA080202431ED026A3D3E97E
:100B90000023F0F723FC00220023F0F753FE002887
:100BA000EAD0002CBEBF4FF480133341E41824EA8E
:100BB00008040025E0E7332E0BDDB6F5806F04D185
:100BC0000246F0F70BFC07460B4638461946BDE8CF
:100BD000F883A2F213424FF0FF3828FA02F810EA25
:100BE000080FF2D010A3D3E90023F0F7F7FB00229F
:100BF0000023F0F727FE0028BED0002C0ADA142EBE
:100C000001D1013406E0C6F134060123B3401D448E
:100C1000AF42F6D825EA0805AEE700252C46ABE73B
:100C20004FF00044A8E700BF9C7500883CE4377E85
:100C30000000F0BFFFFF0F00F8B500BFF8BC08BC14
:100C40009E467047F8B500BFF8BC08BC9E4670478A
:100C50000000000001000000020000000000000091
:100C60008813000010270000204E0000307500009F
:100C7000409C000050C3000060EA0000C0D40100A6
:100C800080A903000053070000EA063700000000B7
:100C90005000000040F7093700000000500000003D
:100CA000C194C10000000000B22700000000000055
:100CB0000000000000000000000000000000000034
:100CC00000000000B5010008F1010008C40C010893
:100CD000FC7F003F00350113C41200082F260008D6
:100CE00041260008CD2500081D260008B92500086A
:100CF000C72500085975336E3148344F3152354E8F
:100D0000395332543653256473253033643A000026
:100D1000352A0008D52A0008452A0008E12A0008DB
:100D2000A52A0008ED2A000800000000552A000846
:100D30000D2A0008D929000891290008E92900088E
:100D4000FD2900089D290008A1290008B5290008EF
:100D50005D2D0008852D0008092D0008F52C0008E0
:100D600052464143005056585858002159756E4814
:100D70006F726E2053545320526576697665210058
:100D800006071600010002004000000000000048B5
:100D90000000004800080048D73E0008CD3E00088B
:100DA000C33E0008000000160100001606000016F1
:100DB0000F0000000F0000000F0000000100000005
:100DC0000300000005000000010000000100000019
:100DD000060000000A0000002000000002000000E1
:100DE00004000000080000001000000040000000A7
:100DF0008000000000010000000200000000000070
:100E000000000000000000000000000001000000E1
:100E1000020000000300000004000000A0860100A2
:100E2000400D0300801A060000350C0040420F0000
:100E300080841E0000093D0000127A000024F400A6
:100E400000366E010048E801006CDC020000000082
:100E50000000000000000000000000000402080084
:100E600010101004101010021010100801000200E1
:100E70000400060008000A000C00100020004000DA
:100E800080000001080402040801010101010103BE
:100E9000070100006572726F723A20526567696FD0
:100EA0006E206973206E6F7420646566696E656478
:100EB00020696E20746865204D573A207365742050
:100EC0006C6F726177616E5F636F6E662E68206112
:100ED00063636F7264696E676C790D0A004D4143FC
:100EE00020727854696D654F75740D0A004D414349
:100EF00020747854696D654F75740D0A004D414337
:100F0000207278446F6E650D0A004D41432074785D
:100F1000446F6E650D0A00080A0C0D0E10121415B0
:100F2000181A1B1D1E2124030502050106020205D5
:100F300000000600000105040400000048E801006C
:100F400048E8010048E8010048E8010048E80100DD
:100F500048E8010090D003000000000003000000FA
:100F60000201000C0B0A090807073200000000000C
:100F70000001020100000000000203020100000065
:100F80000003040302010000000405040302010041
:100F90000005060504030201000607060504030216
:100FA00001070707060504030207070202020202FF
:100FB0000202020202020202020203020202020210
:100FC00002030403020202020204050403020202F5
:100FD00002050605040302020206070605040302D1
:100FE000020707070605040302070733337373F28A
:100FF000F2F2F200000B357DF2F2F233337373DE5E
:10100000DEDEDE52585F2573206F6E2066726571DA
:1010100020256420487A2061742044522025640DE4
:101020000A005258206F6E20667265712025642078
:10103000487A2061742044522025640D0A005458D7
:10104000206F6E206672657120256420487A2061C9
:10105000742044522025640D0A00310032004D7581
:101060006C74695F43004D756C74695F50000000DB
:101070005A1001085C100108630D01085E10010898
:101080006C10010866100108C6F8EEF6FFD6DE9176
:101090006002CE56E7B54DEC8F1F89FAEFB28EFB9A
:1010A00041B35F452353E49B75E13D4C6C7EF58372
:1010B0006851D1F9E2AB622A0895469D30370A2F74
:1010C0000E241BDFCD4E7FEA121D583436DCB45B94
:1010D000A476B77D52DD5E13A6B900C140E379B6B0
:1010E000D48D67729498B085BBC54FED869A661112
:1010F0008AE904FEA078254BA25D80053F2170F1AE
:101100006377AF4220E5FDBF811826C3BE35882E28
:101110009355FC7AC8BA32E6C0199EA344543B0BDF
:101120008CC76B28A7BC16ADDB647414920C48B84E
:101130009FBD43C43931D3F2D58B6EDA01B19C49DE
:10114000D8ACF3CFCAF447106FF04A5C38577397A6
:10115000CBA1E83E96610D0FE07C71CC9006F71CA8
:10116000C26AAE6917993A27D9EB2B22D2A9073365
:101170002D3C15C987AA50A50359091A65D784D0F3
:1011800082295A1E7BA86D2CA584998D0DBDB15462
:101190005003A97D1962E69A459D408715EBC90B5E
:1011A000EC67FDEABFF7965BC21CAE6A5A41024F7C
:1011B0005CF434089373533F0C52655E28A10FB55D
:1011C00009369B3D2669CD9F1B9E742E2DB2EEFBEA
:1011D000F64D61CE7B3E7197F568002C601FC8ED1F
:1011E000BE46D94BDED4E84A6B2AE516C5D75594DE
:1011F000CF100681F044BAE3F3FEC08AADBC4804C8
:10120000DFC17563301A0E6D4C14352FE1A2CC3955
:1012100057F28247ACE72B95A098D17F667EAB83CF
:10122000CA29D33C79E21D763B564E1EDB0A6CE49C
:101230005D6EEFA6A8A4378B324359B78C64D2E019
:10124000B4FA0725AF8EE918D5886F7224F1C7511B
:10125000237C9C21DDDC86859042C4AAD80501123E
:10126000A35FF9D0915827B93813B333BB7089A75E
:10127000B622922049FF787A8FF88017DA31C6B803
:10128000C3B07711CBFCD63A637C777BF26B6FC52A
:101290003001672BFED7AB76CA82C97DFA5947F079
:1012A000ADD4A2AF9CA472C0B7FD9326363FF7CC55
:1012B00034A5E5F171D8311504C723C31896059AF2
:1012C000071280E2EB27B27509832C1A1B6E5AA015
:1012D000523BD6B329E32F8453D100ED20FCB15B00
:1012E0006ACBBE394A4C58CFD0EFAAFB434D338569
:1012F00045F9027F503C9FA851A3408F929D38F53D
:10130000BCB6DA2110FFF3D2CD0C13EC5F97441773
:10131000C4A77E3D645D197360814FDC222A9088EA
:1013200046EEB814DE5E0BDBE0323A0A4906245C76
:10133000C2D3AC629195E479E7C8376D8DD54EA9DB
:101340006C56F4EA657AAE08BA78252E1CA6B4C6A7
:10135000E8DD741F4BBD8B8A703EB5664803F60E00
:10136000613557B986C11D9EE1F8981169D98E94EF
:101370009B1E87E9CE5528DF8CA1890DBFE6426808
:1013800041992D0FB054BB1623232323232320255B
:101390007320253032583A253032583A25303258A9
:1013A0003A253032583A253032583A253032583AB8
:1013B000253032583A253032583A253032583A25BD
:1013C0003032583A253032583A253032583A2530A2
:1013D00032583A253032583A253032583A25303290
:1013E000580D0A00232323232323204465764555E3
:1013F000493A202020202020253032583A2530320A
:10140000583A253032583A253032583A2530325839
:101410003A253032583A253032583A253032580D74
:101420000A00232323232323204170704555493A82
:10143000202020202020253032583A253032583ABA
:10144000253032583A253032583A253032583A252C
:101450003032583A253032583A253032580D0A0089
:1014600023232323232320446576416464723A2096
:1014700020202020253032583A253032583A253065
:1014800032583A253032580D0A004170704B657958
:101490003A2020202020004E776B4B65793A20209F
:1014A000202020004E776B534B65793A2020202076
:1014B00000417070534B65793A202020200044424F
:1014C000496E744B65793A202020004D43526F6F6E
:1014D000744B65793A2020004D434B454B65793A72
:1014E00020202020004D43417070534B65795F30C0
:1014F0003A004D434E776B534B65795F303A0000AD
:10150000000000004150505F8A14010801000000F3
:101510004E574B5F97140108080000004E574B537D
:10152000A41401080900000041505053B1140108EF
:101530000A0000004442495FBE1401080B0000008D
:101540004D435254CB1401080C0000004D434B4551
:10155000D81401080D0000004D434B30E51401087C
:101560000E0000004D415330E51401080F0000004B
:101570004D4E5330F2140108100000005A45524FEE
:10158000BF150108526164696F53656E64204F7620
:10159000657273697A650D0A004952515F52585F4E
:1015A00054585F54494D454F55540D0A005052450B
:1015B000204F4B0D0A0053594E43204F4B0D0A004C
:1015C000484452204F4B0D0A00484452204B4F0DC7
:1015D0000A004952515F4352435F4552524F520DE8
:1015E0000A00040506000000841E0000093D0000FA
:1015F000127A000024F4000048E8010090D00300B3
:1016000020A1070000000000B12800006151000087
:10161000C3A2000002010003FDE20008C1E10008CE
:10162000F9E300083DE2000825ED0008E5E20008C6
:1016300051EA0008C9E80008A1E0000861EF0008CD
:10164000A1ED0008D1E20008B9E1000869E2000854
:1016500041E20008F9E10008EFE10008F1E00008CC
:10166000EDE00008EBE10008E7E1000891E3000885
:10167000BDE30008DDE100087DF0000851E100084D
:1016800019E100084DF00008F5E00008C1E6000887
:1016900045E4000899FE00089FFE0008E5E0000808
:1016A000E9E00008C01200001F000000A8160000BA
:1016B00017000000841C00000F000000E42500005B
:1016C0001E000000B42D00001600000008390000C4
:1016D0000E0000002C4C00001D000000685B0000A4
:1016E00015000000747200000D0000005898000002
:1016F0001C00000034B7000014000000E8E4000003
:101700000C000000783101001B000000686E010031
:101710001300000034CA01000B0000002862020020
:101720001A00000040DB0200120000003C9303009E
:101730000A000000C0C204001900000060B30500E8
:1017400011000000382007000900000020A1070058
:10175000000000000403020201010101000000007A
:10176000000000003C4E554C4C3E003031323334CA
:1017700035363738396162636465666768696A6BF4
:101780006C6D6E6F707172737475767778797A009C
:1017900030313233343536373839414243444546A7
:1017A0004748494A4B4C4D4E4F5051525354555651
:0817B0005758595A00000000CF
:1017B8000000000000000000000000000000000021
:1017C8000000000000000000002B7E151628AED295
:1017D800A6ABF7158809CF4F3C012B7E151628AE0E
:1017E800D2A6ABF7158809CF4F3C082B7E151628D3
:1017F800AED2A6ABF7158809CF4F3C092B7E15163C
:1018080028AED2A6ABF7158809CF4F3C0A000000D6
:10181800000000000000000000000000000B0000B5
:1018280000000000000000000000000000000C00A4
:101838000000000000000000000000000000000D93
:101848000000000000000000000000000000000090
:101858000E00000000000000000000000000000072
:10186800000F000000000000000000000000000061
:101878000000100000000000000000000000000050
:08188800000000000000000058
:08189000B002FF7F010000001F
:041898005D010008E6
:04189C003901000806
:1018A000020000000000000052030020C0D401002C
:1018B00045280008752800088D280008F928000828
:1018C000453000081D300008792F00084F3200080D
:1018D00000000000E52F00084D2F0008113C000813
:1018E000312F00082F2F000855320008812F0008E3
:1018F000352F0008412F00081932000800000100B0
:1019000000000000000000000000000004000000D3
:10191000401F00001027000000180101054D3C4D3C
:101920000400002008190F28040A413F00050A019D
:101930000000050203FFFFFFFFFFFFFFFFFFFF0F98
:101940000103000200000000000000000000000091
:10195000000000000000000000093D001000000031
:10196000A80600200000FF000000000000000000AA
:10197000A80600200000000000000000FF0000009A
:1019800000000000A8060020000000000000000089
:10199000000000000000000000000000E000000067
:1019A00081830008B1820008BD820008E982000836
:1019B0000000000000000000D9830008C982000870
:1019C000498700080000000000000000000000003F
:1019D00000000000000E0F0D0109081101000000B9
:0C19E000FF000000FFFFFFFFFFFFFFFF04
:0400000508003DA909
:00000001FF
